:020000040000FA
:10000000F8050820954E0200994E02009B4E020012
:100010009D4E02009F4E0200A14E02006222EADFC6
:10002000000000000000000000000000A34E0200DD
:10003000A54E020000000000A74E0200A94E0200DB
:10004000AB4E0200AB4E0200C5D90200AB4E02001F
:10005000AB4E02004DBF0200E9C1020039C40200EC
:10006000AB4E0200AB4E0200AB4E0200AB4E0200A4
:10007000AB4E0200AB4E0200AB4E0200AB4E020094
:10008000AB4E0200AB4E0200AB4E0200AB4E020084
:10009000AB4E0200F7DF0200AB4E0200AB4E020097
:1000A000C5F60200AB4E0200AB4E0200AB4E0200A2
:1000B000AB4E0200AB4E0200AB4E0200AB4E020054
:1000C000AB4E0200AB4E0200AB4E020000F002F855
:1000D00000F088F80AA090E8000C82448344AAF15A
:1000E0000107DA4501D100F07DF8AFF2090EBAE858
:1000F0000F0013F0010F18BFFB1A43F0010318475C
:10010000E4AF040024B004000A444FF0000C10F8DF
:10011000013B13F0070408BF10F8014B1D1108BF85
:1001200010F8015B641E05D010F8016B641E01F825
:10013000016BF9D113F0080F1EBF10F8014BAD1C75
:100140000C1B09D16D1E58BF01F801CBFAD505E093
:1001500014F8016B01F8016B6D1EF9D59142D6D3ED
:10016000704700000023002400250026103A28BF15
:1001700078C1FBD8520728BF30C148BF0B60704719
:10018000692939F00386642939F00086752939F028
:10019000FD856F2939F09486782939F0BB8603688C
:1001A000DB0928BF41F0800163293AF01E837329DF
:1001B0003AF02383E3293AF02E83002070471FB5DD
:1001C0009DE803003AF048FA39F0EBFF3AF02AFADA
:1001D0000400002000213AF0A3FF401C60601FBD16
:1001E00010B510BD3AF003FC1146FFF7E8FF00F030
:1001F0001DF93AF021FC03B4FFF7F2FF03BC3AF01B
:1002000051FC00000B49D1F800C04A685CF8043B7F
:100210001068184442F8040B8C4528BFA1F1DC0C8F
:100220008A4228BFA1F1DC02C1F800C04A6020F078
:10023000004070479005001010B5782119483AF039
:10024000BFF919494FF0FF30088010BD16480188EA
:10025000491C09B201800A290CD001EB4102114965
:10026000436841F8223001EB820183684B60C0682B
:1002700088607047FEE70C4910B5B1F90000421CD8
:100280000ED0084A00EB4003401E52F8234002EB18
:1002900083024C6053688B609268CA60088010BD0E
:1002A000FEE700004C0300100400001010B51CF025
:1002B000E4FE05281FD12DF07EFEE0B905F031FBEC
:1002C000C8B9002038F07AFFA8B9012038F076FFCD
:1002D00088B9022038F072FF68B9032038F06EFF49
:1002E00048B907202BF0D6FD052804D107202BF0B4
:1002F000D1FD052807D02DF05EFE00280AD1BDE80B
:1003000010402DF061BE0448406DC0F3C0202DF0B8
:100310005BFE30BF10BD000000C0092030B50246B2
:100320004FF6FF7318460E4C08E000BF12F8015B51
:1003300085EA1025655D85EA002080B2491E89B2F4
:10034000F4D2584030BD024610B5FF20002905D038
:10035000044B545C4440491E185DFAD110BD0000A6
:100360000AC4030040C0072038B50546684605F0BA
:1003700065FD0D4C000611D49DF80000032809D03E
:1003800087200A49206000200860784608490860F4
:10039000872038BD0CF0CCF9000601D5206838BDA7
:1003A000284608F0F9FD38BD080000100C000010C8
:1003B0001000001038B50446684605F03FFD010600
:1003C0000A4801D5006838BD9DF80010032909D0FE
:1003D00087210160064900200860784605490860C9
:1003E000872038BD204608F0C9FE38BD080000103F
:1003F0000C00001010000010014601202CF04FB935
:10040000B00C112C7B1B00000048704798050010B1
:100410004D617920313720323031360070477047D6
:1004200031353A34333A33390000000088B0C24CD9
:100430000027039720883E4640F002002080BF48F6
:1004400026F009F9BE48007802281CD1FFF7FEFE0D
:1004500003A824F0BDFF000601D502F0C2FDFFF79E
:100460000AFF0398B0F58C7F0DDAFFF7EFFE00214D
:10047000B4A02EF03FFA000601D502F0B2FDFFF75E
:10048000FAFE02F0AEFDAD4D288830F4504010D099
:100490000127FFF7DBFE32201AF091FE012012F057
:1004A000DDF910B103202EF002FCFFF7E4FE02F0AC
:1004B00098FD2888810B06D001270FF01DF9000652
:1004C00001D502F08EFD2E801EF0DAFD000601D56A
:1004D00002F087FD01F0CCF906F076FC000601D5AC
:1004E00002F07FFDA24DAE6805A825F0F8FF01F0EF
:1004F00077F910B1012702F074FD01F0FBF9DFF884
:100500007482C0B1FFF7A2FE01F04CFBFFF7B3FE0F
:10051000D8F80000062802D0002197A004E09B49EB
:100520000220087000219AA02EF0E4F9208840F003
:10053000020020800CE001F0FAFB38B1FFF786FEE4
:1005400001F030FBFFF797FE02F04BFD01F07CFE5F
:100550009448A968891B8142FBD306A825F0BFFFF8
:10056000914EDFF84892307800EB400159F83100A5
:100570008047000601D502F034FD01F0CBFE0006F5
:1005800001D502F02EFD9DF81A009DF81610884244
:1005900001D0012000E0002001F0FEFE00B10127A3
:1005A00001F058FF00F0DEFC02A953201AF072FFA0
:1005B000000601D502F015FD9DF8080000F00100CD
:1005C0008DF808006FB9B0B1012012F047F90006AC
:1005D00001D502F006FD11F0DBFC000601D502F0AA
:1005E00000FD9DF8080030B1012012F037F9000637
:1005F00001D502F0F6FC24F099FD4F464FEA0D09B3
:1006000038F036FB2CF0FCFB307800EB400007EBB9
:10061000C000C0688047000601D502F0E2FC3078D7
:1006200000EB400007EBC00040688047000601D5A2
:1006300002F0D7FC307800EB400007EBC000806888
:100640008047000601D502F0CCFC00202DF008FE0A
:10065000D8F800000C2805D005F094F8000601D564
:1006600002F0BFFC207840071ED501202DF0F8FDD8
:10067000D0B9684605F06DFC50B909F1020005F0EB
:1006800079FC28B909F1040005F085FC000601D5C4
:1006900002F0A7FC46499DF804000870684606F081
:1006A000DFFD08B907F058FC33F0FAFB207810F0B2
:1006B000B80F35D001202DF0D3FD000630D4A86846
:1006C0003C49AA68121A8A42FBD32078000701D558
:1006D00011F008FD2088010614D5810612D4C00649
:1006E00013D411F059FD000601D502F07AFC002068
:1006F00007F01CFD000601D502F073FC208820F0F5
:10070000810020802078C00601D506F04BFD2078BE
:10071000800605D5012009F023FC012012F09EF887
:1007200024F066FD000601D502F05BFC2EF0AAFB6A
:10073000FFF7BCFD64E700000200001000C00720C6
:10074000BC0100108E9888818A80208180928090E0
:100750008588209780918E820A8E819080928892DF
:1007600085919C20822096928E0A0A0A0A00000037
:10077000008000400C0000108E9888818A80208FB5
:10078000808C9F9288208F840A0A0000000000104D
:10079000878D208D852082828584858D0A0A0A0AAC
:1007A0000A000000E0C810009EC20720A0C2072077
:1007B00091C20720A08601002DE9F047FD4DFE4EB5
:1007C000FE4F9046C3B15C1E0BD4DFF8F493642255
:1007D000002339F0ABF919F8023008F80430641E30
:1007E000F5D5084310D08920286004203060784671
:1007F00038608920BDE8F0878820286009203060B3
:10080000784638608820F5E7002028603060784618
:1008100038600020EEE710B500220BE0835C03F0A7
:100820000F04092C03D803F0F003902B01D900200A
:1008300010BD521C8A42F1D3012010BD2DE9FF4F9B
:10084000DC4CDD4DDD4E83B08246082A30D872B3D1
:100850000020CDE9000001214FF0860B4FF0200E63
:100860000AEB020313F8019C09F00F03092B14DCB7
:10087000A1FB03784FEAD37C00FB038301FB0C331D
:10088000DDE9008C18EB07074CEB030CCDE9007C8D
:100890004FEA1919B9F1090F12DDC4F800B0784612
:1008A000C5F800E03060862007B0BDE8F08FFFE7B4
:1008B0008820206009202860784630608820F3E78F
:1008C0004FF00A0CA1FB0C3800FB0C80002701FB49
:1008D0000700A3FB091800FB09874FEAE97C03FB2B
:1008E0000C77DDE9008C18EB01014CEB070CCDE92E
:1008F000001C4FF00A0CA3FB0C18002700FB0C8017
:1009000003FB0700521EABD10698DDE90023C100AE
:1009100001208840401EC117801A994107D28920C2
:10092000206004202860784630608920BCE7694652
:10093000069A049839F020FD00202060286078464F
:1009400030600020B0E730B500B90120401E80B211
:1009500040F2B553B0FBF3F2B0FBF3F403FB140029
:100960009206401C120E80B24FF4B77398420BD916
:10097000521CD2B2A0F5B77003E0521CD2B2A0F262
:100980006D1080B29842F8D2202801D2012319E0DC
:100990001F3880B2930701D01C2300E01D2398422A
:1009A00001D802230EE0C01A854D002380B26435C1
:1009B00003E0001B5B1C80B2DBB2EC5C8442F8D32A
:1009C000DB1CDBB20A704B7088707A49002008602B
:1009D00079490860784679490860002030BD10B533
:1009E000027840F26D135A430A80754C43786E3496
:1009F00034F813301A440A8083781A4493B20B8077
:100A00000278940705D14078022802D803EB9200BF
:100A100003E0012000EB92001844088065490020A3
:100A2000086065490860784664490860002010BD88
:100A300010B581784FF0FF32C9B143780D2B18D231
:100A4000DFE803F017070D070A070A07070A070A76
:100A500007001F290BD80FE01E2908D80CE00078EA
:100A6000800702D01C2902D806E01D2904D91046AF
:100A700010BD6FF0010010BD002010BD18B5028838
:100A80000024B2F5FA6F0ED9C2788DF80220827870
:100A90008DF801200078A0F5FA608DF80000684616
:100AA000FFF79DFF00E00C8042480460424804606C
:100AB000784642490860002018BD2DE9F04F88466D
:100AC00000213C4D3C4E3D4F82464FF08609B3EB32
:100AD000420F15D301201EE0A2EB000B1AF80B40C9
:100AE00004F00F04092C0BDCA3EB400E0EEB080CFA
:100AF00030348CF801401AF80B402409092C06DD2B
:100B0000C5F800907846316038608620CDE63034F4
:100B100008F80E40401C9042DED9012000EB420054
:100B2000302204E0A3EB000C401C08F80C20984293
:100B3000F8D929607846316038600020B5E67CB588
:100B40000D4601A9FFF7FFFE1A4C000601D52068EB
:100B50007CBD9DF8040000909DF805309DF80620AE
:100B600018A1284639F07EF813490020206008605B
:100B700078461249086000207CBD3C2310B5B0FBCC
:100B8000F3F2B0FBF3F403FB1403D2B20A20B2FB7E
:100B9000F0F430340C70B2FBF0F400FB142230326D
:100BA0004A703A228A70B3FBF0F23032CA70B3FB5B
:100BB000F0F20FE0080000100C0000101000001010
:100BC00002C10300253032752D253032752D2530B8
:100BD0003275000000FB1230303008715C49002093
:100BE00008605C49086078465B490860002010BDD9
:100BF0003C2310B5B0FBF3F2B0FBF3F403FB14009D
:100C0000564BD2B29A5C0A70185C4870504900206A
:100C100008605049086078464F490860002010BDC0
:100C200018B50C466946FFF78EFE4949000601D506
:100C3000086818BD9DF802204848825C22709DF823
:100C40000120825C62709DF80020805CA070002012
:100C500008604049086078463F490860002018BD98
:100C600070B5044611B939F011FB0146002220236A
:100C70000DE0A05CF02801DB103802E0C02802DBA8
:100C80004038A05402E0802800DBA354521C8A4262
:100C9000EFDB002070BD70B5044611B939F0F6FAEB
:100CA00001460020202311E0225CF02A01DB2354BE
:100CB0000BE0E02A01DB103206E0B02A01DB403A0B
:100CC00002E0802A01DB40322254401C8842EBDBE8
:100CD000002070BD20280BD0092809D00A2807D091
:100CE0000B2805D00C2803D00D2801D00020704718
:100CF0000120704770B50546044600E0641C20786A
:100D0000FFF7E8FF0028F9D1204639F0BFFA421C6E
:100D10002146284639F075FB284670BD10B50446BB
:100D200039F0B4FA011900E0491EA14205D011F8CA
:100D3000010CFFF7CFFF0028F6D1002008702046F5
:100D400010BD10B5FFF7D6FFBDE81040E6E7000084
:100D5000080000100C0000101000001002C1030079
:100D6000F8B56A4E0D4607460222694630462AF01B
:100D700095FE674C000615D4BDF800002A4640F0E9
:100D8000804039462AF095FE00060BD4BDF80000DD
:100D900002222844ADF80000694630462AF089FE58
:100DA000000601D52068F8BD5A490020206008607F
:100DB0007846594908600020F8BD08B50020ADF814
:100DC00000000222694651482AF073FE08BD014620
:100DD00002224E482AF062BE2DE9F04188B000257B
:100DE000022201A949482AF059FE494C00064ED476
:100DF00001202DF080FC000649D4484908884206AD
:100E000006D520F0400008801AF0F7FA00063ED41C
:100E1000002705A8059705F091FD000637D406A820
:100E2000069705F09AFD000631D43D49022008706E
:100E300004A962201AF02EFB000628D400264FF0E9
:100E4000200829E046F08040012203A92AF026FE6E
:100E50009DF81000400714D49DF80C0043280DD0D5
:100E6000F3280BD0F42809D0F5280AD16D1CEDB277
:100E70008DF80C80022D04D1002502E00DB18DF813
:100E80000C80012103A82DF022FA000603D520686A
:100E900008B0BDE8F081761CBDF804008642D1D3CD
:100EA0001C482760076078461B4908600020EFE770
:100EB00010B5FFF782FF164C000604D405202DF074
:100EC0001AFC000601D5206810BD124900202060E0
:100ED0000860784610490860002010BD10B50C4C21
:100EE00018B1FFF76AFF000604D401202DF003FCBF
:100EF000000601D5206810BD06490020206008606A
:100F0000784605490860002010BD0000780D0020DB
:100F1000080000100C00001010000010020000106B
:100F200000000010F8B516460D4604468948012217
:100F300069462AF0B3FD000602D587480068F8BD6F
:100F40009DF80000204000D001202870022C06D01F
:100F50008048401C022231462AF0A0FDF8BD7D48A1
:100F6000C01CF7E710B59EB01BA80BF0D2FB7A4C63
:100F700000064BD41AAA1CA90120FFF7D3FF0006D4
:100F800044D49DF8700028B1BDF86800BDF86C101D
:100F9000884209D97149002020600860784670496C
:100FA000086000201EB010BD02202DF035FA0006AA
:100FB0002CD46C482DF05AFE000627D46948143012
:100FC0002DF054FE000621D41AAA1CA90220FFF716
:100FD000A9FF00061AD49DF87000C8B11DA9BDF87C
:100FE0006800FFF7B0FC000610D49DF874005D495E
:100FF00000909DF875309DF87620263101A838F0D4
:1010000031FE01A82DF032FE000601D52068C9E7A7
:101010005548018841F002010180544902200870BE
:10102000012011F01BFCBDE7FEB501A80BF071FB20
:10103000494C000632D46A4602A90220FFF772FF2B
:1010400000062BD49DF80800444D454E28B1BDF84C
:101050000000BDF80410884206D9002020602860F6
:10106000784630600020FEBD02202DF0D5F9000644
:1010700014D43C482DF0FAFD00060FD43948143042
:101080002DF0F4FD000609D43748018841F0020133
:101090000180012011F0E2FB000601D52068FEBDB1
:1010A00091202060BE202860784630609120FEBDEF
:1010B0004FF0A0430146042218462AF0EFBC4FF03F
:1010C000A0430146042218462AF0F3BCF7B50446B3
:1010D000204882B00E460546012269462AF0DEFC11
:1010E0001D4F00060ED49DF800000EB1204300E015
:1010F000A0438DF800000122694628462AF0D9FC59
:10110000000602D5386805B0F0BD022C06D01148A3
:10111000401C022204A92AF0CCFCF4E70D48C01CB4
:10112000F7E738B500200122014600901046FFF78E
:10113000CDFF094C000606D4012200210220FFF752
:10114000C5FF000601D5206838BD6846FFF7B7FF28
:1011500038BD000004000050080000100C00001012
:10116000100000108BC103000200001000000010EE
:101170002DE9F04F99B0012400250C94841A0895AC
:1011800071EB030404DA16461C4607460D4603E0DD
:101190000C46064617461D4600218B46059116E073
:1011A000022200233046214638F037FD06460C4621
:1011B000022200233846294638F02FFD0D46012231
:1011C00005991BEB020B41F1000107460591F00761
:1011D00001D1F807E4D001200021CDE9220124AAA1
:1011E0000846279482E84300711E64F10000CDE9AF
:1011F0001610CDE91475CDE9127500BFDDE92601A1
:1012000080468946C00729D1DDE92201C20702D103
:10121000249AD2070AD03A1845EB0100CDE92220E2
:10122000DDE9241071186041CDE92410DDE92201C7
:101230000222002338F0F1FCCDE92201DDE924018E
:101240000222002338F0E9FCCDE924010222002328
:101250004046494638F0E1FCCDE92601DDE91201BE
:10126000C20704D0DDE92632181A8A410BDA14A924
:1012700022A800F066FA16A924A800F062FA12A9C2
:1012800026A800F05EFADDE9260110900D91C00756
:10129000B4D00DF15008DDF85C2098E80B009E46B4
:1012A000DDE922C3E1469A46BCEB000C8B4106DB2C
:1012B000DDE9248CB8EB0E037CEB020C0DDA17EBA6
:1012C000090345EB0A0CCDE9223CDDE9243CF31887
:1012D00044EB0C0CCDE9243CE2E7B9EB00006AEBEF
:1012E0000103CDE922032598B8EB0E0160EB020063
:1012F000CDE92410DDE91210109B0D9A5B1A62EB08
:101300000002CDE926320023591A73EB0002FFF6E2
:1013100075AF14E0DB1B60EB05004FF0000CB3EB86
:101320000C0C70F1000C17DBCDE92230901B61EB47
:101330000401021E71F100020EDBCDE92401DDE99A
:101340002230D91B70EB050106DBDDE92421B6EB69
:10135000020C74EB010CDDDB002108461AE000BF33
:10136000DDE922720C9B089DA3FB07C805FB0785DE
:1013700003FB0252CDE922C2DDE92672A3FB07C8B6
:10138000089D491C05FB078503FB0252CDE926C2D7
:1013900040F10000059AB1EB0B0370EB0202DFDBBA
:1013A000DDE9261081F00101014304D04FF0FF3048
:1013B00019B0BDE8F08FDDE92410711A64EB000468
:1013C0002898C0E900140020F2E72DE9FF5F9CB0E7
:1013D0000020CDE90200CDE9040092462E9907AA2B
:1013E0000A20CDE90002994614AB0122491C1AF0EB
:1013F0009EFF00287DD114AB08AA195C0C0902F8E5
:10140000104001F00F0402EB4001401C4C70082812
:10141000F3DB9DF82F70DFF8408311460E2000BFEC
:1014200058F82740461C255CA45D801E4E5D11F8CF
:1014300004C001F805C00E55F2D5002002EB4004AF
:1014400012F810106478904644EA01111954401CB7
:101450000828F3DB19460020079B0DE01C1A0C44FA
:101460000A5C14F8015D2E0146EA15150D541501AC
:1014700045EA12122270401CB0EB530FEED3082342
:1014800012A914A8079AFFF7D9F90028B2D114A914
:101490000EF026FB0028ADD10C2114A8FFF7BBF9F4
:1014A00000287DD0DDE91501CDE90801082208A951
:1014B0000020131A0B440C5C13F8015D0D54401C02
:1014C0001C70B0EB520FF4D300252C462F462E464D
:1014D0002846C3464FF00A0E1BF8001072463039FA
:1014E00001EBC101B1FBF2F3B1FBFEFC0EFB1C11E1
:1014F00000E0AEE04FF0640CA5FB0C2801EB81018D
:1015000003EB410104FB0C84002305FB0344551845
:101510005C4107910A23A7FB031C06FB03C30022BF
:1015200007FB02321BF8003000F10100303B5F186E
:1015300042EBE3760828CFDBDDE91201401B61EBCB
:101540000401864A0023CDE9120138F0EFFACDE913
:10155000122350EA01027CD01AAA0692CDE9005467
:10156000DDE91C23FFF704FE002872D1DDE91A50E3
:10157000A7FB051206FB052207FB00248346DDE9D5
:101580001C230846214638F0D1FA14469846DDE976
:101590001223A2FB050603FB056302FB0B3100E0EF
:1015A0006CE0DDE91C2338F0C1FA15469B4654EA8D
:1015B000080203D0DDE92A01012618E001200021FC
:1015C0001AE000BFDDE92A72A0FB073C01FB07C15E
:1015D00000FB02111846BAEB000379EB010205D2B9
:1015E00052464B4638F0A2FA10461946761CF317BD
:1015F000371B73EB0803E5DBCDE91A0180460C4687
:1016000055EA0B0003D0DDE92C01012617E001208B
:10161000002119E0DDE92C72A0FB073C01FB07C1AA
:1016200000FB02111846BAEB000379EB010205D268
:1016300052464B4638F07AFA10461946761CF31794
:10164000771B73EB0B03E5DBA0FB085301FB0831B1
:1016500000E012E000FB041152464B46284638F0E9
:1016600065FA10461946DDE91C2338F05FFADDE91A
:10167000120150405940084303D0002020B0BDE87B
:10168000F09F0120FAE7F0B5411E85B01E2932D245
:10169000012404FA00F111F0D00F2CD0304FBE68B5
:1016A000401E2D4D8440083D69680C4229D1C1B2CD
:1016B00004912C49002301EBC001D1E90021CDE9BF
:1016C00002212849284A383901EBC001D1E900013B
:1016D000CDE9000141F2E7001946FFF776FE002848
:1016E000286801D0204300E0A0432860B8681F4963
:1016F000801B884202D3002005B0F0BD68682043FB
:10170000686028682040F7E7411E1E290ED201219B
:1017100001FA00F212F0D00F08D0401E81400E48AE
:10172000083842688A4342600120704700207047B1
:1017300000B501231846FFF7E7FF5B1C1E2BF9DD00
:1017400000BD30B5D0E90023D1E90045C0E900452E
:10175000C1E9002330BD00000CC0072000E1F50501
:101760000080004008C2030063777B00404B4C00C0
:1017700038B50446684604F040FB9DF80000204060
:1017800038BD38B50446684604F037FB000602D57C
:10179000FD48006838BD9DF8000020438DF800002A
:1017A000684604F021FB38BD38B50446684604F0AD
:1017B00024FB000602D5F448006838BD9DF80000FF
:1017C000A0438DF80000684604F00EFB38BD01B55B
:1017D000FEF73CFD684604F027FBFEF74CFD08BD14
:1017E0007CB5684604F02AFBE74C000638D49DF827
:1017F00000000025082809D009280DD0E3482560FD
:1018000005607846E249086000207CBD684604F027
:1018100026FB000624D40BE001A805F04BF80006D7
:101820001ED49DF8040001281CD013208DF8000060
:10183000684604F0F9FA000612D48DF8045001A8A5
:1018400005F02EF800060BD48DF8045001A804F022
:1018500032FB000604D4432019F0B1FC000603D586
:1018600020687CBD0220E1E7012010F0F7FF7CBD7D
:101870002DE9F041002402202DF033FAC54DAE6869
:10188000C54F4FF4FA7811E0A868801BB8420DD319
:10189000012024F021F9C821404623F02BFC01202F
:1018A00024F027F9AE68641C042C04DC002024F02A
:1018B00005F90028E8D1012C06D0022C07D0032C12
:1018C00009D0042C11D10EE001F032F90DE0022014
:1018D0001FF0ECFD09E0B14C0120207002F050FF38
:1018E0000020207001E025F0EFFEBDE8F04101206E
:1018F0002DF0F7B90EB568460EF06DF850B193288B
:1019000003D1A2480068062801D00E2000E0112073
:10191000FFF75DFF9C4800680EBD2DE9F34F0027DF
:1019200089B088460F703E4608A938460CF087FA01
:10193000954C000639D49DF82000DFF85092DFF86E
:1019400050A2400607D407A804F067FA00062CD47A
:101950009DF81C0068B3694609980CF0D6FF000694
:1019600023D40125EB4605A9284604F061FD0006B5
:101970001BD405EB85015944052205A8491F38F001
:1019800035FC00B101276D1CEDB2042DEBD9C7B1B8
:10199000834909980880452019F011FC000604D4F9
:1019A000012010F05BFF00060BD520680BB0BDE8EE
:1019B000F08F26607946C9F800600020CAF8001050
:1019C000F4E788F80070F4E72DE9F34F85B00320C1
:1019D000002408700E462746214601200EF04BF8E1
:1019E0000106694802D5006807B0E0E70168DFF842
:1019F0009C91DFF89CA10025052913D08046EB4679
:101A0000694601200EF011F80006D8F80000EBD46A
:101A100005280DD005220BF10400059938F0E6FBEE
:101A200018B103E0357005600DE0671C641CE7E742
:101A300037B1BC4201D1022000E00120307000E04B
:101A40003570C8F800507946C9F800500020CAF82F
:101A50000010C9E730B5044685B000202080022080
:101A60000EF01FF8484D05280BD0694602200DF0F6
:101A7000DCFF00061ED4BDF800002188884200D992
:101A8000208001200EF00DF8052802D069460120C3
:101A900006E000200EF005F805280BD0694600206E
:101AA0000DF0C3FF000605D4BDF800002188884270
:101AB00000D92080286805B030BD2DE9F04387B0FB
:101AC0000646694600200EF00BF82F4D000649D45B
:101AD00003A90B200CF0B3F9000643D40C2203A990
:101AE000684638F083FB0227DFF8A080DFF8A0907B
:101AF000002408B137703EE003A910200CF09FF9D4
:101B000000062FD4694604200DF0EAFF000629D410
:101B1000BDF80000BDF80C108842EBD169460620E4
:101B20000CF08DF900061DD4BDF80000BDF80C10B6
:101B3000401E8142DED169460E200CF080F900067D
:101B400010D403A8FFF786FF00060BD4BDF80000F1
:101B5000BDF80C108842CDD3694600200CF06FF917
:101B6000000603D5286807B0BDE8F0839DF80000A3
:101B70004007BFD534702C607946C8F8004000207B
:101B8000C9F80010EFE70000080000100C0000107A
:101B90001000001000800040C0C62D00140000108E
:101BA000BC000010FEB502A804F048F9FE4C000687
:101BB00037D49DF808000025FC4EFD4F1D2812D09B
:101BC00004F049F808B103F0C8FF01A804F07DF95A
:101BD000000626D49DF8040028B1012809D0022867
:101BE0000BD003280ED02560784635603860002081
:101BF000FEBD012008F0B4F901E008F0F7FF00068F
:101C00000FD410E08DF80050684604F049FE00063D
:101C100007D4432019F0D3FA000602D40BF0DEFEFD
:101C2000EDE72068FEBD012010F018FEFEBD2DE995
:101C3000F0418AB0002606A80DF0CDFEDFF87083D3
:101C4000D94CDA4D932806D1286808286DD005288C
:101C50006BD0062833D0002108460DF00CFF00069B
:101C600063D405A900200EF0D3F900065DD4D14F4E
:101C7000387858B1002101200DF0FDFE000654D443
:101C800005A901200EF0C4F900064ED409A805F0FC
:101C900063F8000649D49DF8240038B300210120E0
:101CA0000DF0E9FE000640D4694601200DF0BDFEAE
:101CB00005280DD00120397881430ED10AE000209B
:101CC000206079462860C8F800100AB0BDE8F081AD
:101CD0000020F0E73978884308D09320206008205E
:101CE000794628609320C8F80010EEE702200DF036
:101CF000D8FE000619D4694602200DF096FE0006B3
:101D000013D4002102200DF0B6FE00060DD405A963
:101D100002200EF07DF92068932806D12868082853
:101D200003D1761CB6B2032EF1D32068CDE72DE99E
:101D3000F04F99B00EA804F070F89B4C000672D4D6
:101D400013A805F009F80006F9D4DFF86882102618
:101D5000DFF85C9298F80000944D4FF0000A4FF0C5
:101D6000160B9227C0B109A80BF0D1FF40F3C010A9
:101D7000401C8DF81C0011D09DF83500010637D5A8
:101D80009DF84C1099B38DF80060684604F04CF84B
:101D9000032027602860AFE18DF81CA09DF84C005F
:101DA00098F80010084217D02868032811D004289A
:101DB0000FD08DF800B000BF9DF80000FFF707FDC1
:101DC000286809282FD9462019F0F9F93020276012
:101DD000E0E78DF80060EFE7FFF7E4FE92E100BF77
:101DE0008DF80000684604F01FF819B0DFE5FFE742
:101DF000C00603D50BF0F2FD0006A0D417A914A865
:101E00000CF0CAFEFFF713FFDFF8AC8193280BD06C
:101E10009DF8350000077DD507A90CA8FFF7D4FD74
:101E200000285ED114E06CE1FFF7BCFE000686D40A
:101E30000E208DF80000684603F0F6FF0006DCD4A3
:101E400000215EA02CF056FD614902200870C8E117
:101E50009DF81C00022804D001287DD000287CD0E9
:101E6000E9E19DF83500400778D501A80BF0CDFEDB
:101E7000002874D103E000BFFFF7A9FCD9E108A94D
:101E800004200DF02DFE0006F8D4BDF82000BDF8AA
:101E90000410401C81427CD19DF83500800602D59B
:101EA000FFF780FE11E015A804F00FF80006E5D456
:101EB0009DF85400012815D0FFF774FE0006DDD40C
:101EC0000EA803F0AAFF0006D8D4BDF8040014A998
:101ED000FFF723FD20688228D0D0922863D0932872
:101EE0007AD133E111A804F034F80006C6D411AE5B
:101EF000B01C04F03FF80006C0D4301D04F04BF8CD
:101F00000006BBD433499DF848000870684603F0CA
:101F100095FF00E06CE10006B0D49DF800000428B5
:101F200009D005283AD01D282BD0FFF73BFE684684
:101F300003F084FFC7E703F08EFE30B103F00DFE1F
:101F400011A805F08DF9000698D4012600270FA9E5
:101F5000304604F036F903E099E0A3E08EE0F1E0CA
:101F600000068BD40F98761CF6B20744102EEED9DB
:101F70003FB11D208DF80000684603F055FF0006B4
:101F800095D4B8F8001011A841F00401A8F8001089
:101F900000E022E005F064F9000688D405F0DCFFDB
:101FA000000684D4C3E753E0080000100C000010C2
:101FB000100000108AC10300020000108E98888172
:101FC0008A80208F808C9F9288208F840A0A00004C
:101FD0000000001091C207203DE0FFF7E3FD00067E
:101FE00084D49DF835009DF8381000F04000491E5B
:101FF000084306D1BDF82010BDF80400891C8842B2
:1020000014D00BF0EBFC00067BD414208DF80000FC
:10201000684603F009FF000673D44E2019F0CFF88C
:1020200000066ED4012010F019FCDEE6401E80B2DE
:1020300014A9FFF772FC2068822862D0922802D08F
:10204000932803D182E0286808287DD11320C7E6B1
:102050002868082878D19DF8500008B11520BFE6FF
:10206000684603F0EBFE00064BD49DF800001D28E7
:1020700069D047E00120B3E60220B1E68DF80060A8
:10208000684603F0D1FE00063BD4332007E08DF80C
:102090000060684603F0C8FE000632D4412019F003
:1020A0008EF89EE0FFF77EFD00062AD49DF83500ED
:1020B0004FF0310610F0600F29D09DF84C0008B3A6
:1020C0008DF800B0684603F0AFFE000619D4422038
:1020D00019F075F86946532019F0DCF9000610D4A0
:1020E0009DF8000010F002008DF8000002D00120E1
:1020F00010F0B4FB27602E6079469220C9F80010DA
:1021000073E680E09DF838000028B5D0B2E701A85A
:102110000BF07BFDB0B914A8FFF7CFFC822872D07A
:10212000922811D0932811D09DF8500080B1022838
:1021300036D0882020600220794628608820C9F89F
:10214000001052E600E076E00F2095E60E2093E6C0
:1021500010F0FEF8012010F081FB5E2019F02FF83E
:102160000CF0B0F9000664D4FE4D0121FD4810F0DA
:10217000FEFB00060AD5FEF769F80BF02FFC0006FF
:1021800057D4FEF778F82078000652D40CF0D6F930
:1021900000064ED495F800010028E6D1182019E079
:1021A0009DF84C0080B18DF800B0684603F03CFE0D
:1021B00000063ED4422019F002F8B8F8001041F0B1
:1021C0000201A8F8001092E79DF8380008B101203C
:1021D00000E002208DF80000684603F025FE0006AE
:1021E00027D4B8F8001041F00201A8F8001019E750
:1021F000FFF7D8FC9DF84C0000289DF838000DD062
:1022000010B10C2001E014E00D208DF800006846AC
:1022100003F00AFE00060CD4402040E708B101207C
:1022200000E002208DF80000684603F0FDFD000686
:1022300001D52068D9E5C4F800A07946C5F800A00A
:102240000020C9F80010D0E510B5C748C74C86B0CB
:10225000007820B10420FFF716FA40B123E00620F1
:10226000FFF711FAF8B90420FFF70DFAD8B90120E9
:10227000FFF709FAB8B9372018F0A1FF02A95320D7
:1022800019F008F9000639D49DF8080010F0020092
:102290008DF8080007D0B648018841F0020101809E
:1022A000012010F0DBFA012004A9CDE9000102466B
:1022B00003AB042109201AF03AF800061ED49DF859
:1022C0000C0005281DD1AB480079C00704D00720B9
:1022D000FFF7D9F968B114E066200BE0682018F028
:1022E0006EFF00060AD4012010F0B8FA000605D4EB
:1022F00007E0652018F063FF0006EFD5206806B000
:1023000010BD9D4900202060086078469B49086008
:102310000020F4E738B5684603F090FD934C0006C2
:1023200029D4974D2878752827D00220FFF720FA66
:1023300070B17B202870684603F087FD00061AD430
:102340001C208DF80000684603F06EFD000612D4D4
:102350000120FFF70DFA80B151202870684603F084
:1023600074FD000607D417208DF80000684603F0BE
:102370005BFD000601D5206838BD9DF800000F28E0
:1023800001D17E2028707C490020206008607846BA
:102390007A490860002038BD2DE9FC4180460320C1
:1023A00024F061F8744E754F704C002530B9B8F1C7
:1023B000000F03D00420FFF7DBF9E8B36946532090
:1023C00019F068F89DF8000010F002008DF8000088
:1023D00002D0012010F042FA3D2018F0F0FE9DF8E6
:1023E000000010B1012010F039FA6549752008701D
:1023F000684603F023FD00061BD4684603F036FD53
:10240000000616D401A803F008FD000611D49DF8BB
:10241000040008B1192000E01A208DF80000684679
:1024200003F002FD000604D40420FFF7AAF9000619
:1024300003D52068BDE8FC8106E082202060784654
:10244000356038608220F5E7256078463560386071
:102450000020EFE72DE9F0438BB000273E4607A8A8
:1024600003F0ECFC414C00067AD49DF81C00DFF828
:102470000881DFF808910025022803D0192801D02F
:102480001A286ED103A9352019F004F8000667D484
:102490009DF80E0000F00F01000900EB800001EB39
:1024A000400000F5FA60ADF814009DF80D0000F052
:1024B0000F01000900EB800001EB40008DF81600D1
:1024C0009DF80C0000F00F01000900EB800001EB0B
:1024D00040008DF8170009A905A8FEF7CFFA03A957
:1024E000362018F0D7FF00063AD49DF80E0000F011
:1024F0000F01000900EB800001EB400000F5FA60DD
:10250000ADF814009DF80D0000F00F01000900EB7C
:10251000800001EB40008DF816009DF80C0000F0E3
:102520000F01000900EB800001EB40008DF817005F
:1025300008A905A8FEF7A2FA68460AF0EAF800061C
:102540007AD404A823F0CBFF000675D4BDF824008C
:1025500020B3BDF80010814220D39DF8100011E097
:102560006AE06DE048C607208AC103000800001039
:102570000200001088D907200C0000101000001085
:1025800090C20720172809D2012703AB352239460C
:102590000220039519F011FF00064DD4BDF820006C
:1025A00088B1BDF8001081420DD39DF8100050B1E4
:1025B000012603AB362231460220039519F0FDFEB9
:1025C000000639D4E7BB56EA070045D006A93420F7
:1025D00018F060FF00062FD49DF81800012826D0BF
:1025E000022804D0032837D14D497D20087006A960
:1025F000532018F04FFF00061ED49DF8180010F06D
:1026000002008DF8180004D0012010F027F9000610
:1026100012D40EB1482000E0472018F0D0FD9DF8FC
:10262000180020B1012010F019F9000604D404A804
:1026300023F055FF000604D520680BB0BDE8F083F9
:102640000AE09DF810000EB1401E00E0401C8DF81D
:10265000100004A823F0A8FF25607946C8F80050B0
:102660000020C9F80010E8E738B50546684603F0D1
:10267000E5FB2C4C000604D4284603F0CEFB0006F4
:1026800001D5206838BD9DF8001006290FD008DC60
:1026900001290CD003290AD0042908D0052908D122
:1026A00005E0072903D0132901D0152901D1012004
:1026B00028701D4900202060086078461B4908608A
:1026C000002038BD38B50546684603F0C8FB154CF8
:1026D000000618D49DF80010072916D006DC0DD28C
:1026E000DFE801F00C130C13131313000E290CD0A8
:1026F00013290AD0152908D01B2906D0284603F033
:102700008CFB000603D5206838BD012028700649DF
:10271000002020600860784604490860002038BD29
:1027200090C20720080000100C00001010000010DC
:1027300010B58AB005A82CF0F2F9D24C000637D4B7
:1027400068462CF0ECF9000632D40220ADF80A00FD
:10275000ADF80200ADF804000A20ADF80600002133
:1027600068462BF059FF000622D40021C6A02CF0A9
:10277000C1F800061CD40021C6A02CF0BBF800064E
:1027800016D4012108462BF0DDFE000610D40021EE
:10279000C1A02CF0AFF800060AD4002105A82BF048
:1027A0003BFF000604D401202BF036FE000602D5C4
:1027B00020680AB010BD2CF043FAFAE72DE9F04F7B
:1027C000834699B00D4608462BF052FEAD4C0006EC
:1027D0007DD458462BF0EDFE00067DD42B465A469C
:1027E000B4A1684637F03EFA002168462CF082F822
:1027F000000671D4B5482A22C5896846294637F0B3
:10280000B5FE0A200DF805000DF101014FF0000999
:1028100005F80190494668462CF06CF800065BD438
:102820002CF00DFBDFF8A8A20646DFF8A8829AF884
:102830000000022805D000EB400108EBC100406811
:102840008047A54FBD680021A4482CF053F800062E
:1028500042D40021A1482CF04DF800063CD40021C0
:102860008CA02CF047F82CF0EAFA861BB868411BC4
:102870004FF47A70B1FBF0F59AF80000022805D009
:1028800000EB400108EBC1004068804706EB4600C2
:10289000C0EBC61005EBC000401EB0FBF5F7ABF176
:1028A00001002CF0D0FA4FF47A714E436843B6FB26
:1028B000F0F2FF1DFB088AA1684637F0D3F968469D
:1028C0002CF0D4F9000607D400218DA000E003E02D
:1028D0002CF010F8000603D5206819B0BDE8F08F81
:1028E0008849C4F800907846C1F80090864908608D
:1028F0000020F2E770B58AB0064605A82CF00FF963
:10290000604D00063CD468462CF009F9000637D427
:102910000121ADF80210ADF80060BDF81400ADF86B
:102920000410ADF80A10ADF80610401E2CF092FA13
:10293000BDF8221000FB01F4BDF80000401E2CF091
:1029400089FA94FBF0F0ADF80E00012168462BF0F7
:1029500063FE000614D40424032E02D10D2C00D1F2
:102960000E2421463046FFF729FF000608D4E41C58
:102970000F2CF1D3002105A82BF04EFE000602D546
:1029800028680AB070BD5F4900202860086078465A
:102990005D4908600020F4E710B500202BF009FE27
:1029A000384C00063AD406202BF062FD000635D4E0
:1029B00000213FA02BF09EFF00062FD401210846E6
:1029C0002BF0C0FD000629D4002150A02BF092FF6F
:1029D000000623D4022101202BF0B4FD00061DD4F3
:1029E00000214AA02BF086FF000617D40121022007
:1029F0002BF0A8FD000611D4002144A02BF07AFF93
:102A000000060BD4022108462BF09CFD000605D4DD
:102A100000213EA02BF06EFF000601D5206810BDFE
:102A20003849002020600860784637490860002057
:102A300010BD10B501202BF0EFFC124C000619D48C
:102A4000012108462BF07EFD000613D405202BF053
:102A50000FFD00060ED4214B1822A533642100205F
:102A60002BF00CFF000605D400212BA02BF042FF19
:102A7000000601D5206810BDBDE8104001202BF0F4
:102A800046BE000008000010465072696E742D3179
:102A9000310000000A00000084A5ACAEADE1E2E028
:102AA000A0E6A8AEADADA0EF20AFA5E7A0E2EC0A8E
:102AB000200A0000200A98908894922025752C20E6
:102AC0009F908A8E91929C2025750A008C0400109C
:102AD0009EC20720A0C2072000800040E0C2030081
:102AE000D1EAEEF0EEF1F2FC3A20257520D1D2D0F9
:102AF0002FD12028257520CCCC2FD1290A00000009
:102B00000A200A000C00001010000010313235209D
:102B1000544543540A000000203420363032323409
:102B200032203030313733370A200A200A000000C3
:102B300070B5ACB002202BF06FFCA44D00067BD426
:102B4000022108462BF0FEFC0006F8D4A0A2A3A1A7
:102B500002A837F087F8002102A82BF0CBFE012154
:102B600008462BF0EFFC0006E9D49DA02CF07EF87F
:102B700001202BF051FC96A298A102A837F072F820
:102B8000002102A82BF0B6FE02A801F0F9F902A874
:102B900000F0ABFE002102A800F0E7FD02A800F063
:102BA00027FE02A801F0EDF902A801F0CCFA2022DC
:102BB0001DA9904828F072FF02AA8DA18EA000F0F6
:102BC00086FD02A82CF052F88EA125A81E9A37F097
:102BD00049F802AA25A98DA000F079FD02A82CF0E1
:102BE00045F888A125A81F9A37F03CF802AA25A924
:102BF0008BA000F06CFD02A82CF038F881A125A86C
:102C0000229A37F02FF802AA25A989A000F05FFDCB
:102C100002A82CF02BF87BA125A8239A37F022F8E4
:102C200002AA25A987A000F052FD02A82CF01EF8E8
:102C300068462BF0AAF900E0BCE086A125A8009A1E
:102C400037F010F802AA25A984A000F040FD02A8E0
:102C50002CF00CF802A800F093FE85A02CF006F8EA
:102C600029A829F05DF92998012832D0032834D009
:102C7000042830D0072832D080A102AA81A000F019
:102C800026FD02A82BF0F2FF824C202202A8E18947
:102C900037F06CFC0E2280A102A837F0F8FB2AA9BD
:102CA0000120CDE9000101461BAB0222092019F0E9
:102CB0003EFB00067ED49DF86C3001A80A22411E1E
:102CC0000A2B52D2DFE803F0510D1151181C2028B5
:102CD0002C4D75A1D1E776A1CFE776A1CDE778A1FC
:102CE000CBE7E189084478A102E0E189084478A1B2
:102CF0000968016002711DE0E189084476A1F7E7E7
:102D0000E089084476A102E0E089084476A10A68D7
:102D10000260898881800DE0E089084474A1F6E7AB
:102D2000E1890DF10200084473A10B6803608988F2
:102D30008180827102A82BF099FF02AA70A172A073
:102D400000F0C5FC02A82BF091FF744800788DF8C4
:102D50006C0070B101280FD0022802AA30D024A143
:102D60000CE0E08908446EA1D1E7E18908446EA136
:102D7000BEE702AA6EA101E002AA6FA170A000F056
:102D8000A6FC02A82BF072FF28F0D7FE01202BF042
:102D9000BEFC552018F013FA1CA803F0A7F8000693
:102DA0000BD41CA802F086FC000606D41CA803F075
:102DB00093F800E001E0000604D528682CB070BD4F
:102DC00064A1DBE701200FF049FDF7E708000010E0
:102DD000465072696E742D313100000025730A006F
:102DE000C8CDD4CED0CCC0D6C8DF20CE20CFC40A28
:102DF0000000000008000020CDC0D0C0C1CED2CA63
:102E0000C00000002531306C7500000020C4C2C82D
:102E1000C3C0D2C5CBDC2CC2D1C5C3CE00000000DC
:102E200020C3CECBCEC2CAC02CC2D1C5C3CE0000F7
:102E300020C4C2C8C3C0D2C5CBDC2CD1C1D0CED136
:102E40000000000020C3CECBCEC2CAC02CD1C1D05E
:102E5000CED100002532644300000000D2C5CCCFA3
:102E6000C5D0C0D2D3D0C020C3CECBCEC2CAC8003A
:102E7000D1C2DFC7DC20D120CFCA0A00556E6B6EED
:102E80006F776E0020CAC0CDC0CB20CEC1CCC5CDDF
:102E9000C00000008C04001020D1CACED0CED1D208
:102EA000DC20C1DBCBC0000052532D323332000096
:102EB00055534200424C5545544F4F544800000072
:102EC0005749464900000000313230300A00000006
:102ED000323430300A000000393630300A00000049
:102EE00031343430300A000033383430300A0000D6
:102EF00035373630300A00003131353230300A0093
:102F0000343830300000000020D1CACED0CED1D22B
:102F1000DC20C2D0C5CCC5CDCDCE00009EC20720DE
:102F200031393230300A0000343830300A000000C5
:102F3000C0D2CECB00000000D8D2D0C8D50000004F
:102F400020CFD0CED2CECACECB20CEC1CCC5CDC024
:102F500000000000C0D2CECB20CDCEC2DBC9000025
:102F60002DE9F843F34DF44FDFF8D083002440B946
:102F70006946012022F07EFD000617D40098C007A4
:102F80001DD0EF4E3088800506D501220021104665
:102F90000AF00CF8000609D43078000609D50122A1
:102FA000114600200AF002F8000602D52868BDE8A4
:102FB000F883308810F4207F08D1800406D42C6078
:102FC00079463C600020C8F80010F0E74FF4FA742E
:102FD000FA21204622F08EF82146002022F08AF8BD
:102FE000F6E72DE9F04F95B04FF00009D14FDFF82B
:102FF00054A3CDF84890DFF840B33B68CAF80030DE
:10300000DBF80000CE49DFF83483CAF804007F26DD
:10301000CD4C0988D8F800204D46892B10D010DC03
:10302000812BFBD006DC062B77D2DFE803F0F7F725
:1030300076F7F7F7822B71D0862BEFD0872B6CD1E8
:10304000ECE0932B14D00ADCA3F18A010929EBD21E
:10305000DFE801F0E463636363FBE4E43E00962B86
:1030600070D0A12BECD0A22BFAD0A32BE7D12CE16E
:103070000A2819D008DC052816D00628E0D0082830
:1030800012D0092806D10FE00B280DD0802819D0C6
:10309000812817D00090AD4901A836F0E3FD00214A
:1030A00001A82BF027FC03E009B9A9A00DE0042535
:1030B000AF492670022008704B2018F080F8FF2DD1
:1030C0003CD1EAE00029F2D1AAA00EF0D2FFEEE74F
:1030D000FDF7BCF813A803F03FFEFDF7CCF89DF810
:1030E0004C0000287DD0DBF8000008282BD00ADC3B
:1030F00019D2DFE800F01828282828282828386066
:10310000CBF800003FE02A2819D008DC09281AD0A3
:10311000202814D0282806D111E0A8E040E030286B
:1031200038D0312836D000219CA02BF0E3FB26704C
:103130008F49022008704B2018F041F8A6E00EF0ED
:103140005AFF2AE0BFE00EF056FF8949CAF8009006
:103150000220CAF8049008704C4612A9532018F0B7
:1031600099F900066FD4129810F00200129007D05F
:103170009148018841F00201018001200FF06EFBAF
:103180003C60CBF8004079460020C8F8001015B02C
:10319000BDE8F08F03202BF08AFD7E202070C7E76A
:1031A000252864D2DFE800F0631E1E2B2B25631355
:1031B000296340323A6340636336633A3A63636338
:1031C0001E2B3434633A63633A5C5C3A2B0031B9AA
:1031D00067490220087000215DA02BF08BFB0425BD
:1031E00053E06EE019B9002174A02BF083FB022597
:1031F0004BE000217AA02BF07DFB012545E019B9B9
:10320000002180A02BF076FB03253EE00A253CE060
:1032100009253AE0834800780228F5D0CAF80090E2
:103220004846CAF804906AE714A9622018F032F9F7
:10323000000608D49DF850000007EFD5684602F05C
:1032400065FF000602D53868A1E71AE09DF8000086
:103250000028E3D05848018841F080010180DDE773
:1032600019B9002170A02BF045FB08250DE0009056
:10327000364901A836F0F6FC002101A82BF03AFBF4
:1032800003E003281DD007281BD026706D00FF2DFA
:1032900003D012A9284600F01DF80020FFF760FEB9
:1032A000694C6A4E207800EB400006EBC000406895
:1032B0008047207800EB400006EBC0008068804724
:1032C000E5E748461BE70428FBD079461846C8F8CE
:1032D00000105CE770B5040008680D4605D0611E5B
:1032E00088420FD14FF4FA6110E05949584A363AF2
:1032F00031F9101032F9100021F0ADFE002818D17C
:103300001B240CE0C00703D04FF4FA71002002E048
:10331000C8214FF4167021F09EFE002809D101202B
:1033200022F005FC2868401C2860A04201D1002042
:10333000286070BD080000100C0000101000001084
:1033400000C007201800001090C2072078AB0400CE
:103350008EE8A8A1AAA020AFA0ACEFE2A8208F849D
:10336000200A0A0A0A0A0A0A0A0A0A0A0A0A0000BB
:103370000000001091A1AEA920AEA1ACA5ADA02087
:10338000E120AFA0ACEFE2ECEE208F84200A0A0A25
:103390000A0A0A0A0A0A0A0A0A0A00008EE8A8A10A
:1033A000AAA0209D8A8B870A0A0A0A0A0A0A0A0A20
:1033B0000A0A0A0A000000000200001091A1AEA94A
:1033C00020AEA1ACA5ADA020E1209D918F87930AEE
:1033D0000A0A0A0A0A0A0A0A0A0A0A0A0000000075
:1033E0008220E7A0E1A0E520ADA5A2A5E0ADAEA5B5
:1033F00020A2E0A5ACEF0A0A0A0A0A0A0A0A0A0A87
:103400000A0A0A0091A1AEA920AEA1ACA5ADA020E8
:10341000E1208E87930A0A0A0A0A0A0A0A0A0A0A95
:103420000A0A0000BC01001091A1AEA920AEA1AC17
:10343000A5ADA020E1208F8F87930A0A0A0A0A0A05
:103440000A0A0A0A0A0A0A009EC20720A0C2072026
:10345000D4C3030070B5874C0546616819B101F803
:10346000010B616070BD0A2D02D10D20FFF7F2FF44
:1034700021680029F6D02846BDE87040084710B5FD
:10348000044602E0641CFFF7E5FF20780028F9D12C
:1034900010BD2DE9FF5F8A460546E94615F8010B88
:1034A00000286FD0252802D0FFF7D4FFF6E715F8E3
:1034B000010B4FF00008302802D02D2802D005E083
:1034C000012000E00220804615F8010B002606E0EE
:1034D00006EB860100EB410615F8010B303EA0F12A
:1034E00030010929F4D96C2801D04C2803D115F8F2
:1034F000010B48F00408002844D00246612801D39B
:10350000203AD2B24F2A3ED006DC422A38D0432A93
:1035100033D0442AC8D138E0532A0FD0552A34D0AA
:10352000582AC1D15FF010035FEA487101D4442AE0
:103530002DD05AF8041B442A2BD02FE05AF8047BD4
:10354000002400E0641C385D0028FBD102E020204C
:10355000FFF780FF5FEA887003D42046641CB04206
:10356000F5D33846FFF78BFF02E02020FFF772FF0C
:103570002046641CB04291D2F7E71AF8040B93E797
:103580000223D1E74EE00823CEE70A23CCE75AF81E
:10359000041B002902DA494248F0080800244F467B
:1035A000B1FBF3F203FB1212B1FBF3F1D2B2092A21
:1035B00005D9782816D04FF0070C6244D2B23032C9
:1035C0003A55641C09B1102CEAD35FEA087003D5A0
:1035D0002D2009F80400641C27465FEAC87004D057
:1035E000302003E04FF0270CE7E72020834602E07D
:1035F0005846FFF72FFF5FEA887003D438467F1CD8
:10360000B042F5D3641E19F80400FFF723FF002C25
:10361000F8D102E02020FFF71DFF38467F1CB042A2
:10362000A9D2F7E7BDE8FF9F0FB410B503A9029830
:10363000FFF72FFF10BC5DF814FB0FB470B50D4CF5
:10364000054606A960600598FFF723FF6068002122
:103650000170401B616070BC5DF814FB0FB470B565
:10366000044C06A9256820600598FFF712FF256025
:10367000F1E7000034C007202DE9F04180462BF02F
:10368000F5FA002821D04FF496764FF4FA77FE4CE5
:10369000FE4D012022F04BFA3146384621F02AFD3A
:1036A000012022F044FAA068A168091AA942FBD3BC
:1036B0002BF0C6FA0028ECD10021F5A02BF01AF966
:1036C0004046BDE8F0412BF0D1BABDE8F0812DE9CC
:1036D000F05F14468B46824636F0D8FD8146584648
:1036E00036F0D4FDEB4D064609EB0600E9890A27C2
:1036F0004FF00008884217D22022204636F036FFCD
:103700004A465146204636F037FEE8893246801B4D
:103710002044594636F030FEE8892754E989641C74
:1037200001F80480BDE8F09F012000EB4101202258
:10373000204636F01BFF4A465146204636F01CFE16
:10374000E889324659462754E889C6EB40002044B0
:10375000401C36F011FEE88904EB40004770E9890F
:1037600004EB410181F80280DCE730B585B0054605
:10377000002004900C4604A821F02AFEFCF766FD08
:103780000499642091FBF0F200FB12120A2392FBD1
:10379000F3F391FBF0F2C0A1684636F063FA2A46D3
:1037A0006946C0A0FFF793FF2846FFF765FFFCF7C7
:1037B00062FDC348006814B111280ED010E0112832
:1037C0002A4608D0BFA1B6A0FFF781FF2846FFF721
:1037D00053FF05B030BDBDA1F5E72068401C206057
:1037E000BCA16846226836F03DFA2A466946EAE7F7
:1037F0007FB506462AF0DFFB0028FBD1A24881688E
:10380000A24A83685B1A9342FBD3032021F0BDFDDB
:10381000044621F0FDFD0100B14D4FF47A704FF0E8
:10382000640232D041F270739C4203DA3246ADA199
:10383000ADA054E094FBF0F100FB114191FBF2F3D9
:1038400094FBF0F294A1684636F00CFA32466946D1
:10385000A5A0FFF73CFF3046FFF70EFFA04A00206F
:103860000A212C3A01E0401C491E52F82030A342A4
:1038700001DB0A28F7DB55F82120A1A1684636F0C4
:10388000F1F932466946A0A029E004F5FA7191FBEE
:10389000F0F300FB131393FBF2F391FBF0F27EA124
:1038A000684636F0DFF9324669468FA0FFF70FFF12
:1038B0003046FFF7E1FE8A490020583900E0401CFD
:1038C00051F82020A24201DC0A28F8DB55F820201C
:1038D0008BA1684636F0C6F9324669468EA0FFF7DE
:1038E000F6FE3046FFF7C8FE7FBD70B5044688B0CF
:1038F00001202AF091FD674E01252846FDF704FFBF
:10390000002838D02A4686A1204636F0ABF920465A
:10391000FFF7B2FEF1892022204636F027FE07A9E4
:103920001420CDE9000102AB012229460A2018F03B
:10393000FEFC2846FDF7A7FE50B1079A611C530014
:1039400002A8FDF7BAF8F189201F084478A109E020
:10395000079858224100601C36F008FEF189A01F2C
:10396000084475A136F07EF9F289601C00211154DB
:103970002046FFF781FE6D1C1E2DBEDB08B070BD1A
:1039800010B504468CB001202AF046FD6CA0FFF76C
:1039900073FE6E490A88A2F5194099381FD06CA1B0
:1039A000684636F05FF9224669466BA0FFF78FFE46
:1039B0002046FFF761FE09A90AA80CF004FBBDF838
:1039C000242063A1684636F04DF92246694663A07B
:1039D000FFF77DFE2046FFF74FFE0CB010BD60A242
:1039E00062A1684636F03EF9224669465AA0FFF7C2
:1039F0006EFE2046FFF740FE5D4A5CA1684636F049
:103A000031F9224669465BA0FFF761FE2046FFF7C9
:103A100033FE5A4A55A1684636F024F922466946D3
:103A200057A0C3E710B50420FDF7ABFE01065648CA
:103A300001D5006810BD0021016021480160784671
:103A400052490860002010BD5148002100F8081FAD
:103A5000FF210176017780F820107047F0B5074606
:103A600087B00C460026032022F0FDFC50B1012651
:103A70003046FFF7D7FF002805D18DF800008DF8FC
:103A8000010087E097E0C7E00080004020A1070028
:103A90000A0000008C04001025752E25303175C2F7
:103AA00000000000C1C0D2C0D0C5DF20D7C0D1CE39
:103AB000C228322E32202D20332E33290000000060
:103AC0000C000010CDCED0CC00000000CDC5CDCE76
:103AD000D0CC00002530346420CED8C8C1CECA0076
:103AE00078000010CDC5D200C0CACAD3CCD3CBDF7A
:103AF000D2CED028362E36202D20382E3429000064
:103B0000257525250000000020C7C0D0DFC6C0C530
:103B1000D2D1DF2E2E2E000020C7C0D0DFC400007F
:103B2000CACEC420C7C0D9C8D2DB2025750A000080
:103B3000CDCED0CC0A000000CDC5CDCED0CC0A0071
:103B4000494420D1C5D0C8C83A0A00000404000086
:103B500025303475000000002031000020320000C4
:103B6000CED2CBC0C4CED7CDC0DF000025730000BD
:103B70001004000020C4E0F2E03A0000200400003D
:103B800020C2F0E5ECFF3A00080000101000001021
:103B9000004002408DF8020040F2DA70ADF81400E7
:103BA00001208DF816008DF8170005A822F01DFDE4
:103BB000684622F0F9FC684622F091FCFF499DF826
:103BC00002508868FE4A8B681B1A9342FBD36846F2
:103BD00022F085FC0EB1FFF737FF9DF802006CB1B3
:103BE000A84202D12068401C2060AFF2181101A841
:103BF000226836F037F83A4601A907E0A8423A466B
:103C000002D0AFF2401101E0AFF24011EDA0FFF79A
:103C10005EFD3846FFF730FD07B0F0BD30B50C0053
:103C2000EBA187B00546D1E90001CDE900010ED036
:103C300022F006FD10B12068401C2060AFF26C112C
:103C400002A8226836F00EF82A4602A908E022F0FF
:103C5000F7FC2A4610B1AFF28C1101E0AFF29C11D3
:103C60006846FFF734FD2846FFF706FD07B030BD74
:103C700030B5D9A30C4605460FCB89B08DE80F00AF
:103C800008A908460CF09FF9D7480068D8B1092860
:103C90002A4621D0AFF2B4116846FFF718FD6CB187
:103CA0002068401C2060AFF2D41104A8226835F0CF
:103CB000D9FF2A4604A96846FFF709FD2846FFF701
:103CC000DBFC09B030BD2A46AFF208216846FFF799
:103CD000FEFC002CE7D1F1E7AFF210216846FFF7B8
:103CE000F6FC002CEAD02168491C2160DBE77FB597
:103CF0000C46054618F0B9FB88B1BB482A46006857
:103D0000012809D0AFF23C21B8A0FFF7E0FCC4B114
:103D10002068401C206009E0AFF23821F4E72A4611
:103D2000AFF26021B1A0FFF7D2FC54B1AFF25C2139
:103D30006846226835F096FF2A466946ABA0FFF731
:103D4000C6FC2846FFF798FC7FBD7FB50C460546AC
:103D500025F06AFB38B12A46AFF278210FE02068DF
:103D6000401C206018E00BF080F870B19E4801689C
:103D700003290AD0042908D02A46AFF2B0219DA019
:103D8000FFF7A5FC002CEAD111E02A46AFF2CC21C6
:103D900098A0FFF79CFC54B1AFF2C8216846226896
:103DA00035F060FF2A46694692A0FFF790FC28464E
:103DB000FFF762FC7FBD30B5054690A085B0006876
:103DC0000C46049002F013FF000607D42A46AFF217
:103DD0000C3104A8FFF77BFC74B918E082482A462E
:103DE0000068192817D0AFF2043104A8FFF76FFC60
:103DF0006CB12068401C2060AFF228316846226810
:103E000035F030FF2A46694604A8FFF760FC2846D3
:103E1000FFF732FCDDE4AFF24C31E6E72DE9F04389
:103E2000814677A00C468BB007C801AB002683E81B
:103E3000070001202AF0F0FA08A80BF0CCFD6A4D2B
:103E4000932803D12868062800D0012600210846BF
:103E50000BF011FE002712E02868082815D117B9C9
:103E60006AA0FFF709FCBDF800206FA14846521C6C
:103E700035F0F8FE4846FFF7FFFB01267F1C694638
:103E800000200CF0C5F80028E6D1DFF8A481D8F8AE
:103E90000000932800D10126002101200BF0EBFD4A
:103EA000002712E02868082815D117B961A0FFF78C
:103EB000E3FBBDF800205CA14846521C35F0D2FE61
:103EC0004846FFF7D9FB01267F1C694601200CF00C
:103ED0009FF80028E6D1D8F80000932800D10126E9
:103EE000002102200BF0C7FD002712E028680828F7
:103EF00015D117B956A0FFF7BFFBBDF800204AA1A6
:103F00004846521C35F0AEFE4846FFF7B5FB012689
:103F10007F1C694602200CF07BF80028E6D1D8F817
:103F2000000093280BD09EB14A46AFF2604101A831
:103F3000FFF7CDFBF4B12068401C20600FE028683B
:103F4000802801D08128EFD14A46AFF26841EEE7E0
:103F50004A46AFF2904101A8FFF7B9FB54B1AFF266
:103F60008C4104A8226835F07DFE4A4604A901A8C8
:103F7000FFF7ADFB4846FFF77FFB0BB0BDE8F083D2
:103F8000704770B58AB0064605A80BF024FD20B135
:103F90003F220C2105A836F0E9FA00258DF82050C3
:103FA0002022052105A836F0E1FA324605A92EA007
:103FB000FFF78DFB3046FFF75FFB5DE000800040C0
:103FC000E0C81000D5CEC420D7C0D1CEC2000000BA
:103FD000CFCE20CFC4000000CFCE20CFC0CCDFD2C8
:103FE000C820CFC4000000000C000010DDD1CFCFEE
:103FF000C7D30000CFCFC7D300000000CEC7D30087
:10400000CFE0ECFFF2FC20CFC4000000CFCEC2D046
:10401000C5C6C4C5CDCDDBC520D4C8D1CAC0CBC8A8
:10402000C7C0D6C8C83A0A0023253034750A000034
:1040300008000010CFCEC2D0C5C6C4C5CDCDDBC5EB
:1040400020C0CAD2C8C2C8C7C0D6C8C83A0A000071
:10405000CFCEC2D0C5C6C4C5CDCDDBC520D1CCC561
:10406000CDDB3A0A00000000D1C5D0C8C9CDDBC9FC
:1040700020CDCECCC5D0000000200BF012FDF74CB7
:1040800020B9694600200BF0D0FC28B13F22142152
:1040900005A836F06BFA08E00A23052205A90DF100
:1040A0000B00FCF70AFD00063AD48DF81E5032468C
:1040B00005A9EBA0FFF70BFB3046FFF7DDFA9DF8F3
:1040C00014003F2816D0BDF8000005A9FCF737FD05
:1040D000000625D4324605A9E7A0FFF7F8FA3046D6
:1040E000FFF7CAFAE948007828B301200BF0D9FCA1
:1040F00050B904E0E6A105A836F0A4F8EAE769465D
:1041000001200BF092FC20B1E1A105A836F09AF84D
:1041100009E0BDF8000005A9FCF711FD000602D575
:1041200020680AB070BD324605A9DCA0FFF7CFFABF
:104130003046FFF7A1FADE48256005607846DD4984
:1041400008600020EDE710B58CB004461822DAA113
:1041500005A836F09CF90BA802F0FEFD9DF82C0096
:1041600008B1DBA101E0AFF28461224605A8FFF7A8
:10417000AEFA2046FFF780FA9DF82C00002879D08F
:10418000694600200BF0EFFB002873D1BDF800203A
:10419000D0A101A8521E35F065FD224601A9CFA08D
:1041A000FFF795FA2046FFF767FABDF80000C9A1AE
:1041B000C0F1190201A835F055FD224601A9CCA095
:1041C000FFF785FA2046FFF757FA694602200BF001
:1041D000CAFB00284ED1BDF80020AFF28C6101A8C7
:1041E00035F040FD224601A9C4A0FFF770FA204631
:1041F000FFF742FA04A902200BF086FB002839D110
:10420000BDF81000BDF80010421AAFF2BC6101A861
:1042100035F028FD224601A9B5A0FFF758FA20463F
:10422000FFF72AFA99480078002823D06946012030
:104230000BF099FB00281DD1BDF80020A5A101A815
:1042400035F010FD224601A9AEA0FFF740FA204646
:10425000FFF712FABDF800009EA1C0F1400201A8CC
:1042600035F000FD224601A9A1A0FFF730FA204653
:10427000FFF702FA0CB010BDF0B5074695B00C463A
:104280000025032009F076FE744E000602D5306842
:1042900015B0F0BD09F087FE000605D411A9052070
:1042A00009F0CDFD00060AD514B12068401C20603D
:1042B00001253F220A21684636F058F914E00A2306
:1042C0000522694611A8FCF7F8FB13A9002009F0A4
:1042D000B6FD000608D49DF84C00000604D514B1C4
:1042E0002068401C2060012500208DF80A006A46E5
:1042F00089A105A835F0B6FC44B1AFF628010DA898
:10430000226835F0AFFC3A460DA906E015B1AFF6CC
:10431000440101E0AFF654013A4605A8FFF7D7F98A
:10432000FBF794FF3846FFF7A7F9FBF7A4FFAEE7CA
:1043300070B57C4C0546B222E18936F017F9E18967
:104340000A206854032178A02AF05EFD0024002191
:1043500028462AF0CFFA641C0A2CF8D32AF070FC05
:10436000BDE8704008202AF0B5B810B588B0044602
:104370002021684636F024F96CA00068009022F0F5
:1043800092FD78B11C286BA1684605D035F0E8FF96
:104390002246AFF6C8010BE035F0E2FF2246AFF649
:1043A000DC0105E063A1684635F0DAFF224666A12C
:1043B000FFF78DF92046FFF75FF9284900200860D4
:1043C0003B49086078463B49086008B0002010BDB2
:1043D0002DE9F14F90B028F00AFB204E344FDFF862
:1043E000D490002488B130F061FE109A88B1AFF605
:1043F0000C1159A0FFF76BF91098FFF73DF91098D1
:10440000FFF7B3FF34603C605AE1AFF62811109A11
:10441000F2E01DA150A0FFF75AF91098FFF72CF910
:1044200028F04DFADFF84481002813D1032029F049
:10443000F3FF98F80C0008F10D05012808D00228B8
:1044400009D0032808D04AA1109835F00BFCAEE043
:104450002846ADE0AEE095E0C4E0000008000010A2
:10446000D0C5C3C8D1D2D0C0D6C8CECDCDDBC9202F
:10447000CDCECCC5D0000000C4C0D2C020D0C5C3B2
:10448000C8D1D2D0C0D6C8C8000000008AC103007D
:104490003F3F2D3F3F2D3F3F00000000C4C0D2C032
:1044A00020C7C0CCC5CDDB20DDCACBC700000000D3
:1044B0000C00001010000010CFC0CCDFD2DC20CFE9
:1044C000C420C0CAD2C8C2C8C7C8D02E00000000CD
:1044D000C4C00000253032750000000020CFC5D0D8
:1044E000C5D0C5C3C8D1D2D0C0D6C8C9000000004D
:1044F0002020D1C2CEC1CEC4CDCE000020D1CCC5AB
:10450000CD00000020C0CAD2C8C2C8C7C0D6C8C922
:1045100020DDCACBC7000000DDCACBC72028257329
:10452000290000008C0400101B3300003F3F3F2097
:104530000000000020424C5545544F4F544820D7AE
:10454000C0D1D2DC00000000CDC5D220C7C0C3CB93
:10455000D3D8CAC800000000CCCEC4D3CBDC2042E4
:104560004C5545544F4F54480000000088D907204F
:10457000CDE5E8E7E2E5F1F2EDFBE920ECEEE4F36E
:10458000EBFC0000F5A1284635F01EFE0246F6A120
:10459000109835F067FB1098FFF76EF8F8A1F9480E
:1045A00035F012FE821CF8A1109835F05BFB1098D4
:1045B000FFF762F828F067FA012029F02DFFF5A037
:1045C000FFF75AF8002021F079FAC0B1022029F053
:1045D00023FFF8A1FAA0109AFFF779F81098FFF7D7
:1045E0004BF80FE76421284632F0D6FE00283FF44E
:1045F0002FAFAFF62831109AAFF2A400ECE728F005
:1046000062FA98F808000328DCD100254FF0220B4D
:104610004FF02E0A2BE06A1CEDA1684635F022FB14
:10462000C5EBC50000EB400008EB40018DF80140F0
:104630001E2208A801F2E12135F09EFE08A835F0FF
:1046400025FE1D2809D98DF83E408DF83DB08DF826
:104650003BA08DF83CA08DF83AA008A96846109AB6
:10466000FFF735F81098FFF707F86D1CEDB298F8D2
:10467000D402A842CFD8C2B2D5A1684635F0F2FA2A
:104680006946D4A0109AFFF722F81098FEF7F4FFBD
:1046900098F8D40210B1AFF6D43101E0AFF6D431BE
:1046A000AFF24C10109AFFF712F81098FEF7E4FFE3
:1046B00098F8D00200F0010028F0E6F834603C6081
:1046C0007946C9F8001011B00020BDE8F08F70B530
:1046D0000446012029F0A0FE20F09AFE002830D0E8
:1046E000C1A0FEF7C9FF18E0002021F0E7F9A0B152
:1046F000022029F091FE2246AEA1C3A0FEF7E7FFFB
:104700002046FEF7B9FFC44900200860C34908608D
:104710007846C3490860002070BD20F079FE00286B
:10472000E2D12046FFF704FEBEA0FEF7A5FFC54D6F
:10473000AC68C54E20F06CFE18B9A868001BB042EA
:10474000F8D3BDE87040022029F066BE10B50446DB
:10475000012027F0D5F922F057FAA0F55960B0F5FD
:10476000C04F224602D0AFF69C4101E0AFF6AC410B
:10477000B6A0FEF7ACFF2046BDE81040FEF77CBFB8
:104780002DE9F041B6B000262D962E962F96309644
:10479000319632963396349626A835962AF0BFF98C
:1047A0009D4C000617D42020ADF8A6000220ADF8DD
:1047B000A2000120ADF89A00ADF89C00ADF8980079
:1047C0000820ADF89E00ADF8A460012126A829F0CC
:1047D00023FF000603D5206836B0BDE8F081022033
:1047E0002AF07FFA9AA0FEF747FF012029F014FE75
:1047F0009EA0FEF741FF03202AF059FAA34C0027A0
:10480000002021F05BF948B1022029F005FEA0A0AC
:10481000FEF732FF012029F0FFFD08E02AF0A1FA9F
:1048200020880743BFB27807EAD5B807E8D52AF051
:1048300098FA20880028FAD1824CA068974DA16888
:10484000091AA942FBD396A0FEF716FF012029F012
:10485000E3FD1DA80BF0BFF820B13F220C211DA8DD
:1048600035F084FEB0468DF88060202205211DA819
:1048700035F07CFE03AA1DA98EA0FEF728FF03A831
:10488000FEF7FAFE1CA821F05BFE18B924A821F05F
:1048900026FE20B188A103A835F0D4FC12E0BDF8B3
:1048A00070209DF89110A2F5FA629DF89000009298
:1048B000CDE901019DF872309DF8732083A103A812
:1048C00035F0D0F9032029F0A7FD03A8FEF7D4FEA8
:1048D000012029F0A1FD03A8FFF707F882A285A116
:1048E00003A835F0BFF9002103A82AF003F882A03D
:1048F000FEF7C2FE2AF035FAB80703AA02D5AFF6D2
:104900003C6101E0AFF63C617EA0FEF7E0FE03A84B
:10491000FEF7B2FE780703AA02D5AFF6586101E0B0
:10492000AFF6586179A0FEF7D2FE03A8FEF7A4FE09
:1049300078A0FEF7A1FE0021084627F09DFE012188
:10494000002027F099FE40B90221002027F094FEB4
:1049500018B103AAAFF69461E6E0E3E0566572731E
:10496000696F6E20000000005379732E20436F6E34
:104970006669672E2053657473202D20257300000F
:104980003D200000F9D907204275696C643A202562
:1049900073000000C8C4C5D220CFCEC8D1CA20D36E
:1049A000D1D2D0CEC9D1D2C22E2E2E0A0A0A0A0ADC
:1049B00000000000CFD0CECFD3D9C5CD000000007D
:1049C000D2C5D1D220424C5545544F4F54480000D7
:1049D00025640000D3D1D2D0CEC9D1D2C220CDC05F
:1049E000C9C4C5CDCE000000CED2CACBDED7C8D256
:1049F000C520C2CDC5D8CDC5C520CFC8D2C0CDC871
:104A0000C50A0A0A0A0A0A00D2C5D1D220C1C0D2F8
:104A1000C0D0C5C900000000080000100C00001044
:104A2000100000100AC2CACBDED7C8D2C520C2CD42
:104A3000C5D8CDC5C520CFC8D2C0CDC8C50A0A0AC1
:104A40000A0A0A000080004080C3C9015553420091
:104A50003D20D2C5D5CDCECBCEC3C8D7C5D1CAC8CF
:104A6000C920CFD0CEC3CECD203D0A00D2C5D1D2F1
:104A700020C4C0D2D7C8CACEC220CAD0DBD8CAC8C8
:104A800020C820C1D3CCC0C3C80A0000E80200106F
:104A9000CFD0CECFD3D9C5CD0A00000020A10700CA
:104AA0003D3D3D2020CFD0CEC3CECD203120203D76
:104AB0003D3D0A00CFC4000058582D58582D585875
:104AC00058582058583A58580A0000002530327576
:104AD0002D253032752D2530327520253032753A2E
:104AE000253032750A000000465072696E742D310F
:104AF0003100000025730A00C4C0D2D7C8CAC80A52
:104B00000000000020CAD0DBD8CAC80020C1D3CC26
:104B1000C0C3C80052533233322D310A200A200A52
:104B200000000000F94903AAF9A0FEF7D0FD03A890
:104B3000FEF7A2FDF9A0FEF79FFD03202AF0B7F8CB
:104B4000002020F0BBFF08B1012700E00027012171
:104B5000002027F091FD30B10221002027F08CFDCC
:104B600008B1012600E000263743E9D0032029F0F0
:104B700053FC0EB1ECA000E0EEA0FEF77DFD01209D
:104B800029F04AFC0321002027F076FD002020F0C8
:104B900095FF0028FAD1EAA0FEF76EFD0021022061
:104BA00027F06AFD0121022027F066FD40B90221AD
:104BB000084627F061FD18B1D44903AA083901E07D
:104BC000D24903AAD2A0FEF782FD03A8FEF754FD46
:104BD000D2A0FEF751FD03202AF069F8002020F052
:104BE0006DFF08B1012700E000270121022027F016
:104BF00043FD30B10221084627F03EFD08B10126F1
:104C000000E000263743E9D0032029F005FC0EB16F
:104C1000C5A000E0C7A0FEF72FFD012029F0FCFB96
:104C20000321022027F028FDA068A168091AA942E3
:104C3000FBD3002020F042FF0028FAD103A8FFF7A1
:104C400085FD03A8FFF7C4FB002103A8FEF706FFBC
:104C5000002103A8FEF789FD002103A8FEF7DEFF6F
:104C6000002103A8FFF704F8002103A8FFF7A3F829
:104C7000002103A8FFF73BF8002103A8FFF765F820
:104C8000002103A8FFF7CAF803A8FFF75CFA002188
:104C900003A8FFF7F1FA47462CA91320CDF8B080FE
:104CA00016F0C3FC08B164202C90A9A11DA82C9A71
:104CB00034F0D8FF03AA1DA9A6A0FEF708FD03A89B
:104CC000FEF7DAFC29F0BCFF03A8FFF731FBAFF2D7
:104CD0003820FEF7D1FC03A8FFF7F9FC012029F0EA
:104CE0009BFB9FA0FEF7C8FC032029F0E0FFA6680D
:104CF000002020F0E3FE00B1A668A068801BA84257
:104D0000F6D3824903AA083997A0FEF7E0FC03A86E
:104D1000FEF7B2FC97A0FEF7AFFC032029F0C7FF17
:104D2000A668002020F0CAFE00B9A668A068801B13
:104D3000A842F6D3032029F06FFB74486430FEF7D5
:104D40009BFC012029F068FB002020F0B7FE002822
:104D5000FAD18BA0FEF790FC032029F0A8FF8B4E20
:104D600007E000BF20F0E3FEA068A168091AB14285
:104D7000FBD3002020F0A2FE00284FF00300F1D06A
:104D800020F0B7FE022020F0A7FE03AA80A168A0B1
:104D9000FEF79DFC03A8FEF76FFC7FA0FEF76CFCFE
:104DA000032029F084FF4FF4FA76C821304620F022
:104DB000A1F9A068A168091AA942FBD3002020F03C
:104DC0007DFE0028F1D003AA71A159A0FEF77FFC57
:104DD00003A8FEF751FC002020F070FE0028FAD155
:104DE000012029F019FB20F013FB00287ED06DA0D4
:104DF000FEF742FC032029F00FFB29F0B2FF6F4DB4
:104E00002878400702D44148643001E03F486C30C4
:104E1000FEF732FC012029F0FFFA69A0FEF72CFC16
:104E2000032029F044FF694E29F00BFAA068A1681D
:104E3000091AB142FBD3002020F040FE0028F3D035
:104E4000022029F0E9FA62A0FEF716FC012029F001
:104E5000E3FA62A0FEF710FC032029F028FF29F0F6
:104E600080FF032029F0D8FA2878400702D5274888
:104E7000643001E025486C30FEF7FEFB03A8FEF726
:104E80007FFD29F0DDFEADF8947025A9392016F0DC
:104E9000CCFBADF8887022A93A2016F0C6FB1B495E
:104EA000BDF8882084311DA834F0DCFE03AA1DA9BA
:104EB0004DA0FEF70CFC03A8FEF7DEFBBDF8942026
:104EC0004DA11DA834F0CEFE03AA1DA94DA0FEF7EA
:104ED000FEFB03A8FEF7D0FB542016F070F92BA8B8
:104EE00001F004F82BA800F0E5FB00E005E02BA89A
:104EF00000F0F2FF0125464E12E103AAAFF24C5139
:104F000044A0FEF7E4FB03A8B6E70000CC3A00009B
:104F100020D0C0C7CCDBCAC0CDC8C50020C7C0CC1C
:104F2000DBCAC0CDC8C5000020CDCED0CC0A0A0A4D
:104F30000000000020CDC5CDCED0CC0A0A0A00006A
:104F400052533233322D320A200A200A0000000068
:104F500025750000DFD0CACED1D2DC20D7CB00002F
:104F6000CACDCECFCAC00A00D0C0C7CCDBCAC0CD24
:104F7000C8C50000C7C0CCDBCAC0CDC8C50A0A007E
:104F8000C8CDC4C8CAC0D2CED0DB0000400D0300DB
:104F9000CFD0CEC9C4C5CD00C4C8CDC0CCC8CA0A04
:104FA00000000000C4C5CDC5C6CDDBC920DFD9C80F
:104FB000CA0A20C7C0CAD0DBD20A0000E60200102D
:104FC000D2C5D1D220C7C0CCCAC00A0000350C005F
:104FD000CFD0CEC9C4C5CD0A0000000020CED2CAB1
:104FE000D0DBD20A00000000D7C8D1CBCE20D6C873
:104FF000CACBCEC2000000002530347520D1C5CA0E
:1050000000000000C7C0C4C5D0C6CAC00000000070
:1050100002000010C4C5CDC5C6CDDBC920DFD9C88C
:10502000CA000000308840F00200308001200DF0FE
:1050300015FC012029F0F0F9BDF888302A464DA171
:1050400003A834F00FFE03A8FEF716FB1CA821F0FE
:1050500077FA18B924A821F042FA28B1AFF2A85182
:1050600003A835F0EFF813E0BDF870209DF891002B
:10507000A2F5FA629DF890100092CDE901109DF81A
:1050800072309DF87320AFF2BC5103A834F0EAFDF2
:10509000032029F0C1F903A8FEF7EEFA012029F058
:1050A000BBF929F0CDFD03A8FFF742F9AFF2186074
:1050B000FEF7E2FA2DA903A8FEF7D0FC2EA903A85B
:1050C000FEF753FB2FA903A8FEF7A8FD30A903A8FC
:1050D000FEF7CEFD32A903A8FEF76DFE33A903A8A3
:1050E000FEF705FE34A903A8FEF72FFE31A903A899
:1050F000FEF794FE35A903A8FFF7BEF8A76803E002
:10510000002020F0DBFC80B9A06843F60951C21BE7
:10511000BDF894004843B2EB801FF1D36D1CADB2D3
:10512000BDF8880085427FF67DAF552016F047F820
:105130002BA800F0DBFE2BA800F0BCFA2BA800F097
:10514000CBFE308840F00200308001200DF086FB5D
:105150000DA0FEF791FA032029F05EF913A0FEF7E7
:105160008BFA308840F00200308001200DF076FB91
:10517000FEE70000D6C8CACB202530347520C8C74A
:1051800020253034750A00003DD2C5D5CDCECBCE1A
:10519000C3C8D7C5D1CAC8C920D2C5D1D220C7C0BB
:1051A000C2C5D0D8C5CD3D0A0A0A0A0028CFCEC450
:1051B000CFC8D1DC290A0A00F0B5036802790D686E
:1051C000002462F30704EB18002242EB0401FE4DB9
:1051D000FE4EDFF8FCC30C0A04D1FE4FE824FF1A90
:1051E0008C4108D289202860012030607846CCF8B4
:1051F00000008920F0BD036001712A6078463260AA
:10520000CCF800000020F0BDF0B500230C681A4671
:105210000979057961F30702016865F307036118ED
:105220005A41E94CE94DEA4E130A04D1E94FE8230B
:105230007F1A934107D28920206001202860784698
:1052400030608920F0BD016002710020206028607C
:10525000784630600020F0BDF0B503680968002290
:10526000CB18D94CD94DDA4E52EB020106D1DFF8FA
:1052700064C3E827BCEB030C8F4107D28920206070
:1052800001202860784630608920F0BD03602260EC
:1052900078462A6030600020F0BDF0B503680968E8
:1052A0000022CB18C84CC94DC94E52EB020106D1A1
:1052B000DFF824C30227BCEB030C8F4107D28920FF
:1052C000206001202860784630608920F0BD0360AE
:1052D000226078462A6030600020F0BD30B5026858
:1052E0000968B94BB94CBA4D8A4207D28920186077
:1052F0000220206078462860892030BD511A016064
:1053000000201860206078462860002030BDF0B58D
:10531000036809680022CB18AB4CAC4DAC4E52EB85
:10532000020106D1DFF8B0C20227BCEB030C8F41AB
:1053300007D28920206001202860784630608920CB
:10534000F0BD0360226078462A6030600020F0BD26
:1053500030B5026809689C4B9C4C9D4D8A4207D22F
:10536000892018600220206078462860892030BD9E
:10537000511A0160002018602060784628600020E3
:1053800030BD10B502880988904B11448E4A904C6C
:10539000B1F5803F07D3892010600120186078465E
:1053A0002060892010BD01800020106018607846C0
:1053B0002060002010BD0021016001718248016061
:1053C00082480160784682490860002070470021C9
:1053D0000160818081717C4801607C480160784671
:1053E0007B490860002070471CB50023CDE90033DD
:1053F000036800938388ADF8043080798DF8060047
:1054000000201060DDE900340968CB1A70EB04035A
:1054100001D2411E05E0DDE90043611A834101D25A
:105420000121116068490860684908607846684948
:10543000086000201CBD2DE9FC410022CDE90022BE
:10544000026800928288ADF8042082798DF80620E7
:10545000DDE900430A680021141941EB0302CDE99C
:105460000042150E584A594B594C08D1DDE90067E6
:10547000DFF868C15A4DBCEB0606BD4108D2892051
:10548000106001201860784620608920BDE8FC810A
:10549000009D0560BDF8045085809DF8065085711B
:1054A00011607846196020600020EFE72DE9FC418B
:1054B0000022CDE90022026800928288ADF8042023
:1054C00082798DF80620DDE900730A6800213E4CE0
:1054D0003E4D3F4EBF1A8B4107D2892020600120EC
:1054E0002860784630608920D0E7DDE90073BA1A79
:1054F00063EB0103CDE900230260BDF80420828044
:105500009DF8062082712160784629603060002075
:10551000BCE72DE9FC410022CDE900220B680979A6
:1055200061F30702016800918188ADF80410817968
:105530008DF80610DDE900145B186241CDE90032F8
:10554000140E2149214A224B06D1DDE90056234F92
:10555000234C7D1BB44107D28920086001201060D4
:1055600078461860892091E7009C0460BDF80440EB
:1055700084809DF8064084710020086010607846A1
:105580001860002082E72DE9F041054600680968AF
:105590000024A1FB002304FB003001FB04014FF4B5
:1055A000FA70101841F100014FF47A72234634F07A
:1055B000BDFA054A054B064EA9B9DFF81CC0022703
:1055C000BCEB000C8F410DE0080000100C00001037
:1055D00010000010FF0FA5D4FFE30B54FFFF63A7DB
:1055E000B3B6E00D08D28920106003201860784619
:1055F00030608920BDE8F0812860146078461C6026
:1056000030600020F6E72DE9F04105460068098882
:105610000024A1FB002304FB003001FB040141F244
:105620008830101841F1000142F21072234634F024
:105630007DFA4E4A4E4B4F4E31B9DFF83CC102273E
:10564000BCEB000C8F4107D289201060032018604A
:10565000784630608920CDE72860146078461C6069
:1056600030600020C6E7018842F20F72491C89B2FF
:105670000180914201D9012101803C49002008604C
:105680003B49086078463B49086000207047018824
:1056900042F20F72491E89B20180914200D9028004
:1056A0003249002008603249086078463149086074
:1056B000002070470168314A491C0160914201D9BC
:1056C00001210160294900200860294908607846C5
:1056D00028490860002070470168284A491E016077
:1056E000914200D9026021490020086020490860E9
:1056F000784620490860002070472DE9F0410446B3
:10570000D1E90001D4E90023A0FB025601FB0261AC
:1057100000FB0311681949418018594142F2107584
:10572000401941F10001521943F1000392185B4105
:1057300034F0FCF90D4B0E4D0E4E0A0A04D1104FF9
:10574000E8223F1A8A4107D2892018600320286086
:105750007846306089204DE7C4E9000100201860D8
:10576000286078463060002044E700000800001000
:105770000C00001010000010FFE30B54FFE0F505D3
:10578000FF0FA5D42DE9FF4718F0FCF96E4C000679
:1057900015D401F0BBFFDFF8B481DFF8B4916D4F91
:1057A000002668B1012820D087281DD0684601F066
:1057B00081F8000603D49DF800000E287ED0AEE0EC
:1057C000684601F077F8000679D403A801F099F84B
:1057D000000674D49DF800000E2805D1BDF80C0019
:1057E000402801D17120387089E0684601F062F8E4
:1057F000000664D49DF800001D2827D2DFE800F0E1
:10580000260F2222222214141414141414140F121A
:10581000121212120F2424242426121212001CF039
:1058200081FA03E0202000E06020387002F01CF8CC
:10583000000674D49DF80000474D0E2811D017289B
:1058400012D014E05020F0E73020EEE78820092144
:105850002060C8F800107946C9F8001004B0BDE80F
:10586000F0870DF0C7F805E02878022844D0012021
:105870000CF0F4FF000652D49DF80000172806D162
:105880002878012835D11CF0BDFA000647D49DF8D0
:1058900000000E2825D12878022826D109F03DFCE9
:1058A000D8B901A806F035FF000638D40DF106007E
:1058B00006F013FF000632D4284801E027E02EE06E
:1058C00000788DF8080017208DF8090001A801F074
:1058D000D3FE000623D4322038709DF800000E2835
:1058E00003D0C0B2172804D009E02878032803D0D9
:1058F00005E02878022802D102F0C3F92E70266054
:105900007946C8F800600020C9F80010A6E7FAF749
:105910009DFC1CF007FAFAF7AEFC01F0A5FF206829
:105920009CE708B5684600F089FA58B99DF8000070
:10593000082807D0092805D00A2803D0084800887D
:10594000002800D0012008BD080000100C00001045
:105950001000001090C2072048C1072091C2072004
:10596000700100102DE9F843CD4ECE4FCE4C0546C8
:105970004FF08808B0F1004F06D0B5F1104F03D0BA
:105980000220C4F800800AE0684601F029F9000608
:1059900028D49DF8000040B10A20C4F8008030608F
:1059A000784638608820BDE8F88301226946284699
:1059B00026F074F8000615D49DF80000FF2809D0E1
:1059C000FF208DF8000001226946284626F071F874
:1059D000000607D4280F8DF80000684601F0F6F89D
:1059E000000601D52068DEE7B049012008700020DC
:1059F000486020603060784638600020D3E7AB49CB
:105A000000200870A8490860A54908607846A549A3
:105A1000086000207047A54901200870A2490020B5
:105A200008609F49086078469E49086000207047DA
:105A3000F8B5684601F0D4F89B4D000618D49DF8DF
:105A40000000974E974FA8B19849002400070C70AA
:105A5000FF218DF800100122694626F02AF8000681
:105A600006D48DF80040684601F0B0F8000609D56C
:105A70002868F8BD882028600A20306078463860A1
:105A80008820F8BD2C607846346038600020F8BD6E
:105A90002DE9F74F92B0144610A801F0A1F8824DFD
:105AA000000649D49DF84000DFF8F481DFF8F49156
:105AB0008827B0B10607304626F007F87B4A401E1B
:105AC0004FF0000A51680B195B1D98420ED22F60EF
:105AD000C8F800A079468820C9F8001015B0BDE8C4
:105AE000F08F0A212F60C8F80010F3E746EA01079B
:105AF0008DF800401298ADF8010093466E4622469C
:105B0000F01C139934F038FC3019FF21C470017176
:105B1000221D711C781C25F0CCFF00060CD4092036
:105B2000B0EB177F01D1621D00E0012269463846C3
:105B300025F0BFFF000601D52868CFE7DBF8041089
:105B40002144091DCBF80410C5F800A07946C8F817
:105B500000A00020C9F80010C0E72DE9F04F524D19
:105B60004F4F99B0D5F8009016A8D7F800A001F0D3
:105B700037F8000664D49DF85800DFF82881040740
:105B800000264FF0010B012201A9204625F086FFD7
:105B9000000655D49DF80400F0B3FF284AD0044411
:105BA000241D04F0704025F090FF24F07041401E49
:105BB000884211D39DF8040040280DD8761CE2E7F6
:105BC000641E012201A9204625F068FF000637D493
:105BD0009DF80400402808D9882028607946C7F835
:105BE00000B0C8F8001019B079E7241AA41E0222E8
:105BF00015A9204625F052FF000621D4A41C9DF8CB
:105C0000042002A9204625F049FF000618D4BDF85B
:105C1000540040F0005000E00CE09DF8042002A980
:105C200025F047FF00060BD49DF8040021180C1A3C
:105C3000E41E761E002EC3D1FFF7FAFE000601D542
:105C40002868D0E7C5F800907946C7F800A0484614
:105C5000C8F80010C7E708B5684600F0C1FF08B1F2
:105C6000002008BD9DF800000028FAD0000701229E
:105C7000694625F013FF000605D50B48006800288B
:105C8000EFD0012008BD9DF8000008B1FF28F8D131
:105C900000208DF80000684600F098FFE0E7000063
:105CA0000C000010100000100800001040C1072078
:105CB0002DE9F0418046F84816461D4600780F460B
:105CC00080B11A46404625F0E9FEF44C000606D4A1
:105CD0002A4639464046FFF7DBFE000602D520681B
:105CE000BDE8F0812A4631464046BDE8F04125F046
:105CF000E0BE38B5022269464FF0704025F0CEFE76
:105D0000E64C000602D5208885B201E0BDF80050BF
:105D100001F092F8E249E34A854206D10020206072
:105D2000086078461060002038BD8820206011206F
:105D3000086078461060882038BD2DE9FF4FD74CA9
:105D4000D74ED84F81B0994692468B4600254FF0EA
:105D500070484A465146019825F0ABFE000611D422
:105D600001F06AF8ADF8000002226946404625F0CD
:105D7000A0FE000606D44A465946019825F08EFE3C
:105D8000000603D5206805B0BDE8F08F4A465146AD
:105D9000584634F02BFA10B9FFF7ABFF58B16D1C21
:105DA000ADB2032DD5D3822020602220306078460A
:105DB00038608220E7E70020206030607846386055
:105DC0000020E0E700B587B00246B7481C236946CB
:105DD000FFF7B3FF07B000BDC0EBC000401F40F0AD
:105DE0007040072225F05ABE38B5B04C0246012358
:105DF00069462046FFF75CFF38BDAC4B01460122E7
:105E0000184625F04BBE38B5A84C0246641C012349
:105E100069462046FFF74CFF38BDA44B01465B1C8A
:105E20000122184625F03ABE38B5A04C0246A41C03
:105E3000012369462046FFF73BFF38BD9B4B0146D7
:105E40009B1C0122184625F029BE38B5974C024606
:105E5000E41C012369462046FFF72AFF38BD934B17
:105E60000146DB1C0122184625F018BE38B58F4CC0
:105E70000246241D012369462046FFF719FF38BD5D
:105E80008A4B01461B1D0122184625F007BE1CB592
:105E9000C0EBC00026300A4640F000500723694698
:105EA000FFF706FF1CBDC0EBC000263040F00050DD
:105EB000072225F0F3BD38B57C4C02464B34012354
:105EC00069462046FFF7F4FE38BD784B01464B3358
:105ED0000122184625F0E2BD38B5744C02464C3418
:105EE000042369462046FFF7E3FE38BD6F4B0146A9
:105EF0004C330422184625F0D1BD38B56B4C024610
:105F00005034022369462046FFF7D2FE38BD674B66
:105F1000014650330222184625F0C0BD38B5634C07
:105F200002465234042369462046FFF7C1FE38BDBD
:105F30005E4B014652330422184625F0AFBD38B5FA
:105F40005A4C02465634022369462046FFF7B0FEFB
:105F500038BD564B014656330222184625F09EBDE9
:105F600038B5524C02465834022369462046FFF7A2
:105F70009FFE38BD4D4B014658330222184625F08E
:105F80008DBD38B5494C02465A3401236946204636
:105F9000FFF78EFE38BD454B01465A3301221846A5
:105FA00025F07CBD38B5414C02465B34042369467C
:105FB0002046FFF77DFE38BD3C4B01465B33042293
:105FC000184625F06BBD832208B502EB80000A4617
:105FD00040F0005004236946FFF76AFE08BD8322A3
:105FE00002EB800040F00050042225F057BD38B588
:105FF0002E4C02468734042369462046FFF758FE9C
:1060000038BD2A4B014687330422184625F046BD89
:1060100038B5264C02468B34022369462046FFF7EA
:1060200047FE38BD214B01468B330222184625F02E
:1060300035BD38B51D4C02468D34042369462046D3
:10604000FFF736FE38BD194B01468D330422184642
:1060500025F024BD38B5154C02469134022369461B
:106060002046FFF725FE38BD104B01469133022232
:10607000184625F013BD38B50C4C02469334012365
:1060800069462046FFF714FE38BD084B014693339E
:106090000122184625F002BD40C10720080000106B
:1060A0000C00001010000010020000F0280000207A
:1060B00038B5FA4C0246042369462046FFF7F8FD3E
:1060C00038BD38B5F54C0246241D042369462046E8
:1060D000FFF7EEFD38BD38B5F04C02460834042316
:1060E00069462046FFF7E4FD38BDEC4B0146083316
:1060F0000422184625F0D2BC38B5E84C02460C34D0
:10610000012369462046FFF7D3FD38BDE34B014626
:106110000C330122184625F0C1BC38B5DF4C0246CD
:106120000D34042369462046FFF7C2FD38BDDB4B22
:1061300001460D330422184625F0B0BC38B5D74CC3
:1061400002461134022369462046FFF7B1FD38BDEF
:10615000D24B014611330222184625F09FBC38B5B8
:10616000CE4C02461334022369462046FFF7A0FDB9
:1061700038BDCA4B014613330222184625F08EBCA7
:10618000CD2208B502EB80000A4640F000500423FF
:106190006946FFF78DFD08BDCD2202EB800040F07F
:1061A0000050042225F07ABC40F20D1208B502EB33
:1061B00080000A4640F0005004236946FFF778FD4E
:1061C00008BD40F20D1202EB800040F000500422A6
:1061D00025F064BC38B5B14C0246953404236946B9
:1061E0002046FFF765FD38BDAC4B014695330422D0
:1061F000184625F053BC38B5A84C02469934042300
:1062000069462046FFF754FD38BDA44B014699333B
:106210000422184625F042BC38B5A04C02469D34F5
:10622000012369462046FFF743FD38BD9B4B0146DD
:106230009D330122184625F031BC38B5974C0246F3
:106240009E34042369462046FFF732FD38BD934B48
:1062500001469E330422184625F020BC38B58F4CE9
:106260000246A234042369462046FFF721FD38BDCB
:106270008A4B0146A2330422184625F00FBC38B5DC
:10628000864C0246A634042369462046FFF710FDDB
:1062900038BD824B0146A6330422184625F0FEBBCA
:1062A00038B57E4C0246AA34012369462046FFF7E2
:1062B000FFFC38BD794B0146AA330122184625F070
:1062C000EDBB38B5754C0246AB3402236946204617
:1062D000FFF7EEFC38BD714B0146AB330222184686
:1062E00025F0DCBB38B56D4C0246AD34042369465D
:1062F0002046FFF7DDFC38BD684B0146AD33042274
:10630000184625F0CBBB38B5644C0246B1340123A6
:1063100069462046FFF7CCFC38BD604B0146B133DF
:106320000122184625F0BABB38B55C4C0246B2349F
:10633000012369462046FFF7BBFC38BD574B014699
:10634000B2330122184625F0A9BB38B5534C02469A
:10635000B334022369462046FFF7AAFC38BD4F4BF1
:106360000146B3330222184625F098BB38B54B4C92
:106370000246B534042369462046FFF799FC38BD30
:10638000464B0146B5330422184625F087BB38B585
:10639000424C0246B934042369462046FFF788FC84
:1063A00038BD3E4B0146B9330422184625F076BB72
:1063B00038B53A4C0246BD34042369462046FFF7FF
:1063C00077FC38BD354B0146BD330422184625F015
:1063D00065BB38B5314C0246C134042369462046BA
:1063E000FFF766FC38BD2D4B0146C1330422184629
:1063F00025F054BB38B5294C0246C5340123694603
:106400002046FFF755FC38BD244B0146C533012219
:10641000184625F043BB1CB500EB800000F27D1050
:106420000A4640F0005005236946FFF741FC1CBDB9
:1064300000EB800000F27D1040F00050052225F0B6
:106440002DBB4FF4CA7208B502EB40000A4640F07B
:10645000005002236946FFF72BFC08BD4FF4CA72B7
:1064600002EB400040F00050022225F017BB4FF431
:10647000CE7208B502EB40000A4640F000500223FD
:106480006946FFF715FC08BD4FF4CE7202EB4000E1
:1064900040F00050022225F001BB0000BC000020AB
:1064A0001CB500EB800001EB810100EB810000F2E4
:1064B0008D1040F0005005236946FFF7F9FB1CBD25
:1064C00000EB800001EB810100EB8100134600F23C
:1064D0008D1040F000500522194625F0DFBA090161
:1064E00008B501EB800000F2D22040F000500423F8
:1064F0006946FFF7DDFB08BD090101EB800013468B
:1065000000F2D22040F000500422194625F0C6BA0D
:106510001CB500EB800001EB810100EB810000F273
:10652000CD3040F0005005236946FFF7C1FB1CBD8C
:1065300000EB800001EB810100EB8100134600F2CB
:10654000CD3040F000500522194625F0A7BA38B5E5
:10655000F84C0246042369462046FFF7A9FB38BDE4
:10656000F44B01460422184625F098BA1CB500EBFE
:10657000800000F225500A4640F00050052369468D
:10658000FFF796FB1CBD00EB800000F2255040F0A9
:106590000050052225F082BA38B5E64C0246183480
:1065A000042369462046FFF783FB38BDE14B0146D3
:1065B00018330422184625F071BA1CB500EB800090
:1065C00000F23D500A4640F0005005236946FFF7AF
:1065D0006FFB1CBD00EB800000F23D5040F000500E
:1065E000052225F05BBA1CB500EB800000F251508B
:1065F0000A4640F0005005236946FFF759FB1CBDD1
:1066000000EB800000F2515040F00050052225F0D0
:1066100045BA1CB500EB800000F265500A4640F018
:10662000005005236946FFF743FB1CBD00EB8000CB
:1066300000F2655040F00050052225F02FBA1CB53D
:1066400000EB800001EB810100EB810000F265505E
:1066500040F0005005236946FFF72AFB1CBD00EB04
:10666000800001EB810100EB8100134600F26550D0
:1066700040F000500522194625F010BA1CB500EB79
:10668000800001EB810100EB810000F22D6040F001
:10669000005005236946FFF70BFB1CBD00EB800093
:1066A00001EB810100EB8100134600F22D6040F008
:1066B00000500522194625F0F1B91CB500EB800009
:1066C00001EB810100EB810000F60D0040F000506D
:1066D00005236946FFF7ECFA1CBD00EB800001EBD7
:1066E000810100EB8100134600F60D0040F00050E0
:1066F0000522194625F0D2B91CB500EB800000F642
:1067000079200A4640F0005005236946FFF7D0FA89
:106710001CBD00EB800000F6792040F000500522FF
:1067200025F0BCB940F6862208B502EB40000A46C7
:1067300040F0005002236946FFF7BAFA08BD40F660
:10674000862202EB400040F00050022225F0A6B95C
:106750001CB500EB800001EB810100EB410000F66D
:106760007D2040F0005005236946FFF7A1FA1CBDCB
:1067700000EB800001EB810100EB4100134600F6C5
:106780007D2040F000500522194625F087B940F6DB
:10679000EE2208B502EB40000A4640F0005002230A
:1067A0006946FFF785FA08BD40F6EE2202EB40008D
:1067B00040F00050022225F071B940F6F62208B5EB
:1067C00002EB40000A4640F0005002236946FFF702
:1067D0006FFA08BD40F6F62202EB400040F0005090
:1067E000022225F05BB938B5534C024602236946B4
:1067F0002046FFF75DFA38BD4F4B0146022218468E
:1068000025F04CB938B54C4C0246A41C022369460D
:106810002046FFF74DFA38BD474B01469B1C02222C
:10682000184625F03BB938B5434C0246241D0123D8
:1068300069462046FFF73CFA38BD38B53E4C024663
:10684000641D022369462046FFF732FA38BD3A4BF1
:1068500001465B1D0222184625F020B938B5364C9A
:106860000246E41D022369462046FFF721FA38BD9F
:10687000314B0146DB1D0222184625F00FB938B511
:106880002D4C02460934012369462046FFF710FAD1
:1068900038BD294B014609330122184625F0FEB8C0
:1068A00038B5254C02460A34012369462046FFF7D5
:1068B000FFF938BD204B01460A330122184625F066
:1068C000EDB840F6093208B502EB40000A4640F048
:1068D000005002236946FFF7EBF908BD40F6093284
:1068E00002EB400040F00050022225F0D7B838B546
:1068F000114C02464134022369462046FFF7D8F97D
:1069000038BD0D4B014641330222184625F0C6B86A
:1069100038B5094C02464334022369462046FFF746
:10692000C7F938BD044B014643330222184625F00F
:10693000B5B8000026050020000B002038B5FC4C3F
:106940000246042369462046FFF7B2F938BDF84BEA
:1069500001460422184625F0A1B838B5F44C024689
:10696000241D042369462046FFF7A2F938BDF04BE9
:1069700001461B1D0422184625F090B838B5EC4C92
:1069800002460834042369462046FFF791F938BDD2
:10699000E74B014608330422184625F07FB81CB5A2
:1069A00000EB800000F64C300A4640F00050052312
:1069B0006946FFF77DF91CBD00EB800000F64C3006
:1069C00040F00050052225F069B838B5D84C024691
:1069D0002034042369462046FFF76AF938BDD44BBA
:1069E000014620330422184625F058B838B5D04C5B
:1069F00002462434012369462046FFF759F938BD81
:106A0000CB4B014624330122184625F047B840F607
:106A1000663208B502EB80000A4640F000500423BD
:106A20006946FFF745F908BD40F6663202EB800083
:106A300040F00050042225F031B81CB500EB800076
:106A400001EB810100EB810000F6653040F0005061
:106A500005236946FFF72CF91CBD00EB800001EB14
:106A6000810100EB8100134600F6653040F00050D4
:106A70000522194625F012B81CB500EB800001EB89
:106A8000810100EB810000F6C93040F00050052381
:106A90006946FFF70DF91CBD00EB800001EB810199
:106AA00000EB8100134600F6C93040F0005005228B
:106AB000194624F0F3BF40F61E5208B502EB8000E1
:106AC0000A4640F0005004236946FFF7F1F808BD7C
:106AD00040F61E5202EB800040F00050042224F0E9
:106AE000DDBF38B5934C0246012369462046FFF7C7
:106AF000DFF838BD8F4B01460122184624F0CEBF87
:106B000038B58C4C0246641C042369462046FFF7C6
:106B1000CFF838BD874B01465B1C0422184624F091
:106B2000BDBF38B5834C0246641D04236946204628
:106B3000FFF7BEF838BD7F4B01465B1D04221846A7
:106B400024F0ACBF38B57B4C0246093404236946B7
:106B50002046FFF7ADF838BD764B014609330422D5
:106B6000184624F09BBF38B5724C02460D340423FE
:106B700069462046FFF79CF838BD6E4B01460D3341
:106B80000422184624F08ABF38B56A4C02461134F4
:106B9000022369462046FFF78BF838BD654B014656
:106BA00011330222184624F079BF38B5614C0246F1
:106BB0001334022369462046FFF77AF838BD5D4B4F
:106BC000014613330222184624F068BF38B5594CE9
:106BD00002461534012369462046FFF769F838BD9F
:106BE000544B014615330122184624F057BF2DE9B6
:106BF000F84304226946002020F0E0FF4E4C0006D6
:106C00000FD44E49009882274D4D4E4E4FF0190833
:106C100088420DD104226946104620F0CFFF0006BD
:106C200002D52068BDE8F88347490098884206D01D
:106C300027607846C5F8008030608220F2E70020A7
:106C400020602860784630600020EBE72DE9F043B3
:106C5000394EDFF8EC80DFF8EC9091B000254FF46E
:106C6000005700246119684600F0FAF820226946AE
:106C7000204621F0B9F800060ED42034BC42F1D3EE
:106C800000246119684600F0EBF8202208A920468C
:106C900020F094FF000603D5306811B0BDE8F08302
:106CA000202208A9684633F0A1FA40B182201921B8
:106CB0003060C8F800107946C9F80010EDE72034BC
:106CC000BC42DED3ED1DFF2DCBD9002030607946CC
:106CD000C8F80000C9F80010DFE770B58CB00020DC
:106CE0008DF8240015480A9024226946042020F0DB
:106CF00065FF114D000617D4FFF7A8FF000613D457
:106D000000244FF40056012209A9204621F06CF816
:106D1000000609D4641CB442F5D324226946042039
:106D200021F062F8000611D528680CB070BD000093
:106D3000450B0020620D0020080000109CE63496F0
:106D40000C00001010000010CEFAADDE04220AA9DB
:106D5000002021F049F8E8E738B5044669460020EC
:106D600008F001FE0106434801D5006838BDBDF8B2
:106D7000001001B101212170002101603E48016035
:106D800078463E490860002038BDFF2008F025BF46
:106D900010B588B06846C11D06F0A4FA354C00064F
:106DA0000BD40DF10E00FEF712FB000605D40DF119
:106DB0001500FEF70CFB000602D5206808B010BDD8
:106DC0006846FEF7FFFFF9E738B5FEF792FF294C5A
:106DD00048B36846FFF7C0FF00061FD49DF80000C7
:106DE000F0B1702014F0EBF9000617D4712014F004
:106DF000E6F9000612D46F2014F0E1F900060DD474
:106E0000FFF7C6FF000609D4722014F0D8F9000677
:106E100004D46F2014F0D3F9000604D5206838BDDF
:106E2000FFF7B6FFF8E714490020206008607846B5
:106E300012490860002038BD00B589B01E2269469D
:106E4000D00624F02BFE000604D50A48008880B244
:106E500009B000BD1C210DF10200F9F75FFAF7E758
:106E60005FF0000200F8011B491C521C202AF9D3D4
:106E700070470000080000100C0000101000001007
:106E80007FB5054603A8FEF7D9FF264C000640D47F
:106E90009DF80C00012832D00026022809D0872056
:106EA000206021480660784620490860872004B0A9
:106EB00070BD002005F064FC00062AD42888ADF8D7
:106EC00004006888ADF8060028798DF808008DF870
:106ED000096001A804F070FB00061AD469462B2053
:106EE00014F0D8FA000614D411489DF80010007868
:106EF000C90704D0012802D001208DF80C0003A896
:106F0000FEF7A3FF000604D4284601F0FDFE0006AC
:106F100001D52068CBE703208DF80C0003A8FEF70D
:106F200083FFC4E7080000100C00001010000010E0
:106F30009EC2072038B504466846FEF77FFF01066B
:106F40000A4801D5006838BD9DF80010032909D012
:106F500087210160064900200860784605490860DD
:106F6000872038BD204602F0FFF938BD0800001028
:106F70000C0000101000001038B504466846FEF7FB
:106F80005DFF01060A4801D5006838BD9DF8001074
:106F9000032909D08721016006490020086078464E
:106FA00005490860872038BD204602F091FA38BDB7
:106FB000080000100C0000101000001038B5044646
:106FC0006846FEF73BFF01060A4801D5006838BD58
:106FD0009DF80010032909D087210160064900208F
:106FE0000860784605490860872038BD204602F0D1
:106FF0004DFB38BD080000100C0000101000001000
:1070000038B504466846FEF719FF01060A4801D55F
:10701000006838BD9DF80010032909D08721016060
:10702000064900200860784605490860872038BD79
:10703000204602F0DFFB38BD080000100C000010F5
:107040001000001038B504466846FEF7F7FE01064A
:107050000A4801D5006838BD9DF80010032909D001
:1070600087210160064900200860784605490860CC
:10707000872038BD204602F099FC38BD080000107A
:107080000C0000101000001038B504466846FEF7EA
:10709000D5FE01060A4801D5006838BD9DF80010EC
:1070A000032909D08721016006490020086078463D
:1070B00005490860872038BD204602F00BFD38BD29
:1070C000080000100C0000101000001038B5044635
:1070D0006846FEF7B3FE01060A4801D5006838BDD0
:1070E0009DF80010032909D087210160064900207E
:1070F0000860784605490860872038BD204602F0C0
:10710000A1FD38BD080000100C0000101000001098
:1071100038B504466846FEF791FE01060A4801D5D7
:10712000006838BD9DF80010032909D0872101604F
:10713000064900200860784605490860872038BD68
:10714000204602F013FE38BD080000100C000010AD
:107150001000001038B56846FEF770FE0E4C0006B1
:1071600011D49DF80000032809D087200B49206026
:107170000020086078460A490860872038BD02F080
:10718000ADFE000601D5206838BD04208DF8000052
:107190006846FEF749FE38BD080000100C000010DC
:1071A000100000102DE9FE43294C0026206882289B
:1071B00000D001266846FEF741FE00063AD49DF84D
:1071C00000001D280DD101A800F04AF8000631D4B6
:1071D0002048018821F00201018000F0BDFE000678
:1071E00028D49DF8000000251B4FDFF8708003288D
:1071F0000DD004280BD00E2809D01B2807D08720DB
:10720000206079463D60C8F80010BDE8FE8300208C
:1072100002F0A6FE00060DD49DF800001B280BD03E
:107220006846FEF71CFE000604D46846FEF7FCFD27
:10723000000601D52068E8E716B101200BF00EFB2F
:10724000256079463D600020C8F80010DDE70000A9
:1072500008000010020000100C00001010000010C8
:107260002DE9F04796B0824613A8FEF7E7FD504C93
:10727000000654D49DF84C10002505264D4FDFF82C
:1072800038810DF13C0904290AD01D2948D08720F6
:10729000206079463D60C8F8001016B0BDE8F08760
:1072A00014A9504602F09FFF20B192282AD09328BB
:1072B00075D123E09DF85000002873D03F48007836
:1072C00000286FD01D208DF84C0013A8FEF7ACFDF0
:1072D000000664D44846FFF775F800065FD412A88C
:1072E000FFF781F800065AD40AF0E1FF60B3256089
:1072F00079463D600020C8F80010CEE7F8F7A6FFF9
:107300000E2005E03868312849D1F8F79FFF162094
:107310008DF84C0013A8FEF787FDF8F7ACFF3EE0B0
:107320000DA806F0F4FC000639D412A90F9806F057
:1073300045FF000633D44846FFF73AF800062ED43E
:1073400012A8FFF746F8CDE70C208DF801000F9842
:10735000CDF802001298CDF80600684607F020FF2D
:1073600000061CD4684609F081F8000617D4FEF721
:1073700072FC18B1FEF743FB000610D4684607F014
:107380003AFF00060BD4684609F09BF8000606D4C5
:10739000FEF761FC28B1FEF73EFB000602D520682F
:1073A0007BE7FFE78DF84C6013A8FEF73DFD74E71F
:1073B000080000100C000010100000108AC103002B
:1073C00070B586B005460E4603A8FEF737FD2D4C76
:1073D00000064ED49DF80C001D280DD104A8FFF71F
:1073E0003FFF000645D42848018821F002010180B2
:1073F00000F0B2FD00063CD49DF80C1001292DD000
:107400000020022909D087212160204908607846A0
:107410001F490860872006B070BD2988ADF80410A8
:107420006988ADF8061029798DF808108DF80900E3
:1074300001A804F0C1F800061BD469462B2014F003
:1074400029F8000615D413489DF800100078C907E4
:1074500004D0012802D001208DF80C0003A8FEF70B
:10746000F4FC000605D43146284603F03DFB000637
:1074700001D52068CFE706208DF80C0003A8FEF7A1
:10748000D3FCC8E708000010020000100C00001038
:10749000100000109EC2072038B56846FEF7CEFCEB
:1074A0000F4C000616D49DF80000062809D087204E
:1074B0000C4920600020086078460B49086087204E
:1074C00038BD03F093FB000604D46846FEF7C7FC02
:1074D000000601D5206838BD6846FEF7A5FC38BD1A
:1074E000080000100C0000101000001038B5054610
:1074F0006846FEF7A3FC0F4C000612D49DF800006E
:10750000062809D087200C492060002008607846B2
:107510000A490860872038BD284603F09FFB000613
:1075200001D5206838BD07208DF800006846FEF7B9
:107530007BFC38BD080000100C000010100000108B
:1075400038B504466846FEF779FC01060B4801D5BC
:10755000006838BD9DF8001004290BD0062909D019
:1075600087210160064900200860784605490860C7
:10757000872038BD204603F0B3FC38BD080000105A
:107580000C0000101000001038B504466846FEF7E5
:1075900055FC01060B4801D5006838BD9DF8001068
:1075A00004290BD0062909D0872101600649002053
:1075B0000860784605490860872038BD204603F0FA
:1075C00051FD38BD080000100C0000101000001024
:1075D00038B504466846FEF731FC01060B4801D574
:1075E000006838BD9DF8001004290BD0062909D089
:1075F0008721016006490020086078460549086037
:10760000872038BD204603F0DFFD38BD080000109C
:107610000C0000101000001038B505466846FEF753
:107620000DFC124C000617D49DF80000022809D06A
:1076300087200F4920600020086078460D490860C7
:10764000872038BD002005F09BF8000604D42846AA
:1076500003F0B2FF000601D5206838BD01208DF887
:1076600000006846FEF7E0FB38BD0000080000108F
:107670000C0000101000001038B505466846FEF7F3
:10768000DDFB1F4C000632D49DF8000010281FD0EF
:107690000CDC0C281CD004DC012819D002280DD1E8
:1076A00016E00D2814D00E2808D111E013280FD0B1
:1076B00014280DD015280BD0182809D0872011497F
:1076C00020600020086078460F490860872038BD98
:1076D0006846FEF7BAFB000609D46846FEF7C6FB0B
:1076E000000604D4284609F0A1F8000601D5206858
:1076F00038BD08208DF800006846FEF795FB38BDC0
:10770000080000100C000010100000102DE9F041DE
:1077100086B002A8FEF792FB504C00067ED49DF87E
:10772000080001274E4E0025082807D0092805D05B
:107730000A2874D0872006B0BDE8F08109F020F94E
:10774000009031684FF00A080191042821D005DC2F
:1077500048B1012809D0032829D118E0052802D012
:10776000822824D11FE0009560E06846FFF7E6F824
:10777000000670D401A8FFF7F0F800066BD48DF86E
:10778000088002A8FEF750FB000664D44EE00820F3
:1077900000E009208DF8080002A8FEF745FB0090E4
:1077A0003068019042E003290DD004290BD00AF083
:1077B00099FC03A8FFF77EF800064CD49DF80C0056
:1077C0000E2803D011E006F009F92FE004A9622089
:1077D00013F060FE00063ED49DF81000C00704D0F0
:1077E0000120F9F77BFB000635D40098822801D0F0
:1077F000922801D106F0F2F86846FFF79FF80006DC
:1078000029D401A8FFF7A9F8000624D49DF80800A0
:1078100009280BD08DF8088002A801E01BE00DE0DC
:10782000FEF702FB15E000BFCDE90075009820606F
:107830000199316079460B4A11607CE78120CDE9DE
:1078400000056846FFF77AF8000604D401A8FFF7A0
:1078500084F80006E8D520686DE7000008000010F5
:107860000C000010100000102DE9F04186B003A8B4
:10787000FFF720F8364C000660D402A8FEF7DEFAC7
:1078800000065BD401A8FFF762F8000656D404A8EE
:10789000FFF76DF8000651D49DF8080087272D4D9D
:1078A0002D4E4FF000080A2801D0092835D109F0E3
:1078B000E1FF000642D401980128684608D0FEF78F
:1078C000CEFA00063AD49DF80800092805D013E046
:1078D000FEF7D6FA000631D414E00198922801D0C0
:1078E000822802D113208DF800009DF80C00142886
:1078F00002D10C208DF800000198932802D10E20AF
:107900008DF800006846FEF78FFA000616D49DF841
:107910000800092814D00A2808D027607846C5F83E
:1079200000803060872006B0BDE8F0819DF80C0033
:107930000E2805D1FAF78EFD000601D52068F2E782
:10794000019820600499296079463160EBE70000D6
:10795000080000100C0000101000001038B505469B
:107960006846FEF76BFA164C00061FD49DF800001F
:107970000C2809D087201349206000200860784631
:1079800011490860872038BD6846FEF75EFA000698
:107990000CD40D208DF800006846FEF767FA00064B
:1079A00004D4284603F0CEFE000601D5206838BD79
:1079B00008208DF800006846FEF736FA38BD000052
:1079C000080000100C00001010000010F0B585B089
:1079D00001A808F000F8344C000655D46846FEF7BC
:1079E0002DFA000650D49DF8000002252F4E304F8E
:1079F00013281ED00CDC0D281BD004DC012818D065
:107A000002280DD115E00E2813D0102808D143E02C
:107A100014280ED015280CD018280AD01B283BD0CB
:107A2000872020600020306078463860872005B0CD
:107A3000F0BD012004F0A4FE000625D404A804F043
:107A400027FB000622D59DF81000E8B1012809D0D7
:107A5000022810D0882020600920306078463860E5
:107A60008820E4E7F8F7F2FB18208DF8000006E024
:107A7000F8F701FC08E0F8F7E9FB8DF800506846DC
:107A8000FEF7D2F90006F3D52068D0E78DF8005054
:107A90006846FEF7C9F9CAE792202060784635604B
:107AA00038609220C3E70000080000100C000010AE
:107AB000100000102DE9F04786B0824602A807F0BA
:107AC0008AFF374C00065AD43648374D374E007877
:107AD000022788B105A805F021FF00064FD49DF8C4
:107AE0001500AC2808D09220206078462F603060C6
:107AF000922006B0BDE8F0870620F9F7C4FD38B93A
:107B00000420F9F7C0FD18B90120F9F7BCFD88B1D0
:107B10006846FEF793F9000631D49DF800004FF057
:107B200000084FF0870902280CD00D2815D018281E
:107B300027D112E091202060B12028607846306083
:107B40009120D6E701A8FFF707F9000617D41849D6
:107B50009DF804000978084213D101A9504604F0A9
:107B600029F8B0B19DF8040048B1F8F76FFB182070
:107B70008DF800006846FEF757F9F8F77CFB20689F
:107B8000B7E7C4F800907846C5F8008030608720D9
:107B9000AFE78DF800706846FEF746F9A9E70000E8
:107BA0000800001002C007200C0000101000001098
:107BB0008AC10300F8B506466846FEF73FF9504C07
:107BC000000650D49DF800004E4D132812D004DC5E
:107BD00001280FD00E2804D10CE015280AD01B284C
:107BE00008D0872020600020286078464649086039
:107BF0008720F8BDFAF71BF893281ED06846FEF7D9
:107C000024F900062FD49DF800001B2819D002206B
:107C10008DF800006846FEF729F9000623D40120FC
:107C200004F0AEFD00061ED4304609F081FE50B1CE
:107C30008F280FD0922816D117E0F8F707FB0E20F7
:107C400019E01020E4E708208DF800006846FEF7F0
:107C5000EBF8F8BDF8F7FAFA2868072801D11420E4
:107C600009E0F8F708FB2068F8BDF8F7EFFA286894
:107C70003128F6D116208DF800006846FEF7D4F8BA
:107C8000EFE72DE9FC4101A8F9F7A1F81C4C00062B
:107C90000BD4BDF804001B4E1B4F002540B16946B4
:107CA000622013F0F7FB000609D52068BDE8FC81CF
:107CB000812020607846356038608120F6E79DF8A5
:107CC0000000800703D5002110A026F013FEF9F76D
:107CD00083F830B1F8F7BAFA0AF004FAF8F7CBFAF9
:107CE000E3E70F48018841F00201018001200AF01A
:107CF000B5FD25607846356038600020D6E7000085
:107D0000080000100C000010100000108493818BFC
:107D1000888A809220848E8A938C858D92800A0036
:107D200002000010F8B506460D466846FEF786F8D4
:107D30001C4C00062DD49DF80020132A19D008DC15
:107D4000012A16D0022A14D00E2A12D0102A06D1E7
:107D50000FE0142A0DD0152A0BD0182A09D087203D
:107D6000114920600020086078461049086087208B
:107D7000F8BD6846FEF769F800060AD46846FEF7C3
:107D800075F8000605D42946304609F09BFF000629
:107D900001D52068F8BD08208DF800006846FEF780
:107DA00043F8F8BD080000100C000010100000108F
:107DB000F8B506460D466846FEF740F81D4C00062D
:107DC00027D49DF800101C4A1C48102911D004DC4F
:107DD00002290ED00D2904D10BE0112922D014293B
:107DE00007D087212160002111607946016087203A
:107DF000F8BD6846FEF729F800060AD46846FEF783
:107E000035F8000605D4294630460AF017F8000672
:107E100001D52068F8BD08208DF800006846FEF7FF
:107E200003F8F8BD91212160A92111607946016014
:107E30009120F8BD080000100C0000101000001088
:107E40003EB501A8FDF7E9FF214C00063ED4684687
:107E5000FDF7F4FF000639D402A901201DF00AFE47
:107E6000000633D49DF800001A4D022806D00E28D3
:107E700004D0102802D00298C00705D004F0B2FA4E
:107E800080B1922822D114E09DF804208721124865
:107E900021600AB1042100E00021296079460160D7
:107EA00087203EBD10208DF800006846FDF7BCFF1E
:107EB0003EBD2868312809D1F8F7C8F916208DF899
:107EC00000006846FDF7B0FFF8F7D5F920683EBD21
:107ED000080000100C0000101000001038B5054616
:107EE0006846FDF7ABFF184C00061DD49DF8000056
:107EF000112809D0872015492060002008607846A5
:107F000013490860872038BD1248296801606968F4
:107F10004160A9688160342013F051F9000603D450
:107F200026F08EFE000601D5206838BD284608F0F0
:107F300081F810B10AF0D6F8F6E702208DF80000BB
:107F40006846FDF771FF38BD080000100C000010F6
:107F50001000001090CA07202DE9FC416846FDF78B
:107F60006DFF194C000622D49DF800000025174E25
:107F7000174F052809D01D2820D08720206078467B
:107F8000356038608720BDE8FC8101A90120FEF73B
:107F900026F800060BD404F0E7FA000607D4012007
:107FA0008DF800006846FDF73FFF000601D5206808
:107FB000E9E7019800B101200AF054F925607846FC
:107FC000356038600020DEE7080000100C0000106B
:107FD0001000001038B56846FDF730FF0E4C000663
:107FE00011D49DF80000072809D087200B49206094
:107FF0000020086078460A490860872038BD04F0F0
:10800000DBFA000601D5206838BD01208DF800009C
:108010006846FDF709FF38BD080000100C0000108D
:108020001000001038B504466846FDF707FF01064A
:108030000A4801D5006838BD9DF80010032909D011
:1080400087210160064900200860784605490860DC
:10805000872038BD204604F035FC38BD08000010EC
:108060000C0000101000001038B504466846FDF7FB
:10807000E5FE01060A4801D5006838BD9DF80010EC
:10808000032909D08721016006490020086078464D
:1080900005490860872038BD204604F08BFC38BDB8
:1080A000080000100C0000101000001038B5044645
:1080B0006846FDF7C3FE01060A4801D5006838BDD1
:1080C0009DF80010032909D087210160064900208E
:1080D0000860784605490860872038BD204604F0CE
:1080E000E1FC38BD080000100C000010100000106A
:1080F00038B504466846FDF7A1FE0106204801D5C3
:10810000006838BD9DF8001001290BD0022909D064
:10811000872101601B490020086078461A490860E1
:10812000872038BD204604F03BFE38BD38B50446F4
:108130006846FDF783FE0106114801D5006838BD89
:108140009DF8001001290FD0032910D004290ED06A
:1081500005290CD0872101600A4900200860784673
:1081600009490860872038BD0121204605E00AF052
:1081700013F826F065FD0021084604F08BFE38BD9B
:10818000080000100C000010100000102DE9F8434A
:108190008046694601201DF06DFC104C00060DD490
:1081A00000980F4E0F4FC0074FF0000509D0002276
:1081B0000121404604F0FAFE000609D52068BDE81A
:1081C000F883872020607846356038608720F6E79E
:1081D00025607846356038600020F0E70800001020
:1081E0000C0000101000001038B504464FF000409D
:1081F000FDF7B8FB000602D51648006838BD2046DA
:10820000FDF79DFE00061FD4A01CFDF7A9FE000689
:108210001AD4201DFDF7B5FE000615D40AF0DAFBCE
:10822000000602D509F05EFF0EE06846FDF75EFE2F
:10823000000609D46846FDF73DFA000604D46846F6
:10824000FDF74AFE000602D5FDF787FC38BDFDF7B5
:10825000EFFB38BD080000102DE9F04188B001A8FF
:10826000FDF7DBFD384C00065ED49DF80400374F67
:10827000374E48B1912020609C20306078463860AD
:10828000912008B0BDE8F08106A901201DF0F2FBA5
:10829000000649D406984FF00005C00746D068464E
:1082A000FDF7CCFD00063FD46846FDF7CEFD000685
:1082B0003AD46846FDF7DAFD000635D408208DF87B
:1082C00000006846FDF7B0FD00062DD44FF0010810
:1082D0008DF8088002A8FEF7E3FA000624D40320F4
:1082E0008DF80C0003A8FDF7E6FD00061CD4194923
:1082F0000220087014482560FEF720FB000613D406
:1083000013483560FEF729FB00060DD4ADF8108048
:1083100004A8FEF7ECFA000606D4ADF8145005A840
:10832000FEF7F6FA000608D52068AAE78720206045
:108330007846356038608720A3E725607846356049
:10834000386000209DE700000800001010000010B9
:108350000C000010000000102DE9FF47064668469B
:1083600004F0D7F9A24C000665D4BDF800004FF424
:10837000B46148433178C1EB011100EB81007178A1
:10838000451802A8FEF7E8FC000654D403A8FAF743
:108390006BF900064FD49DF80C00E8B395499DF8A1
:1083A0000800DFF854920978DFF850A208424FF035
:1083B00086074FF0170817D06946022005F03FFDE9
:1083C000000638D401A9032005F039FD000632D497
:1083D000BDF80000BDF80410C0EB001000EB400039
:1083E00001EB4010854215D36846FEF705FA0006FA
:1083F00021D401A8FEF710FA00061CD4BDF8000035
:10840000BDF80410C0EB001000EB400001EB401081
:1084100085420BD2276000E008E07946C9F8008069
:108420008620CAF8001004B0BDE8F08730461EF080
:10843000BBF8000601D52068F5E704F019FAF2E769
:108440002DE9FF4781466946532013F023F8684C15
:10845000000629D49DF8000000F004008DF800000B
:1084600001A8FDF7EBFC00061ED49DF80400624D48
:10847000624E0027DFF88881102817D009DC022817
:1084800014D00D2819D091210E287DD00F2806D1A7
:108490009AE011280AD0192815D01A2813D003A859
:1084A000FAF7E2F8000670D52068BCE74846FFF707
:1084B00053FF05E088F800700FE048461EF074F89E
:1084C0000006F1D4F6E74846FFF746FF0028EBD157
:1084D00098F80000C246022805D0276078462F6031
:1084E000306000209FE79DF8000020B14D2012F081
:1084F00066FE0006D8D448461DF0F1FF0006D3D42E
:10850000404999F8028088683F4A8B681B1A934259
:10851000FBD348461DF0E3FF0006C5D499F80210CE
:10852000414507D1822020600520286078463060D0
:10853000822078E703218AF8001034494FF00108BF
:1085400001A881F80080FDF79BFC0006ACD401A8CF
:10855000FDF76AFC0006A7D40420F9F725F9000608
:10856000A2D49DF8000020B101200AF077F900069E
:108570009AD402A9532012F08DFF000694D49DF8DE
:10858000080010F0010001E01BE024E08DF8080075
:1085900008D001200AF062F9000685D409F0F8FC41
:1085A000000681D49DF8080020B101200AF056F998
:1085B000000686D4C4F8008078462F603060012021
:1085C00031E7A020216001E0D220216028607846B8
:1085D0003060912027E79DF80C108720206011B1B2
:1085E0000420286000E02F607846306087201AE77A
:1085F000080000108AC103000C00001010000010D9
:108600004AC1072000800040E0C81000A40000100C
:108610002DE9FE43054601A8FEF79EFBAB4C000684
:108620002BD49DF80400AA4EAA4F4FF086084FF0B5
:108630001A09A8B1A848007848B16946022005F097
:10864000FEFB000619D4BDF8000085421CD3684625
:10865000F9F700FA000610D4BDF80000854213D3E4
:1086600002A8FAF701F8000607D49DF8080098B1AF
:108670006846FEF7C1F8000602D52068BDE8FE8313
:10868000BDF80000854207D2C4F800807846C6F8DD
:10869000009038608620F1E7002020603060784646
:1086A00038600020EAE72DE9F14F88B000278DF807
:1086B000047003A90898F8F7E1F9BDF80C0048F236
:1086C0006901834D834E814C401E4FF086094FF067
:1086D000140A884205D300BFC4F80090C5F800A072
:1086E0005EE001A9532012F0D5FE00067ED49DF86D
:1086F000040000F004008DF804006846FDF79EFBBE
:108700000006F3D49DF80000102820D009DC0228D0
:108710001DD00D281BD091210E2868D00F2808D11C
:1087200098E0112813D0192811D01A280FD01C282E
:108730000DD006A8F9F798FF000657D49DF8181039
:108740008720002920607CD0042028608AE0BDF8C2
:108750000C00FFF75DFFDFF8848138B3862845D130
:1087600088F800709DF800001C2810D01A283DD011
:1087700019283BD06846FDF768FB000636D41C205C
:108780008DF800006846FDF74FFB00062ED402204E
:10879000F8F7F7FF000629D41A20C4F800902860E3
:1087A00078463060862009B0BDE8F08F02A81DF041
:1087B000C7FE00064FF0010B07D54FF4FA60ADF885
:1087C00008008DF80AB08DF80BB005A902A8F8F7DB
:1087D00055F9BDF80C10BDF8140098F8002081423E
:1087E000404610D9012A08D0418001E05EE02EE029
:1087F00088F800B0C4F800B062E042888A4204D031
:1088000088F8007068E7012AF7D008981DF0EDFE9F
:1088100000064BD44FF0020988F800909DF8040040
:1088200048B13A2012F0CBFC00063FD401200AF0F8
:1088300015F800063AD40220F8F7B6FF000635D442
:1088400000E00EE09DF800001C280FD018E0A020EA
:10885000216001E0D22021602860784630609120BC
:10886000A1E72F607846306087209CE76846FDF7D7
:10887000F6FA00061AD46846FDF7D6FA000615D4B3
:1088800003F0F6FF9DF80000192807D01A2805D03C
:10889000276078462F603060002084E79DF8040050
:1088A00050B13E2012F08BFC000601D520687AE71B
:1088B00000210BA026F01EF888F80090C4F800B044
:1088C00078462F60306001206DE70000080000103E
:1088D0000C000010100000108AC103004AC10720DC
:1088E000200A200A200A200A200A200A200A200A38
:1088F000000000002DE9FF4782469046894601A806
:1089000007F069F8F94C00062FD46846FDF796FA8F
:1089100000062AD49DF800000026F54FF54D1328D7
:108920001ED00CDC0D281BD004DC012818D0022836
:108930000DD115E00E2813D0102808D128E01428F6
:108940000ED015280CD018280AD01B2820D087203C
:10895000206078463E602860872004B0BDE8F0873C
:10896000012003F00DFF000601D52068F5E742461F
:108970004946504604F016FD000603D579462068A6
:108980002960EAE7266078463E6028600020E4E738
:108990009220206002203860784628609220DCE730
:1089A0002DE9FF4782469046894601A807F013F853
:1089B000CE4C00062DD46846FDF740FA000628D4B8
:1089C0009DF800000026CA4FCA4D13281CD00CDCAD
:1089D0000D2819D004DC012816D002280DD113E08F
:1089E0000E2811D0102808D126E014280CD0152804
:1089F0000AD0182808D01B281ED08720206078466F
:108A00003E6028608720A8E7012003F0B9FE000639
:108A100001D52068A1E742464946504604F07AFD58
:108A2000000603D579462068296096E726607846D7
:108A30003E602860002090E792202060022038608D
:108A400078462860922088E72DE9FF41074601A873
:108A500006F0C1FFA54C000630D46846FDF7EEF9DC
:108A600000062BD49DF80000A149A24D0226132830
:108A70001FD00CDC0D281CD004DC012819D00228E2
:108A80000DD116E00E2814D0102808D127E01428A4
:108A90000FD015280DD018280BD01B281FD08720E9
:108AA00020600020086078462860872004B0BDE878
:108AB000F081012003F064FE000601D52068F5E78F
:108AC000384604F091FD000603D5794620682960F8
:108AD000ECE78DF800606846FDF7A6F9E6E792201E
:108AE000206078460E6028609220DFE72DE9FF477E
:108AF0008146884601A806F06EFF7C4C00062DD406
:108B00006846FDF79BF9000628D49DF80000002672
:108B1000774F784D13281CD00CDC0D2819D004DCBD
:108B2000012816D002280DD113E00E2811D01028EC
:108B300008D125E014280CD015280AD0182808D010
:108B40001B281DD08720206078463E602860872043
:108B500003E7012003F014FE000601D52068FCE6BF
:108B60004146484604F0DAFD000603D57946206800
:108B70002960F2E6266078463E6028600020ECE638
:108B80009220206002203860784628609220E4E637
:108B90002DE9FF478146884601A806F01CFF534C8B
:108BA00000062DD46846FDF749F9000628D49DF843
:108BB000000000264E4F4F4D13281CD00CDC0D2812
:108BC00019D004DC012816D002280DD113E00E289C
:108BD00011D0102808D125E014280CD015280AD06F
:108BE000182808D01B281DD08720206078463E60BA
:108BF00028608720B1E6012003F0C2FD000601D500
:108C00002068AAE64146484604F0F1FD000603D577
:108C1000794620682960A0E6266078463E60286094
:108C200000209AE692202060022038607846286072
:108C3000922092E610B504F0F7FD02062B482C4B6B
:108C40002C4903D500687A460A6010BD00220260F4
:108C500078461A600860104610BD2DE9FF41804635
:108C600001A806F0B8FE214C00062DD46846FDF799
:108C7000E5F8000628D49DF8000000261C4F1D4D85
:108C800013281CD00CDC0D2819D004DC012816D0C8
:108C900002280DD113E00E2811D0102808D12BE0A6
:108CA00014280CD015280AD0182808D01B2823D047
:108CB0008720206078463E6028608720F6E6012005
:108CC00003F05EFD000601D52068EFE6404604F0A3
:108CD000C8FD000603D5794620682960E6E62660CF
:108CE00078463E6028600020E0E6000008000010A2
:108CF0000C0000101000001092202060022038604C
:108D0000784628609220D1E6F0B5054641799E4C20
:108D10009E4F9F4E8DB0862009B1042902D9206054
:108D2000062005E0297909B11E2907D92060052010
:108D300038607846306086200DB0F0BD698828889C
:108D400003F07EFC00067DD468796946FDF79CFB44
:108D5000000677D4BDF800100020A1F57F42FF3A4D
:108D600071D0064600906846FDF7D7F9000669D431
:108D70006846FDF703FE000664D4012769463846BD
:108D8000FDF7FEF900065DD47F1CFFB2112FF5D36D
:108D90006846FDF71FFA00067ED46846FDF72BFAF9
:108DA000000679D4012769463846FDF70CF900061C
:108DB00072D47F1CFFB20B2FF5D3012769463846CA
:108DC000FDF779FE000667D47F1CFFB2112FF5D3A3
:108DD0006846FDF7BCFB00065ED46846FDF7DCFB89
:108DE000000659D46846FDF702F9000654D46846D7
:108DF000FDF71FF900064FD46846FDF7D3F80006CB
:108E00004AD40127009669463846FDF700FE000661
:108E100042D47F1CFFB2052FF5D9ADF8006068463B
:108E2000FDF78CF9000637D46846FDF798F900067F
:108E300032D46846FDF7ECF800062DD46846FDF7FD
:108E400009F901E028E029E0000625D40096012672
:108E500069463046FDF7A8F900061DD4761CF6B227
:108E6000112EF5D32846FDF76AF8000614D4A81C85
:108E7000FDF776F800060FD4281DFDF782F80006EE
:108E80000AD4012009F0EAFC000605D44FF00040A6
:108E9000FCF768FD000608D520684DE78B212160AE
:108EA000386078463060084646E701248DF8004077
:108EB0006846FDF700F8000633D436480470681D94
:108EC000FDF71AF900062CD46846FDF70FF80006E6
:108ED00027D46846FCF7EEFB000622D46846FCF770
:108EE000FBFF00061DD46846FDF711F8000618D4F4
:108EF0006846FCF7B8FB000613D46846FCF7FDFF94
:108F000000060ED46846FDF713F8000609D468463B
:108F1000FCF7D0FB000604D46846FCF7FFFF000610
:108F200002D5FCF71AFE07E709F07CF9000624D405
:108F30008DF8014068798DF8020007F0EFF900061E
:108F40001BD4684606F02CF9000616D4684607F0D4
:108F50008DFA000611D4FCF752FD00060DD46846C8
:108F600006F049F9000608D4684607F0AAFA000698
:108F700003D4FCF750FD000602D509F0B3F8D0E7A2
:108F8000FCF756FDD8E60000080000100C000010A9
:108F9000100000100000001070B5057A724E94B0F9
:108FA0000446102D0AD986207049306003200860DD
:108FB00078466F490860862014B070BD0DB9012550
:108FC000257260680E9021460EA8FCF7DCFA0006B8
:108FD00005D44FF00040FCF7C5FC000601D5306811
:108FE000EAE76846FDF7A3F8000652D40EA96846E2
:108FF000FCF753F900064CD46846FDF78EF80006DE
:1090000047D46846FDF7A4F8000642D4BDF8000036
:10901000401CADF800006846FDF790F8000638D413
:1090200069462846FDF7B8F8000632D40EA968460E
:10903000FCF733F900062CD469462846FDF7A0F862
:10904000000626D469462846FDF7BBF8000620D462
:1090500021466846FCF75BF900061AD469462846A3
:10906000FDF7A2F8000614D404F10800FDF7D4F8C7
:1090700000060ED42046FDF7E0F8000609D4201DB6
:10908000FDF7ECF8000604D40EA8FDF7F8F800068A
:1090900002D5FCF762FD8FE7012025F0BDF900063F
:1090A00058D409F014FB000654D40D208DF80500A7
:1090B000207A8DF813006068CDF807002068CDF89D
:1090C0000B000E98CDF80F002A4905A831F0BAF828
:1090D0000DF10600FDF71AF800063BD401A806F0D2
:1090E0005FF8000636D401A807F0C0F9000631D4B5
:1090F000012006F072FD00062CD46846FDF72CFE18
:10910000000627D49DF8000090B11B48007878B184
:1091100010A8FCF7FBFF00061CD48DF84C5020680B
:1091200011900E98129010A805F042FA000611D482
:10913000FCF765FC00060DD401A806F05CF80006FB
:1091400008D401A807F0BDF9000603D4FCF763FCBE
:10915000000602D508F0C6FF9BE70649002008700C
:10916000FCF766FC28E70000080000100C00001067
:1091700010000010CECA07208AC1030070B5057A1E
:10918000744E94B00446102D0AD98620724930607E
:1091900003200860784671490860862014B070BDCD
:1091A00005B9012560680E9021460EA8FCF7EBF981
:1091B000000605D44FF00040FCF7D4FB000601D5B3
:1091C0003068EBE76846FCF7B2FF000662D40EA9F0
:1091D0006846FCF783F800065CD46846FCF79DFF00
:1091E000000657D46846FCF7C4FF000652D4BDF809
:1091F0000000401CADF800006846FCF7B0FF000618
:1092000048D46846FDF7C4FB000643D40EA968465F
:10921000FCF743F800063DD46846FDF7AFFB0006B7
:1092200038D469462846FCF7B7FF000632D40EA9A9
:109230006846FCF753F800062CD469462846FCF72C
:109240009FFF000626D469462846FCF7BAFF0006B1
:1092500020D421466846FCF77BF800061AD46946FC
:109260002846FCF7A1FF000614D404F10800FCF71F
:10927000D3FF00060ED42046FCF7DFFF000609D41A
:10928000201DFCF7EBFF000604D40EA8FCF7F7FF47
:10929000000602D5FCF761FC80E709F0F8F900064A
:1092A0004FD40E208DF80500207A8DF813006068E9
:1092B000CDF807002068CDF80B000E98CDF80F0010
:1092C000274905A830F0BEFF0DF10600FCF71EFF90
:1092D000000636D401A805F063FF000631D401A8CA
:1092E00007F0C4F800062CD46846FDF735FD0006EB
:1092F00027D49DF8000090B11A48007878B110A8E2
:10930000FCF704FF00061CD48DF84C502068119027
:109310000E98129010A805F09BF9000611D4FCF7E6
:109320006EFB00060DD401A805F065FF000608D409
:1093300001A807F0C6F8000603D4FCF76CFB000692
:1093400002D508F0CFFEA5E7054900200870FCF71C
:109350006FFB23E7080000100C0000101000001045
:10936000CECA07208AC1030030B504460079544DA7
:109370008FB008B110280AD98620524928600320EE
:10938000086078465049086086200FB030BD4FF025
:109390000040FCF7E7FA000601D52868F5E76846C3
:1093A000FCF7C5FE000636D421466846FBF796FF5B
:1093B000000630D46846FCF7B0FE00062BD42079B6
:1093C0006946FCF7E9FE000625D421466846FBF70E
:1093D00085FF00061FD420796946FCF7D1FE000600
:1093E00019D4201DFCF78FFF000614D42046FCF78B
:1093F00079FF00060FD46846FDF7B2F800060AD4DC
:1094000021466846FBF749FF000604D46846FDF78D
:109410009EF8000602D5FCF7A0FBB6E709F017F9A5
:10942000000647D408208DF805000025CDF8065029
:109430000DF10B00FCF73EFF00063BD46846FCF73D
:109440004AFF000636D4BDF80000ADF80C008DF8D8
:109450000A502068CDF80E0001A805F0A1FE000614
:1094600028D401A807F002F8000623D46846FDF7C7
:1094700073FC00061ED49DF8000048B11348007824
:1094800030B120680E900EA805F035F9000611D411
:10949000FCF7B5FA00060DD401A805F0ACFE0006F5
:1094A00008D401A807F00DF8000603D4FCF7B3FABE
:1094B000000602D508F016FEADE7FCF7B9FA64E73E
:1094C000080000100C000010100000108AC10300FA
:1094D00030B504460079694D91B008B110280AD919
:1094E000862067492860032008607846654908603F
:1094F000862011B030BD4FF00040FCF733FA000673
:1095000001D52868F5E70DA8FCF711FE000650D438
:1095100021460DA8FBF7C1FE00064AD40DA8FCF7B2
:10952000FCFD000645D420790DA9FCF735FE0006A8
:109530003FD421460DA8FBF7B0FE000639D42079B0
:109540000DA9FCF71DFE000633D40EA8FDF7D2FAD4
:1095500000062ED49DF8380088B10DA9FDF7B8FAA1
:10956000000626D421460DA8FBF7B8FE000620D43D
:109570000DA99DF83800FDF79EFA000619D40DA834
:10958000FCF7EEFF000614D421460DA8FBF7A6FE5B
:1095900000060ED40DA8FCF7DAFF000609D4201D42
:1095A000FCF7B1FE000604D42046FCF79BFE000643
:1095B00002D5FCF7D2FA9CE709F01FF8000656D452
:1095C00004208DF801000FA94C2011F063FF000664
:1095D0004DD49DF83C00800702D49DF8380020B996
:1095E000684605F0DDFD000641D49DF83C009DF87D
:1095F000381000F00100401E084204D1684606F011
:1096000035FF000633D40DA8FDF7A6FB00062ED4C7
:109610009DF8340048B11C48007830B120681090A3
:1096200010A805F092F8000621D4FCF7E8F900062E
:109630001DD49DF83C00800702D49DF8380020B965
:10964000684605F0D8FD000611D49DF83C009DF851
:10965000381000F00100401E084204D1684606F0B0
:1096600030FF000603D4FCF7D6F9000602D508F057
:1096700039FD9EE7FCF7DCF93BE70000080000102D
:109680000C000010100000108AC1030030B5044621
:109690000079544D8FB008B110280AD9862052495C
:1096A00028600320086078465049086086200FB083
:1096B00030BD4FF00040FCF755F9000601D5286891
:1096C000F5E76846FCF733FD000636D421466846C8
:1096D000FBF7E3FD000630D46846FCF71EFD0006EC
:1096E0002BD420796946FCF757FD000625D4214686
:1096F0006846FBF7D2FD00061FD420796946FCF7C7
:109700003FFD000619D4201DFCF7FDFD000614D412
:109710002046FCF7E7FD00060FD46846FCF746FF3D
:1097200000060AD421466846FBF7B7FD000604D4BC
:109730006846FCF731FF000602D5FCF70EFAB6E7E3
:1097400008F03BFF000647D407208DF805000025F0
:10975000CDF806500DF10B00FCF7ACFD00063BD434
:109760006846FCF7B8FD000636D4BDF80000ADF839
:109770000C008DF80A502068CDF80E0001A805F005
:109780000FFD000628D401A806F070FE000623D4C1
:109790006846FDF7E1FA00061ED49DF8000048B1C6
:1097A0001348007830B120680E900EA804F0FAFF3C
:1097B000000611D4FCF723F900060DD401A805F02A
:1097C0001AFD000608D401A806F07BFE000603D4AB
:1097D000FCF721F9000602D508F084FCADE7FCF7A0
:1097E00027F964E7080000100C00001010000010BA
:1097F0008AC1030070B504460079684E92B0032513
:1098000008B1102809D9862030606548056078467F
:1098100064490860862012B070BD4FF00040FCF72C
:10982000A1F8000601D53068F5E70DA8FCF77FFC2C
:10983000000650D421460DA8FBF750FD00064AD47F
:109840000DA8FCF76AFC000645D420790DA9FCF7A9
:10985000A3FC00063FD421460DA8FBF73FFD000600
:1098600039D420790DA9FCF78BFC000633D40EA85F
:10987000FDF740F900062ED49DF8380088B10DA9F7
:10988000FDF726F9000626D421460DA8FBF726FD94
:10989000000620D40DA99DF83800FDF70CF900064C
:1098A00019D40DA8FCF782FE000614D421460DA899
:1098B000FBF714FD00060ED40DA8FCF76DFE0006A4
:1098C00009D4201DFCF71FFD000604D42046FCF738
:1098D00009FD000602D5FCF740F99CE708F04DFEB3
:1098E000000655D48DF801500FA94C2011F0D2FD7F
:1098F00000064DD49DF83C00800702D49DF8380046
:1099000020B9684605F04CFC000641D49DF83C00A7
:109910009DF8381000F00100401E084204D168464E
:1099200006F0A4FD000633D40DA8FDF715FA0006D5
:109930002ED49DF8340048B11B48007830B120681F
:10994000109010A804F058FF000621D4FCF757F837
:1099500000061DD49DF83C00800702D49DF8380015
:1099600020B9684605F047FC000611D49DF83C007C
:109970009DF8381000F00100401E084204D16846EE
:1099800006F09FFD000603D4FCF745F8000602D55B
:1099900008F0A8FB9FE7FCF74BF83CE70800001035
:1099A0000C000010100000108AC1030010B504461E
:1099B00090B04FF00040FBF7D5FF000603D54348B9
:1099C000006810B010BD0EA8FCF7B1FB000626D44D
:1099D0000EA8FCF7DCFC000621D40E980D90214661
:1099E0000DA8FBF77BFC000619D40DA8FCF795FB2E
:1099F000000614D40DA8FCF7F7FB00060FD421468F
:109A00000DA8FBF74AFC000609D40DA8FCF7E2FB01
:109A1000000604D42046FCF7A9FC000602D5FCF79A
:109A20009CF8CEE708F089FD000648D408208DF8A0
:109A300001000E98CDF802000DF10700FCF77EFC46
:109A400000063CD40DA8FCF78AFC000637D4BDF80C
:109A50003400ADF8080000208DF806002068CDF82D
:109A60000A00684605F09CFB000628D4684606F00C
:109A7000FDFC000623D40DA8FDF76EF900061ED4E8
:109A80009DF8340048B11248007830B120680F903A
:109A90000FA804F030FE000611D4FBF7B0FF00065B
:109AA0000DD4684605F0A7FB000608D4684606F00A
:109AB00008FD000603D4FBF7AEFF000602D508F050
:109AC00011FBACE7FBF7B4FF7BE7000008000010D8
:109AD0008AC1030030B5044691B04FF00040FBF757
:109AE00041FF564D000619D40DA8FCF720FB0006D7
:109AF00031D40DA8FCF74BFC00062CD421460DA850
:109B0000FBF7CBFB000626D40DA8FCF706FB0006EE
:109B100021D40EA8FCF7EEFF000602D5286811B08C
:109B200030BD9DF83800C8B10DA9FCF7D1FF000683
:109B300011D421460DA8FBF7D1FB00060BD40DA9CB
:109B40009DF83800FCF7B7FF000604D42046FCF768
:109B50000DFC000611D5FCF700F8E0E70DA8FCF7B6
:109B600043FB0006F7D421460DA8FBF7B7FB000620
:109B7000F1D40DA8FCF72EFBE6E708F0BEFC0006CA
:109B800056D404208DF801000FA94C2011F082FC5E
:109B900000064DD49DF83C00800702D49DF83800A3
:109BA00020B9684605F0FCFA000641D49DF83C0057
:109BB0009DF8381000F00100401E084204D16846AC
:109BC00006F054FC000633D40DA8FDF7C5F80006D6
:109BD0002ED49DF8340048B11948007830B120687F
:109BE000109010A804F0B1FD000621D4FBF707FF88
:109BF00000061DD49DF83C00800702D49DF8380073
:109C000020B9684605F0F7FA000611D49DF83C002B
:109C10009DF8381000F00100401E084204D168464B
:109C200006F04FFC000603D4FBF7F5FE000602D554
:109C300008F058FA8FE7FBF7FBFE70E7080000100A
:109C40008AC1030030B5044691B04FF00040FBF7E5
:109C500089FE444D000656D40EA8FCF768FA0006AB
:109C600026D40EA8FCF793FB000621D40E980D9085
:109C700021460DA8FBF711FB000619D40DA8FCF72F
:109C80004CFA000614D40DA8FCF7BFFA00060FD456
:109C900021460DA8FBF701FB000609D40DA8FCF72F
:109CA000AAFA000604D42046FCF760FB000603D5A0
:109CB000FBF753FF11B030BD08F0BFFB00064AD4DC
:109CC0000DA8FDF749F8000645D49DF8340048B1C9
:109CD0002548007830B120680F900FA804F062FD8D
:109CE000000638D407208DF801000E98CDF8020048
:109CF0000DF10700FCF722FB000604D40DA8FCF7C9
:109D00002EFB000601D52868D4E7BDF83400ADF875
:109D1000080000208DF806002068CDF80A0068468B
:109D200005F03EFA000616D4684606F09FFB0006D2
:109D300011D4FBF764FE00060DD4684605F05BFA0B
:109D4000000608D4684606F0BCFB000603D4FBF707
:109D500062FE000602D508F0C5F9A9E7FBF768FE28
:109D6000A8E70000080000108AC1030010B50446EF
:109D700092B04FF00040FBF7F5FD000603D55548C3
:109D8000006812B010BD0DA8FCF7D1F900062ED462
:109D90000DA8FCF7FCFA000629D421460DA8FBF714
:109DA0009DFA000623D40DA8FCF7B7F900061ED4CF
:109DB0000EA8FCF79FFE000619D49DF83800C8B124
:109DC0000DA9FCF785FE000611D421460DA8FBF76E
:109DD00085FA00060BD40DA99DF83800FCF76BFE40
:109DE000000604D42046FCF7C1FA000611D5FBF7A3
:109DF000B4FEC6E70DA8FCF708FA0006F7D4214622
:109E00000DA8FBF76BFA0006F1D40DA8FCF7F3F9E7
:109E1000E6E708F0F2FA000656D403208DF80100B8
:109E20000FA94C2011F036FB00064DD49DF83C00E4
:109E3000800702D49DF8380020B9684605F0B0F9D3
:109E4000000641D49DF83C009DF8381000F0010058
:109E5000401E084204D1684606F008FB000633D4D1
:109E60000DA8FCF779FF00062ED49DF8340048B108
:109E70001948007830B12068109010A804F0BCFC9C
:109E8000000621D4FBF7BBFD00061DD49DF83C0065
:109E9000800702D49DF8380020B9684605F0ABF978
:109EA000000611D49DF83C009DF8381000F0010028
:109EB000401E084204D1684606F003FB000603D4A6
:109EC000FBF7A9FD000602D508F00CF98FE7FBF7B8
:109ED000AFFD56E7080000108AC1030000B58FB03F
:109EE0004FF00040FBF73EFD000603D51B4800681D
:109EF0000FB000BD08F061FA000626D410208DF8DE
:109F000001000DA8FCF713F900061ED40D98CDF83A
:109F10000200684605F044F9000616D4684606F0CB
:109F2000A5FA000611D4FBF76AFD00060DD46846B9
:109F300005F061F9000608D4684606F0C2FA00068A
:109F400003D4FBF768FD000604D508F0CBF8FBF757
:109F500004FECDE7FBF76CFDCAE700000800001027
:109F6000F0B5734D070091B0288802D040F0200072
:109F700001E040F0100028804FF00040FBF7F2FCB9
:109F80006C4E000671D40EA8FCF7C0F8000668D429
:109F900069469DF83800FCF777FA000661D4BDF8F1
:109FA00000006946401CADF800009DF83800FCF741
:109FB0005EFA000655D46846FBF798FF000650D4B9
:109FC0006846FBF789FB00064BD46846FBF784FF25
:109FD000000646D46846FBF79AFF000641D468465F
:109FE000FBF755FB00063CD46846FBF786FF0006EE
:109FF00037D46846FBF79CFF000632D46846FBF76F
:10A000006BFB00062DD46846FBF788FF000628D4BA
:10A01000002468460094FCF780F800067AD468466D
:10A02000FCF79AFE000602D508F05CF819E0022061
:10A0300024F0F2F9000614D438003F4F0DD09DF8FB
:10A04000000028B1387818B103F0C8FC000608D425
:10A0500008F07EF9000604D411E008F079F9000652
:10A0600004D5FBF77AFD11B0F0BD53E09DF8000078
:10A0700028B1387818B103F0B1FC0006D4D40FA988
:10A080006A2011F0D2FA000644D49DF83C0010F08A
:10A0900002008DF83C0002D0742011F090F88DF889
:10A0A00000406846FCF728F80006BDD48DF8004053
:10A0B0006846FBF700FF0006B6D46846FBF7CFFE04
:10A0C0000006B1D49DF80000022806D18DF80040AA
:10A0D0006846FBF798FE0006A6D402208DF805001E
:10A0E00006F01CF900069FD401A805F059F80006F7
:10A0F0009AD4FBF784FC000696D401A805F07BF8FF
:10A10000000691D4FBF787FC00068DD4FBF790FC8A
:10A11000000601D53068A6E7288820F0B000288026
:10A1200006483460046078460549086000209AE7D4
:10A1300002000010080000108AC103000C0000108B
:10A1400010000010FE49098801807047FC494988C9
:10A150000180704730B58FB005460B208DF80100A7
:10A160000DA8FBF7D4FEF74C000630D4BDF8340040
:10A17000ADF80A000DA8FBF7B9FE000627D40D982C
:10A18000CDF8060028798DF80C002888ADF802007B
:10A190006888ADF80400684605F002F8000616D499
:10A1A000684606F063F9000611D4FBF728FC0006A8
:10A1B0000DD4684605F01FF8000608D4684606F07E
:10A1C00080F9000603D4FBF726FC000602D52068C0
:10A1D0000FB030BDDC490020206008607846DB49C4
:10A1E00008600020F4E72DE9F34F9BB007461C9967
:10A1F000002011900870D2493888DFF84CB30880ED
:10A20000788848803879CF4D862408B11E2804D933
:10A2100005212C60CBF8001012E0388848F6AD61BB
:10A22000142688421DD878884FF01708B0F5B46F0F
:10A230000DD32C607846C549CBF80080086002E059
:10A240007946C248016086201DB0BDE8F08F05A8A0
:10A25000FBF77FFE00067CD43888BDF814108842D6
:10A2600003D22C60CBF80060EAE70DD105A8FBF71C
:10A2700081FE0006EFD47888BDF81410884203D21E
:10A280002C60CBF80080DBE702A8FBF795FE000608
:10A29000E1D405A8FBF74BFF0006DCD40599029832
:10A2A000814209D08C20286000207946CBF800003C
:10A2B000A64801608C20C7E7022005F08EFC00064E
:10A2C000C9D4012003F056FE0006C4D44FF000406C
:10A2D000FBF748FB0006BED46846FBF717FF0006F5
:10A2E0007DD405A8FBF723FF0006F9D4059898B1A3
:10A2F00002A99DF80000FCF79BF80006F0D405A920
:10A3000002A8FAF759FF0006EAD402A99DF8000056
:10A31000FCF781F80006E3D405A8FCF739FB00063A
:10A32000DED4059898B102A99DF80000FCF744FB23
:10A330000006D5D405A902A8FAF73EFF0006CFD43F
:10A3400002A99DF80000FCF72AFB0006C8D402A968
:10A3500000E0D9E09DF80000FCF780F80006BFD4CB
:10A36000BDF8080002A9401CADF808009DF80000E7
:10A37000FCF767F80006B3D405A8FBF7E9FE000672
:10A38000AED4BDF8140098B102A99DF80000FCF706
:10A390000BFA0006A4D405A902A8FAF7F2FF0006FA
:10A3A0009ED402A99DF80000FCF7F1F9000697D4AD
:10A3B00005A8FBF7DEFE000692D4BDF81400A8B194
:10A3C00002A99DF80000FCF705FA000688D405A94B
:10A3D00002A8FAF7D6FF000687D402A900E08AE2B5
:10A3E0009DF80000FCF7E9F9000687D401208DF8FC
:10A3F0000400C0B205A9FBF7CFFE000684D405987F
:10A40000B8B19DF8041002AA9DF80000FCF758F8B6
:10A41000000685D405A902A8FAF7CEFE000688D466
:10A420009DF8041002AA9DF80000FCF739F8000618
:10A4300085D49DF8040005A9FBF7C3FE000685D46A
:10A440000598B8B19DF8041002AA9DF80000FCF729
:10A4500053F800068FD405A902A8FAF7FDFE0006FE
:10A4600089D49DF8041002AA9DF80000FCF737F883
:10A47000000685D49DF80400401CC0B28DF804008D
:10A480001028B6D905A8FBF7AFFE000688D4059EB4
:10A490004FF000089EB102A99DF80000FCF7B0F84B
:10A4A000000684D405A902A8FAF786FE00068DD41A
:10A4B00002A99DF80000FCF796F8000686D405A8CE
:10A4C000FBF7A3FE000687D405984FF00009B0F112
:10A4D000000A13D002A99DF80000FCF7A7F80006B7
:10A4E0008CD405A902A8FAF767FE000686D402A953
:10A4F0009DF80000FCF78DF800068AD401A90B2016
:10A5000010F0C8FF000601D528689DE69DF80400FC
:10A51000012801D0032823D105A8FBF708FE000677
:10A5200086D402AA01219DF80000FCF701F800067C
:10A5300085D405A902A8FAF73FFE00068AD407E0F1
:10A54000A6000010080000100C0000101000001001
:10A5500002AA01219DF80000FBF7DAFF000688D46B
:10A560009DF80400022803D0042801D0062873D1E6
:10A5700046EA0A0048EA090108436ED086EA0A0161
:10A5800088EA0900014368D000200990BAEB06016F
:10A5900079EB080005D2B6EB0A0A68EB0904012042
:10A5A00004E0BAEB060A69EB080400201A900020C8
:10A5B00081468046064601208DF80400C0B205A9F8
:10A5C000FBF7EAFD00068BD405999DF8040019EB12
:10A5D000010948EB060805A9FBF7F3FD000685D441
:10A5E000059810B10998401C09909DF80400401C82
:10A5F000C0B28DF804001028E0D9002610208DF894
:10A600000400C0B205A9FBF7C7FD000688D4059871
:10A61000049030434BD00498AAFB003204FB002086
:10A620000AFB06015FEA58024FEA39001818514147
:10A630004A4643462FF07AFABAEB000A049A64EBD2
:10A640000104B9EB02091A9A68EB060832B1049AC0
:10A65000101A66EB010604E082E056E0049A101836
:10A660004E4109990590491E09919DF8041002AACE
:10A670009DF80000FBF75CFF0006A4D405A902A822
:10A68000FAF79AFD00069ED49DF8041002AA9DF8E0
:10A690000000FBF73DFF000695D400BF9DF80400C5
:10A6A000401E10F0FF008DF80400AAD158E05AEACD
:10A6B0000400F3D059EA0800F0D19DF8040005A980
:10A6C000FBF77FFD00068AD405980028E6D01A988B
:10A6D00048B1092028600020CBF800007846FE49E8
:10A6E00008600920B0E5099800EBD070421012EB29
:10A6F0000A0044EBE271099A4FEAE2732FF016FA6E
:10A70000BAEB000A64EB0104A8E701208DF804000D
:10A71000C0B205A9FBF740FD0006AED40598B8B15C
:10A720009DF8041002AA9DF80000FBF701FF000647
:10A73000A3D405A902A8FAF73FFD00069DD49DF811
:10A74000041002AA9DF80000FBF7E2FE000694D474
:10A750009DF80400401CC0B28DF804001028D7D921
:10A7600001248DF8044000BF9DF8040005A9FCF702
:10A77000AFF9000687D40598B8B19DF8041002AA75
:10A780009DF80000FCF788F9000685D405A902A809
:10A79000FAF712FD000696D49DF8041002AA9DF85F
:10A7A0000000FCF769F900068DD49DF80400401CF8
:10A7B000C0B28DF804001128D6D305A8FBF7D0FE4F
:10A7C0000006AAD4059898B102A99DF80000FBF7ED
:10A7D000DAFE0006A1D405A902A8FAF7EDFC0006EE
:10A7E0009BD402A99DF80000FBF7C0FE000694D49C
:10A7F00005A8FBF7DBFE00067DD4059898B102A9F9
:10A800009DF80000FBF7E6FE000674D405A902A837
:10A81000FAF7D2FC00066ED402A99DF80000FBF7FF
:10A82000CCFE000667D48DF8044000BF9DF80400FC
:10A8300005A9FBF7D4FB00065DD40598B8B19DF8D7
:10A84000041002AA9DF80000FBF709FF000652D48D
:10A8500005A902A8FAF7B0FC00064CD49DF8041034
:10A8600002AA9DF80000FBF7EAFE000643D49DF81B
:10A870000400401CC0B28DF804000B28D6D305A8F4
:10A88000FBF755FC000636D4059898B378883C2130
:10A89000B0FBF1F0401CC1B28DF8041002AA9DF883
:10A8A0000000FBF7FBFE000625D405A902A8FAF775
:10A8B00083FC00061FD49DF8041002AA9DF8000036
:10A8C000FBF7DCFE000616D4397902AA9DF80000D9
:10A8D000FBF703FF00060ED405A902A8FAF76CFCEB
:10A8E000000608D4397902AA9DF80000FBF7E5FEBE
:10A8F000000600D400E087E08DF804409DF80400D5
:10A9000005A9FCF791F800067ED49DF8041002AA70
:10A910009DF80000FCF7A1F8000675D405A902A86F
:10A92000FAF74AFC00066FD49DF8041002AA9DF8BD
:10A930000000FCF782F8000666D49DF80400401C75
:10A94000C0B28DF804000528D8D902A90120FBF770
:10A95000AAFA000658D405A90120FBF740FB00061F
:10A9600052D49DF80000012814D002280DD00328ED
:10A970000BD004280ED0882002212860CBF80010CC
:10A9800079465548016088205EE405A902A8FAF7D7
:10A990008DFD03E005A902A8FAF74DFD00067AD463
:10A9A00002A90120FBF773FA000674D4012005F018
:10A9B00014F900066FD413A8FCF7CEF900066AD488
:10A9C00046499DF84C004FF092060978084267D03E
:10A9D00016A9032005F084F800065CD418A9052008
:10A9E00003F02DFA000656D4052216A918A82FF058
:10A9F000FDFB88B1FBF7B1F8422010F0E0FB03202B
:10AA000024F055F9312000E01BE02E60CBF8000067
:10AA10007846314908605CE012A9002003F00FFA83
:10AA2000000638D49DF8480080062FD507F070FC4A
:10AA3000000604D43846FFF78DFB000602D507F068
:10AA400051FB28E03888ADF828007888ADF82A0056
:10AA500038798DF82C0014A90AA803F0FAFEDBF867
:10AA6000000028280FD028780006E8D414A8FBF7A7
:10AA70009FFC0006E3D415A8FBF7ABFC0006DED470
:10AA80001C98047015E001201190EFE705A8FBF772
:10AA90004EFB000602D5FBF760F80CE4059840B9C0
:10AAA00007F036FC0006CAD43846FFF753FB000611
:10AAB000C5D48DF8044001A8FBF7A5F90006BED463
:10AAC000119868B128212E60CBF800107946024811
:10AAD0000160922019E50000100000108AC10300F7
:10AAE000FAF7A6FF11E50000F8B5054646793B4C9C
:10AAF0003B4A3C4B86200EB1022E02D92060072033
:10AB000005E02E790EB11E2E06D9206005201060BA
:10AB1000784618608620F8BD29B16988288801F038
:10AB20008FFD000641D40027012600976946304674
:10AB3000FBF749FA000638D4761CF6B20B2EF5D393
:10AB40006846FBF754FA00062FD46846FBF771FA03
:10AB500000062AD46846FBF725FA000625D4ADF88E
:10AB600000706846FBF754FA00061ED46846FBF7EF
:10AB700071FA000619D42846FBF7E1F9000614D44F
:10AB8000A81CFBF7EDF900060FD4281DFBF7F9F917
:10AB900000060AD4012007F061FE000605D44FF03C
:10ABA0000040FAF7DFFE000601D52068F8BD02205C
:10ABB0008DF800006846FBF77EF9000607D40A49C5
:10ABC00001200870681DFBF715FC000602D5FAF796
:10ABD000C4FFF8BDFAF72CFFF8BD00000800001014
:10ABE0000C00001010000010000000101CB54FF009
:10ABF0000040FAF7B7FE000602D5174800681CBDF2
:10AC000007F078FF00061ED400248DF80040684647
:10AC1000FBF751F9000616D48DF8044001A8FBF7A4
:10AC2000E9FB00060FD46846FBF719F900060AD4C1
:10AC30009DF8000002280BD18DF800406846FBF714
:10AC4000E2F8000604D507F04DFAFAF786FF1CBDBE
:10AC5000FAF7EEFE1CBD0000080000102DE9F04FD1
:10AC6000054600799A4C9B4E9B4F93B04FF0860857
:10AC70004FF0050B08B11E2804D9C4F80080C6F8AF
:10AC800000B017E0288848F6AD614FF014098842FB
:10AC900005D900BFC4F80080C6F800900AE06888B3
:10ACA0004FF0170AB0F5B46F0AD300BFC4F80080A4
:10ACB000C6F800A078463860862013B0BDE8F08F53
:10ACC00002A8FBF746F9000615D42888BDF808103D
:10ACD0008842DFD309D102A8FBF74CF900060AD459
:10ACE0006888BDF808108842E0D34FF00040FAF7BA
:10ACF00039FE000601D52068DFE76846FBF784FBD4
:10AD000000067CD402A8FBF757F9000677D4029816
:10AD100098B103A99DF80000FBF7FBFC00066ED478
:10AD200002A903A8FAF748FA000668D403A99DF817
:10AD30000000FBF7E1FC000661D403A99DF80000C8
:10AD4000FBF7FDFC00065AD4BDF80C0003A9401C1B
:10AD5000ADF80C009DF80000FBF7E4FC00064ED4B3
:10AD60000120804602A9FBF73AF9000647D4029871
:10AD7000A8B103AA41469DF80000FBF7F9FC0006C4
:10AD80003DD402A903A8FAF717FA000637D403AA9C
:10AD900041469DF80000FBF7DBFC00062FD408F1CC
:10ADA0000100C0B280460A28DCD903A90120FBF7C4
:10ADB0007AF8000623D402A90120FBF710F9000657
:10ADC0001DD49DF800004FF0880801280BD0022800
:10ADD00003D00220C4F800801DE002A903A8FAF7FE
:10ADE00065FB04E00BE002A903A8FAF724FB0006C8
:10ADF00005D403A90120FBF74AF8000602D5FAF7AB
:10AE0000ACFE5AE79DF80000012809D002280AD0BC
:10AE10000920C4F8008030607846386088204CE70C
:10AE20008DF815B002E006208DF8150002A8FBF79A
:10AE30006EF8000642D4BDF80800401CADF81E00B4
:10AE400002A8FBF753F8000638D40298401CCDF84E
:10AE50001A0002A8FBF749F900062FD402980890BF
:10AE60001E490DF125002FF0EDF928798DF8240009
:10AE70002888ADF816006888ADF8180005F04EFA7D
:10AE800000061BD405A804F08BF9000616D405A80B
:10AE900005F0ECFA000611D4FAF7B1FD00060DD466
:10AEA00005A804F0A8F9000608D405A805F009FBD8
:10AEB000000603D4FAF7AFFD000602D507F012F939
:10AEC0009DE7064900200870FAF7B2FDF5E600009C
:10AED000080000100C00001010000010CECA07205F
:10AEE00030B5044600785C4D91B008B10A280AD903
:10AEF00086205A492860042008607846584908602E
:10AF0000862011B030BDA0680D90211D0DA8FAF764
:10AF10003AFB000605D44FF00040FAF723FD000687
:10AF200001D52868EDE70EA8FBF76BF8000650D4B2
:10AF30000DA90EA8FAF7B1F900064AD40EA8FBF73E
:10AF400056F8000645D40EA8FBF76CF8000640D46E
:10AF5000BDF83800401CADF838000EA8FBF758F8D3
:10AF6000000636D420780EA9FBF739F8000630D455
:10AF70000DA90EA8FAF791F900062AD420780EA997
:10AF8000FBF721F8000624D40EA8FBF715F80006FD
:10AF90001FD40DA90EA8FAF780F9000619D40EA83F
:10AFA000FBF700F8000614D42046FBF764F800060F
:10AFB0000FD4201DFBF77CF800060AD404F108002A
:10AFC000FBF77FF8000604D40DA8FBF784F8000611
:10AFD00002D5FAF7C2FD94E707F099FB000635D4D5
:10AFE0000FA8FAF772FF000630D49DF83C00022843
:10AFF00003D107F093FD000628D49DF83C000128FA
:10B0000027D109208DF8010020788DF802000D98D5
:10B01000CDF80300684604F0C3F8000616D468466D
:10B0200005F024FA000611D4FAF7E9FC00060DD465
:10B03000684604F0E0F8000608D4684605F041FAD6
:10B04000000603D4FAF7E7FC000602D507F04AF839
:10B05000BFE7FAF7EDFC54E7080000100C00001001
:10B060001000001030B504460078544D8FB008B180
:10B070000A280AD9862052492860042008607846A8
:10B080005049086086200FB030BDA0680D90211D8A
:10B090000DA8FAF778FA000605D44FF00040FAF749
:10B0A00061FC000601D52868EDE70EA8FAF7A9FFB4
:10B0B000000650D40DA90EA8FAF710F900064AD4DC
:10B0C0000EA8FAF794FF000645D40EA8FAF7AAFFD7
:10B0D000000640D4BDF83800401CADF838000EA87A
:10B0E000FAF796FF000636D420780EA9FAF777FF14
:10B0F000000630D40DA90EA8FAF7F0F800062AD4FD
:10B1000020780EA9FAF75FFF000624D40EA8FAF7FC
:10B1100053FF00061FD40DA90EA8FAF7DFF80006AA
:10B1200019D40EA8FAF73EFF000614D42046FAF709
:10B13000A2FF00060FD4201DFAF7BAFF00060AD4BA
:10B1400004F10800FAF7BDFF000604D40DA8FAF7D1
:10B15000C2FF000602D5FAF700FD94E707F0F7FA00
:10B16000000624D40A208DF8010020788DF8020012
:10B170000D98CDF80300684604F012F8000616D4C6
:10B18000684605F073F9000611D4FAF738FC00069A
:10B190000DD4684604F02FF8000608D4684605F080
:10B1A00090F9000603D4FAF736FC000602D506F043
:10B1B00099FFD0E7FAF73CFC65E7000008000010B3
:10B1C0000C0000101000001030B504460078564DF9
:10B1D0008FB008B10A280AD9862054492860042073
:10B1E000086078465249086086200FB030BDA068DC
:10B1F0000D90211D0DA8FAF7C6F9000605D44FF0F1
:10B200000040FAF7AFFB000601D52868EDE70EA86D
:10B21000FAF719FF000650D40DA90EA8FAF73DF869
:10B2200000064AD40EA8FAF704FF000645D40EA87B
:10B23000FAF71AFF000640D4BDF83800401CADF8FC
:10B2400038000EA8FAF706FF000636D420780EA9BB
:10B25000FAF7C5FE000630D40DA90EA8FAF73EF89D
:10B2600000062AD420780EA9FAF7ADFE000624D4F1
:10B270000EA8FAF7A1FE00061FD40DA90EA8FAF732
:10B280002DF8000619D40EA8FAF78CFE000614D487
:10B290002046FAF7F0FE00060FD4201DFAF708FF4B
:10B2A00000060AD404F10800FAF70BFF000604D4E4
:10B2B0000DA8FAF710FF000602D5FAF74EFC94E746
:10B2C00007F065FA000629D411208DF801000EA8B8
:10B2D000FAF797FE000621D40E98CDF802000D98DB
:10B2E000CDF80600684603F05BFF000616D46846FA
:10B2F00005F0BCF8000611D4FAF781FB00060DD466
:10B30000684603F078FF000608D4684605F0D9F8CF
:10B31000000603D4FAF77FFB000602D506F0E2FE32
:10B32000CBE7FAF785FB60E7080000100C0000107F
:10B33000100000102DE9F04F85B06846FAF76DFD5A
:10B34000F84F00060ED49DF80000DFF8DC93DFF81C
:10B35000DCA30024012809D001A90120FBF768F82B
:10B36000000607D5386805B0BDE8F08F3C60C9F825
:10B3700000401CE18DF800400DF104029DF8000032
:10B380009DF80410135C401CC0B219448DF80410E1
:10B390008DF800000528F1D31046FAF70CF80006E6
:10B3A0007DD4A0460494ADF80C400124E04EDFF8B3
:10B3B00084B325463078022805D000EB40000BEB23
:10B3C000C00040688047E8B2054601A9FBF723F8B2
:10B3D0000006E5D401A92846FBF7E1FA0006DFD410
:10B3E00003A92846FBF72DF80006D9D403A928465F
:10B3F000FBF73DF80006D3D403A92846FBF7C7F9AD
:10B4000000064CD403A92846FBF7D7F9000646D41A
:10B410008DF800409DF8001001AA2846FBF740F87F
:10B4200000063CD49DF8001004AA2846FBF757F804
:10B43000000634D49DF8001001AA2846FBF768F8EE
:10B4400000062CD49DF80000401CC0B28DF800000E
:10B450001028DFD901A92846FBF7C5F800061ED43D
:10B4600001A92846FBF7D5F8000618D48DF800404E
:10B470009DF8001001AA2846FBF7E1F800060ED45B
:10B480009DF80000401CC0B28DF800000A28EFD9DA
:10B490008DF800409DF8001001AA284600E073E0F6
:10B4A000FBF7ECF800066FD49DF80000401CC0B21A
:10B4B0008DF800001828EDD98DF800409DF8001097
:10B4C00001AA2846FBF7F9F800065DD49DF80000B4
:10B4D000401CC0B28DF800001E28EFD98DF8004046
:10B4E0009DF8001001AA2846FBF7A7FA00064BD4E6
:10B4F0009DF80000401CC0B28DF800000528EFD96F
:10B500008DF800409DF8001001AA2846FBF7B4FA18
:10B51000000639D49DF80000401CC0B28DF8000030
:10B520001028EFD901A92846FBF720F800062BD4F4
:10B5300001A92846FBF741F8000625D46D1CEDB2A1
:10B54000042D7FF637AF25463078022805D000EB72
:10B5500040010BEBC10040688047E0B2044601A9FE
:10B56000FBF7CAF800060FD403A92046FBF7DAF868
:10B57000000609D428468DF80050C1B201AA204621
:10B58000FBF7E6F8000602D5FAF7E7FAEBE69DF8D6
:10B590000000401CC0B28DF800000A28EDD9641CE0
:10B5A000E4B2022CD0D9C7F80080C9F800807946EF
:10B5B0000020CAF80010D6E6F0B504460179594DCE
:10B5C000594E5A4F8FB0862009B11E2902D92860E2
:10B5D00005200DE0218848F6AD62914202D928602D
:10B5E000142005E06188B1F5B46F07D328601720F7
:10B5F00030607846386086200FB0F0BD0EA902207A
:10B6000004F0C1FC000615D4BDF83800A0B103F069
:10B61000CBFC00060ED446480678012E04D001204B
:10B6200007F01CF9000605D44FF01040FAF79AF91C
:10B63000000609D52868DFE7912028608A2030605D
:10B64000784638609120D7E7FFF774FE000620D4D3
:10B6500001F00EF900061CD42046FBF7C4F80006E2
:10B6600017D4A01CFBF7CEF8000612D4201DFBF760
:10B67000DAF800060DD401208DF800006846FAF7CC
:10B68000C2FB000605D469462B200FF003FF00061D
:10B6900002D5FAF762FAAFE79DF80000C00701D1C2
:10B6A0006079E8B3012E49D06846FAF71FFC00061E
:10B6B00033D46846F9F7FEFF00062ED46846FAF741
:10B6C0000BFC000629D406F089FC000625D41A4993
:10B6D0000220087012208DF805006946042004F04D
:10B6E000FFF9000619D4BDF80000401CADF80600B3
:10B6F00020798DF810002088ADF808006088ADF83A
:10B700000A006846FAF7F2FB000606D40098039098
:10B7100001A803F070FD000610D506F0E3FCB8E7C1
:10B720000CE00000080000100C00001010000010D9
:10B730009EC20720A0C2072000000010FAF778F987
:10B740005AE70000F8B505460379384C3849394ABC
:10B7500086200BB11E2B02D9206005200EE02B881D
:10B7600048F6AD671426BB4202D920600E6006E0A1
:10B770006B88B3F5B46F06D3206017200860784655
:10B7800010608620F8BD2C490120FAF751FE000612
:10B7900040D42A490220FAF74BFE00063AD4284644
:10B7A000FAF7CDFB000635D4A81CFAF7D9FB000642
:10B7B00030D4281DFAF7E5FB00062BD40025684697
:10B7C0000095FBF7BBF8000624D468460095FBF70C
:10B7D000C4F800061ED48DF800606846FBF760F8D8
:10B7E000000617D40120ADF800006846FBF77FF88B
:10B7F00000060FD469461C200FF04CFE000609D449
:10B800009DF8000040B1ADF800506846FAF775FBAE
:10B81000000601D52068F8BD032009498DF8000015
:10B82000022008706846FAF746FBF8BD08000010D1
:10B830000C0000101000001064C1072069C107202F
:10B84000000000102DE9FC414FF00040FAF78AF8A3
:10B850004C4C00067ED46846F9F7B9FD00062AD4A0
:10B8600001273E46F0B205466946FAF710FB00068E
:10B8700021D46D1CEEB20B2EF4D300256846009542
:10B88000FAF72AFB000616D4ADF800506846FAF71E
:10B8900034FB00060FD468460095FAF73FFB00061C
:10B8A00009D4ADF800700220C0B206466946FBF725
:10B8B00008F8000605D506F015FCFAF74EF9BDE8C4
:10B8C000FC81761CF0B21B28EED92F4F042269466A
:10B8D000384620F0E3F800064ED42C4E0098B042D3
:10B8E00027D004226946381D009520F0E2F80006B2
:10B8F00042D4254804226946083020F0DAF80006D0
:10B900003AD42148042269460C3020F0D2F80006CF
:10B9100032D41D4804226946103020F0CAF80006CF
:10B920002AD4042269463846009620F0C2F8000660
:10B9300022D41548042269461430009520F0B9F845
:10B94000000619D4104804226946183020F0B1F8D6
:10B95000000600E010E00FD40B48042269461C30BA
:10B9600020F0A7F8000607D40748042269462030D3
:10B9700020F09FF8000601D52068A0E7FAF758F8F4
:10B980009DE700000800001004000020CEFAADDEA4
:10B99000FEB56846F9F70FFD284C000640D4002795
:10B9A0000125ADF808702E46F0B206466946FAF752
:10B9B00032FD000634D402A93046FAF742FD0006F3
:10B9C0002ED402A93046FAF752FD000628D402A967
:10B9D0003046FAF7DCFE000622D402A93046FAF718
:10B9E000ECFE00061CD469463046FAF7FCFD000662
:10B9F00016D469463046FAF70CFE000610D4761CC1
:10BA0000F6B2042ED0D9E8B205466946FAF774FEBC
:10BA1000000605D402A92846FAF784FE000601D5DF
:10BA20002068FEBD6D1CEDB2022DECD904482760E4
:10BA300007607846034908600020FEBD080000103A
:10BA40000C000010100000107CB506466846F9F79F
:10BA5000B2FC0D4D000607D401246A46314620464B
:10BA6000FAF70CFE000601D528687CBD641CE4B220
:10BA7000052CF2D305490020286008607846044967
:10BA8000086000207CBD0000080000100C000010C1
:10BA9000100000107CB506466846F9F78CFC0D4D89
:10BAA000000607D401246A4631462046FAF705FE0F
:10BAB000000601D528687CBD641CE4B2052CF2D3D5
:10BAC0000549002028600860784604490860002085
:10BAD0007CBD0000080000100C00001010000010D9
:10BAE000FEB507466846F9F766FC144D000617D404
:10BAF0000026012402966A4639462046FAF7D0FC11
:10BB000000060DD402AA39462046FAF7E8FC0006E2
:10BB100006D46A4639462046FAF7FAFC000601D5F3
:10BB20002868FEBD641CE4B2052CE4D304482E60F2
:10BB300006607846034908600020FEBD080000103A
:10BB40000C000010100000102DE9FC41074668466B
:10BB5000F9F731FC144E000615D401252C46E0B24D
:10BB600004466A463946FAF76AFD00060BD4641C9F
:10BB7000E4B2052CF3D3E8B204466A463946FAF734
:10BB8000E7FD000602D53068BDE8FC81641CE5B223
:10BB9000032DF0D305490020306008607846044941
:10BBA00008600020F0E70000080000100C00001002
:10BBB000100000102DE9F04F97B080464FF00009BB
:10BBC0008A4681F80090052002F0D4F9FE4C000668
:10BBD0007ED4FF2004F001F80006F9D415A8FBF785
:10BBE000BBF80006F4D46946002003F0BCFE000652
:10BBF000EED4BDF800009027F44DF54E192802D37D
:10BC000001202760E1E06946022004F0BCF900064B
:10BC1000DED4BDF8000090B1EE480DF12C0B007899
:10BC200000287CD06946012003F09DFE0006CFD499
:10BC3000BDF80000402805D303202760C5E00C2094
:10BC40002760C2E014A9002002F0F9F80006BFD472
:10BC50009DF85000010902D004202760B5E00107DB
:10BC60000BD5400709D4872020607846C5F800909E
:10BC70003060872017B0BDE8F08F03A9052002F0DF
:10BC8000DEF80006A4D46946032003F029FF00066D
:10BC90009ED42068052805D0052203A968462EF009
:10BCA000A5FAD0B19DF8500000077DD56946002067
:10BCB00003F016FF00068BD403A90B2002F0BFF897
:10BCC000000685D40C2203A968462EF08FFA00E006
:10BCD0008EE028B10520276077E00720276074E018
:10BCE00003A90C2002F0ABF8000691D4062208F15B
:10BCF000060103A82EF07AFA10B10620276064E04E
:10BD000003A9112002F09BF8000671D406224146D7
:10BD100003A82EF06BFA18B10820276055E0D4E094
:10BD200069460E2002F08BF8000661D403A800F0EB
:10BD3000F0FC00065CD4BDF80000BDF80C10884291
:10BD400007D963200FF03BFA000651D40920276081
:10BD50003BE003A9F4F7F7FD9DF80C00694600F5F8
:10BD6000FA60ADF82C009DF80D008DF82E009DF8BE
:10BD70000E008DF82F000F2002F061F8000637D476
:10BD8000BDF800103C20B1FBF0F28DF83020B1FB83
:10BD9000F0F200FB12108DF831008DF8329003A9FB
:10BDA000102002F04CF800E023E0000620D46946A1
:10BDB000042003F095FE00061AD4BDF80000BDF87B
:10BDC0000C10884206D00A20276028607846306030
:10BDD00090204FE76946062002F031F8000672D441
:10BDE000BDF80C00BDF80010401C8142EBD110E002
:10BDF00069E002F0D8F800287FF46FAF0BF104007F
:10BE00001AF06DFB00065ED40BA81AF099FB000631
:10BE100059D403F009F9000655D40BF107010020AD
:10BE200003F05EFE00064ED4D8F80610CDF83F10A1
:10BE3000B8F80A00ADF84300D8F80010CDF8451066
:10BE4000B8F80400ADF8490013A9042003F048FE37
:10BE5000000638D4D8F806100791B8F80A00ADF8F3
:10BE60002000D8F80010CDF82210B8F80400ADF882
:10BE70002600D8F80C000A9006A90BA8F4F7FEFDDE
:10BE8000BDF84C00ADF81A0006A8FAF758F80006FD
:10BE900019D49DF830109DF83100C1EB011100EB71
:10BEA0008100ADF800006846FAF75AF800060AD497
:10BEB0004948FAF766F8000605D44FF00040F9F754
:10BEC00051FD000604D52068D4E60BF1040097E785
:10BED00006F00AFD000675D406A806F01AFD000655
:10BEE00070D49DF8500000070ED43A48007858B13D
:10BEF0003A48007800280BA802D002F077FE01E053
:10BF000002F05FF800066FD4324F4FF001088AF854
:10BF100000803878D8B102F0D5FA000664D4012147
:10BF20002F4806F024FD00060AD5F4F78FF901F03A
:10BF300055FDF4F7A0F906F0D5F8F9F70EFEC2E7C3
:10BF400002F0FCFA00064FD420680028E7D0112048
:10BF500003F0CFFF000647D406A9002003F0D9FF65
:10BF6000000641D4387858B107A9052001F067FFD1
:10BF7000000639D406A9012003F0CBFF000633D414
:10BF8000122003F0B6FF00062ED49DF85400D0B165
:10BF90006846F9F7ABFF000626D46846F9F78AFB36
:10BFA000000621D46846F9F797FF00061CD400BFAD
:10BFB000FAF7EEFE000617D44F468AF80090F9F71C
:10BFC00037FD0FE010E014E0080000100C00001036
:10BFD000100000108AC1030091C2072002C0072090
:10BFE00048C6072000064DD506F07CF8F9F7B5FDE8
:10BFF00040E647468DF800806846FAF7C6FE000620
:10C00000F2D4ADF81090CDF80C908DF81290B8469F
:10C0100038468DF80070C0B203A9F9F738FF000662
:10C02000E2D49DF80000401CC0B28DF800000A2840
:10C03000F1D94F4603A8CDF80C90F9F74DFF000653
:10C04000D2D403A80397F9F769FF0006CCD4ADF862
:10C050000C7003A8F9F751FF0006C5D44046ADF8AF
:10C060000C808DF80080C0B203A9FAF72AFC000604
:10C07000BAD49DF80000401CC0B28DF800001B2807
:10C08000F1D995E7276078462F6030600020F1E510
:10C090002DE9F04FDFF838B38046CE4E9BF8000014
:10C0A000CD4DCE4C97B04FF0920A4FF0020940B1FF
:10C0B00016A801F033FC00067ED49DF85900AC2888
:10C0C00046D1002188F80010052001F053FF00063A
:10C0D000F2D4FF2003F081FD0006EDD415A8F9F796
:10C0E0009CFE0006E8D49DF8540048B191202060E1
:10C0F0009C20286078463060912017B0BDE8F08F12
:10C100006946012003F02FFC0006D5D4BDF80000DD
:10C110009027402802D30320276023E069460220AD
:10C1200003F031FF0006C7D4BDF80000C0B101F034
:10C130003AFF0006C0D42868232809D00FA90020A0
:10C1400001F07DFE0006B7D49DF83C0000090BD03D
:10C15000C4F800A07846C5F8009030609220CCE783
:10C160000C202760286061E003A9052001F067FE2C
:10C170000006A1D46946032003F0B2FC00069BD45C
:10C1800020684FF0070A28B90522694603A82EF057
:10C190002DF898B39DF83C0000077DD56946002036
:10C1A00003F09EFC000687D403A90B2001F047FE94
:10C1B00000068DD40C2200E0ACE003A968462EF006
:10C1C00015F810B105202760CCE769460E2001F074
:10C1D00036FE000686D403A800F09BFA000694D42D
:10C1E000BDF80000BDF80C10884208D063200EF0A6
:10C1F000E6FF000689D409202760B3E713E069460B
:10C20000042003F06DFC00068DD403A9102001F07A
:10C2100016FE00067ED4BDF80000BDF80C104FF0ED
:10C220000A0A884206D02760C5F800A07846306028
:10C23000902062E76946062001F001FE000669D4FD
:10C24000BDF80C00BDF80010401C8142EBD103A9E1
:10C250000C2001F0F4FD00065CD46946012003F0D7
:10C260003FFC000656D40622694603A82DF0BEFF07
:10C2700010B10620276075E703A9112001F0DFFD4A
:10C28000000647D46946022003F02AFC000641D488
:10C29000062203A9684600E005E02DF0A7FF30B1B3
:10C2A000082027605EE701F07EFE0028BBD106ADC6
:10C2B000281D1AF014F900062CD406A81AF040F92B
:10C2C00000067DD4E91D002003F00AFC000677D4A7
:10C2D0000DF12B01012003F003FC000670D40DF1D9
:10C2E0003101022003F0FCFB000669D40EA90420F2
:10C2F00003F0F6FB000663D4BDF83800ADF8420049
:10C3000010A906A8F4F7BAFB11A9052001F097FDC2
:10C31000000600E054E053D44FF00040F9F722FB50
:10C3200000064DD406F007FB000640D49DF83C0003
:10C3300000070BD49BF80000002806A802D002F0EA
:10C3400055FC01E001F03DFE000630D4012188F8E3
:10C35000001002F0B7F8000629D4214D0121204831
:10C3600006F005FB00060AD5F3F770FF01F036FB77
:10C3700000061CD4F3F77FFF2078000617D402F0E4
:10C38000DDF8000613D495F800010028E6D111204D
:10C3900003F0AFFD00060AD410A9012003F0B9FD97
:10C3A000000604D4122003F0A4FD000604D505F015
:10C3B00099FEF9F7D2FBA0E6F9F73AFB000601D5A2
:10C3C00020689AE688F80090012006F047FA94E683
:10C3D00002C00720100000100C0000100800001020
:10C3E00048C607202DE9F0438BB007A9012019F0BA
:10C3F00041FB594C000645D4684601F088FC000614
:10C4000040D408A9032003F06BFB544DDFF85081A2
:10C41000000616D40027052208A903A82DF0E6FE81
:10C4200080B142200EF0CBFE00062BD4922020607B
:10C430003120794628609220C8F800100BB0BDE882
:10C44000F08301279DF811004FF0000641074FF0DF
:10C45000870903D4C4F800902E606DE0400654D5DF
:10C4600006A8F9F7EBFC000674D49DF818000E2816
:10C4700001D0002FEED060200EF0A1FE000602D504
:10C4800005F030FE66E001F08EFD000662D46846DD
:10C4900000F03FF900065DD40DF1020000F01DF937
:10C4A000000657D41E208DF80400684601F0F4FD04
:10C4B00000064FD48DF800606846F9F7A4FC00062A
:10C4C00048D4684601F0A1FB000643D4BDF8000043
:10C4D000401E80B201F0C3FF00063BD4214D012174
:10C4E000204806F044FA000606D5F3F7AFFE01F047
:10C4F00075FAF3F7C0FE2DE002F020F8000629D40B
:10C5000095F800010028EAD11BE00798C00707D082
:10C510008DF800606846F9F776FC00061AD410E042
:10C520006846F9F77AFC000614D49DF8000040B183
:10C530000420C4F80090286079468720C8F80010CD
:10C540007CE733200EF03BFE000603D401F017FE1B
:10C55000000695D4206871E7080000100C00001058
:10C560001000001048C6072038B54FF00040F9F71A
:10C57000F9F9104D000617D400248DF800406846E4
:10C58000F9F7BAFD000606D48DF800406846F9F7C1
:10C5900092FC000602D5F9F7E0FA38BD684600942F
:10C5A000F9F7BBFD000601D5286838BDF9F740FA58
:10C5B00038BD0000080000101CB54FF00040F9F72E
:10C5C000D1F9000602D51D4800681CBD01A8F9F785
:10C5D0001BFF00062CD46846F9F788FC000627D418
:10C5E0006846F9F767F8000622D46846F9F774FC44
:10C5F00000061DD46846F9F78AFC000618D4684680
:10C60000F9F731F8000613D46846F9F776FC00060E
:10C610000ED400248DF8044001A8F9F7EBFE0006C3
:10C6200006D48DF800406846F9F745FC000602D5AF
:10C63000F9F793FA1CBDF9F7FBF91CBD08000010CF
:10C640002DE9FC5F9B4D9C4E9C4C894607004FF0AA
:10C6500086084FF0140A03D048F6AD60874204D92B
:10C66000C4F80080C5F800A008E04FF0170BB9F53A
:10C67000B46F08D3C4F80080C5F800B078463060C5
:10C680008620BDE8FC9F01A8FAF7B6F800060BD497
:10C69000BDF804003F1A4FF4B4604743E0D4684645
:10C6A000FAF7BAF8000601D52068EAE7BDF80010ED
:10C6B000A9EB0100C019DDD40021B0F5B46F06DB91
:10C6C0008A2020607846296030608A20D9E721607E
:10C6D0007846296030600020D3E738B504466846C4
:10C6E00019F0FDFE0106754801D5006838BD9DF8BA
:10C6F00000209DF80110C2EB021201EB82012180A3
:10C70000002101606B48016078466B490860002099
:10C7100038BD38B50446684619F012FF000602D548
:10C720006648006838BD21466846F4F7A7F938BD69
:10C730007CB50025ADF800506846FFF7CEFF5F4C92
:10C74000000604D401A8FFF7E4FF000601D5206825
:10C750007CBDBDF80010BDF80400FFF771FF55491E
:10C76000554A38B1912020608820086078461060D2
:10C7700091207CBD256078460D60106000207CBD56
:10C780002DE9FE43DFF8388181464A4E98F80000D3
:10C79000494F4A4C002510B188F8005062E06946C4
:10C7A0003D200EF042FF000651D49DF80000E8B392
:10C7B000012188F8001001A8FFF78FFF000646D47A
:10C7C00002A8FFF7A6FF000641D4BDF80800BDF897
:10C7D0000410C0EB001000EB400001EB401801A872
:10C7E000FAF7EDF9000632D402A8FAF7D7F90006F5
:10C7F0002DD4BDF80800BDF80410C0EB001000EB0C
:10C80000400001EB40109DF80010C1EB011100EB5E
:10C810008101414526D8B9F1000F1BD062200EF0EE
:10C82000CEFC000613D46946532000E01AE00EF057
:10C8300031FE00060BD49DF8000010F002008DF8C8
:10C84000000007D0012006F009F8000602D5206894
:10C85000BDE8FE8387202060052030607846386080
:10C860008720F5E725607846356038600020EFE7DF
:10C870001CB56846FFF731FF104C00060ED401A826
:10C88000FFF747FF000609D401A8FAF77DF9000673
:10C8900004D46846FAF789F9000601D520681CBD62
:10C8A00004490020206008607846034908600020A1
:10C8B0001CBD00000C00001010000010080000104B
:10C8C0004EC1072010B5044690B04FF00040F9F774
:10C8D00049F8000603D53648006810B010BD201D89
:10C8E000FAF773F8000617D404F10800FAF77EF897
:10C8F000000611D4207A0EA9FAF796F800060BD498
:10C90000211D0EA8F8F7C9FC000605D4207A0EA94F
:10C91000FAF77DF8000602D5F9F71FF9DDE70DA952
:10C920004B200EF0B7FD00063CD49DF83400C00744
:10C9300003D005F04CFF000634D413208DF801001D
:10C94000207A8DF802006068CDF803009DF834006D
:10C95000800704D5684602F023FC000622D49DF827
:10C960003400C00704D0684603F080FD000619D4E7
:10C97000F9F745F8000615D49DF83400800704D572
:10C98000684602F038FC00060CD49DF83400C0075D
:10C9900004D0684603F095FD000603D4F9F73BF890
:10C9A000000602D505F09EFBB6E7F9F741F894E7DB
:10C9B0000800001010B5044690B04FF00040F8F7A2
:10C9C000D1FF000603D53648006810B010BD201D09
:10C9D000F9F7FBFF000617D404F10800FAF706F890
:10C9E000000611D4207A0EA9FAF71EF800060BD41F
:10C9F000211D0EA8F8F772FC000605D4207A0EA9B6
:10CA0000FAF705F8000602D5F9F7A7F8DDE70DA952
:10CA10004B200EF03FFD00063CD49DF83400C007CB
:10CA200003D005F0F4FE000634D414208DF8010084
:10CA3000207A8DF802006068CDF803009DF834007C
:10CA4000800704D5684602F0ABFB000622D49DF8AF
:10CA50003400C00704D0684603F008FD000619D46E
:10CA6000F8F7CDFF000615D49DF83400800704D5F3
:10CA7000684602F0C0FB00060CD49DF83400C007E5
:10CA800004D0684603F01DFD000603D4F8F7C3FF89
:10CA9000000602D505F026FBB6E7F8F7C9FF94E7D4
:10CAA0000800001070B592B0002604468DF8406072
:10CAB0004079B74DA0B110A8F9F7B8FB000674D4BF
:10CAC0009DF8400008B110280AD98620B149286095
:10CAD000032008607846B0490860862012B070BD17
:10CAE0004FF00040F8F73EFF0006E8D460790028D8
:10CAF00075D06846F9F71BFB00066CD4A079214677
:10CB00000028684652D0F8F7E9FB000663D468466F
:10CB1000F9F703FB00065ED469469DF84000F9F77B
:10CB20003BFB000657D4A07921460028684640D038
:10CB3000F8F7D4FB00064ED469469DF84000F9F79B
:10CB40001FFB000647D410A8F9F7DDFB000642D40E
:10CB50002046F9F7C7FB00063DD420796946F9F76E
:10CB6000B7FF00067FD421466846F8F796FB00061B
:10CB700079D420796946F9F79EFF000673D4A0792D
:10CB80000028684618D0F9F7EBFC00066BD4214664
:10CB90006846F8F782FB000665D46846F9F7D7FCCB
:10CBA000000660D405F069FC73E0BFE0F8F775FBA0
:10CBB000ABE7F8F772FBBDE7F9F7F8FC000652D4D3
:10CBC00021466846F8F769FB00064CD46846F9F739
:10CBD000E3FCE5E703E046E005F084FA43E00FA854
:10CBE000F9F7A5FA00063ED40FA8F9F7D0FB000626
:10CBF00039D40F980090A07921460028684635D096
:10CC0000F8F76CFB00062ED46846F9F786FA0006A2
:10CC100029D42046F9F7AAFB000624D4A0790028DD
:10CC2000684626D0F9F7E0FA00061CD4214668468B
:10CC3000F8F733FB000616D46846F9F7CBFA00067E
:10CC400011D420796946F9F743FF00060BD4214639
:10CC50006846F8F722FB000605D420796946F9F703
:10CC60002AFF000613D5F8F778FF37E7F8F715FB2A
:10CC7000C8E7F9F7CAFA0006F5D421466846F8F77E
:10CC80000CFB0006EFD46846F9F7B5FAD7E705F0D4
:10CC900014FC0006A0D4A079A8B108208DF80500E6
:10CCA00020798DF80A00617901A871B1CDF806608C
:10CCB000C01DF9F7FFFA00068ED46846F9F70BFBA2
:10CCC000000689D40EE00720E8E70F99CDF806109A
:10CCD000C01DF9F733FB000628D46846F9F73FFB7F
:10CCE000000623D4BDF80000ADF80C002068CDF894
:10CCF0000E000EA94C200EF0CDFB000616D49DF8B8
:10CD00003800800704D501A802F04AFA0006C1D411
:10CD10009DF83800C00704D001A803F0A7FB000667
:10CD2000B8D46846FAF718F8000601D52868D5E6A1
:10CD30009DF8000060B11948007848B12068119052
:10CD4000A079002811A820D001F0D5FC0006A1D4BC
:10CD5000F8F755FE00069DD49DF83800800704D5ED
:10CD600001A802F048FA000694D49DF83800C007E4
:10CD700004D001A803F0A5FB00068BD4F8F73FFE12
:10CD8000000687D4F8F754FEA8E601F00BFDDDE7B6
:10CD9000080000100C000010100000108AC10300F1
:10CDA00071B581B04FF00040F8F7DCFD7A4C000619
:10CDB0003CD403208DF800006846F9F77CF80006A3
:10CDC00062D419208DF800006846F9F769FD000665
:10CDD0005AD472490220087001A91920F9F771FD8F
:10CDE000000623D4012005F039FD00064CD402F0E2
:10CDF000B8FB000648D4BDF8040002F018FB00069A
:10CE000042D420680025052807D0654E02F0F6FBC5
:10CE1000000639D42068D8B913E0F8F79EFE000662
:10CE200004D4012021F073FC000601D520687CBDEC
:10CE3000812020605B48056078465B49086081205E
:10CE40007CBD7078062803D0052801D00B28DDD1E1
:10CE500021F0F6FE000617D4012021F058FC000650
:10CE600012D4012005F0FAFC00060DD48DF8005014
:10CE70006846F9F720F8000606D48DF80050684699
:10CE8000F9F70EFD000602D5F8F767FE7CBDF8F74E
:10CE9000CFFD7CBD2DE9F843064689464FF00040A2
:10CEA000F8F760FD3C4C00066CD496B103208DF879
:10CEB00000006846F8F7FFFF000622D419208DF81D
:10CEC00000006846F9F7ECFC00061AD4334902204A
:10CED00008706846F9F71BF8000653D46946192014
:10CEE000F9F7EFFC00064DD4012005F0B7FC000671
:10CEF00007D403F0FEFB000603D403F00CFC00068D
:10CF000003D5F8F72AFEBDE8F8832068254FDFF83F
:10CF10009880002505280FD1F8F71FFE000631D4B0
:10CF2000012021F0F4FB00062CD4812020607946FA
:10CF30003D60C8F80010E6E703F032FC000606D4B6
:10CF400020680028F8D021F07BFE000602D505F00D
:10CF5000C9F8D6E7F8F76CFD000613D4A6B1484629
:10CF600005F07CFC00060DD48DF800506846F8F7FB
:10CF7000A2FF000606D48DF800506846F9F790FC31
:10CF8000000601D52068BEE7256079463D60002097
:10CF9000C8F80010B7E700000800001000000010FB
:10CFA0009CCA07200C000010100000102DE9FC4165
:10CFB0002F4C90460F460026C0B3F9F78EFE40B1C5
:10CFC000F3F744F900212BA021F094FCF3F753F977
:10CFD00043E08DF800606846F8F706FF6846F8F70A
:10CFE00012FF02208DF800006846F8F73FFF0006A8
:10CFF00033D46846F8F729FF00062ED46846F8F7C0
:10D0000013FF000629D40120ADF80400054601A94C
:10D010002846F9F756FC00061FD46D1C1B2DF6D9C7
:10D0200002F002F8FEF70EFC000616D4C7B1404627
:10D030000FF043FA000610D400200EF03CFE00066C
:10D040000BD40FF081FA20B900200FF0DDFC0006B0
:10D0500003D4F4F766F8000602D52068BDE8FC8129
:10D060000B482660066078460A4908600020F5E70C
:10D07000080000108EE8A8A1AAA020A8ADA8E6A8E4
:10D08000A0ABA8A7A0E6A8A8208E87930A0000005E
:10D090000C000010100000102DE9F0418AB0BB48D0
:10D0A000F8F795F9BA48F8F792F906A8F9F754FE97
:10D0B000B84C000652D49DF818000527B64EDFF88C
:10D0C000DC82002510B307A912200EF0E3F9000658
:10D0D00044D408A92E200EF0DDF900063ED405A8A0
:10D0E000F9F7E8FB000639D49DF81C10C80705D0F5
:10D0F0009DF814000E2812D0142810D09DF81400AA
:10D100000F2803D19DF82000800708D427607946B6
:10D1100035600520C8F800100AB0BDE8F081A04FC6
:10D12000880715D5002002F0BCFC000616D469461D
:10D13000002002F07AFC000610D4BDF80210022094
:10D1400002F099FC000609D4BDF80200788008E0DE
:10D150000021022002F08FFC000601D52068DBE7E9
:10D160007D803D702560794635600020C8F800104C
:10D17000D2E72DE9F04F89B04FF00005854CDFF87C
:10D180001C82854F06008DF814504FF0050B04D01B
:10D19000012E02D0022870D09DE0DFF804A24FF0EB
:10D1A00000096946022002F040FC20B1052830D079
:10D1B00093287DD152E09AF8000060B1BAF80210CD
:10D1C000BDF80220481C824211D0022002F053FC1C
:10D1D000000674D44AE001218AF80010BAF802105F
:10D1E000BDF802204B1C9A42EFD1AAF802206848F1
:10D1F00001A9F8F78EF9000661D464480DF1090120
:10D20000F8F787F900065AD4BDF80210AAF8021000
:10D210002CE0012E1FD105A8F8F7FFFD00064ED423
:10D220009DF81400B8B106A90120F9F701F900062C
:10D2300045D406A95648F8F76CF900063FD406A96C
:10D240000220F9F7F5F8000639D406A94F48F8F797
:10D2500060F9000633D48AF8005034E0BAF80210BE
:10D26000491CAAF802103868082828D109F10109D8
:10D27000B9F1640F95DB2EE0FFE705A8F8F7CDFDC7
:10D2800000061CD49DF81400E8B106A90120F9F7A6
:10D29000CFF8000613D406A93D48F8F73AF900067E
:10D2A0000DD406A90220F9F7C3F8000607D400E060
:10D2B00005E006A93548F8F72CF900060BD52068DB
:10D2C00009B0BDE8F08FC4F800B079463D60052094
:10D2D000C8F80010F4E7256079463D600020C8F8E2
:10D2E0000010EDE72DE9F04F83468DB08A460846E1
:10D2F000F8F76DF85846F8F76AF80AA8F9F72CFD20
:10D30000244C000630D49DF82800DFF89080224F8E
:10D31000002578B3002002F0C4FB000624D469463F
:10D32000002002F082FB00061ED4BDF8021002208D
:10D3300002F0A1FB000617D405AE0DF11D0905A9E9
:10D34000022002F072FB206810B193280FD015E084
:10D35000311D5846F8F7DDF8000605D44946504619
:10D36000F8F7D7F8000606D520680DB0A9E73868A9
:10D370000828E4D002E020680528E0D1256079463D
:10D380003D600020C8F80010EFE70000CF0000105B
:10D39000C8000010080000100C0000101000001061
:10D3A00050C107202DE9F04399B080462E208DF81A
:10D3B000580016468946072000F0DCFDF74C0006B1
:10D3C00054D4FF2002F009FC00064FD418A8F8F747
:10D3D00024FD00064AD49DF86000F14FF14D48B19C
:10D3E000912020609C20386078462860912019B0F8
:10D3F000BDE8F08317A800F091FA000636D49DF836
:10D400005C004FF0920110F08C0F4FF0020204D13B
:10D410009DF85D0038B1B42805D0216078463A60A7
:10D4200028609220E3E7E04819F059F800061DD47F
:10D43000DD48001F074619F083F8000616D4DB48C4
:10D440000DF13B01D0F800020D90B888ADF838001E
:10D45000B8798DF83A00002002F042FB000605D4AE
:10D4600015A9042002F03CFB000601D52068BEE7A8
:10D470002022312168462DF079F852208DF80000E5
:10D48000BDF83410CA4816AB4A46085C8DF8010056
:10D490009DF83610C748415C8DF802109DF8371092
:10D4A000415C8DF803109DF83810415C8DF8041034
:10D4B0009DF83910405C8DF80500DDF83B00CDF893
:10D4C0000600DDF83F00CDF80A00DDF84300CDF896
:10D4D0000E00D8F80410CDF81210B8F80800ADF816
:10D4E0001600D8F80A100691B8F80E00ADF81C0026
:10D4F000BDF85400010A8DF81E108DF81F0031216F
:10D50000684618F004FC9DF8580030707946206891
:10D5100029606CE72DE9F0438DB0804601208DF83D
:10D52000000017468946072000F024FD9B4C0006AA
:10D5300026D40CA800F0F2F9000621D49DF83000A2
:10D54000974E10F08C0F974D4FF092004FF0020164
:10D5500003D19DF83120B42A06D02060784631608E
:10D56000286092200DB043E709A9002002F0B8FA24
:10D57000000605D407A9052000F061FC000601D5CE
:10D580002068EFE72022162101A82CF0EFFF53209E
:10D590008DF80400B8F80010ADF8051098F80200F6
:10D5A00009AB8DF8070093E8070002AB83E807009A
:10D5B000079805909DF820008DF8180015216B46FE
:10D5C0004A4601A818F0A3FB92289DF80000387085
:10D5D00003D0794620682960C4E7002020603060CD
:10D5E000784628600020BDE7F0B506468BB00720DE
:10D5F00000F0C0FC694C00067ED40AA8F8F70DFCC8
:10D60000000679D49DF82800654D664F40B1912001
:10D6100020609C2028607846386091200BB0F0BDD7
:10D6200009A800F07BF9000672D49DF824004FF0A1
:10D63000020110F08C0F4FF0920003D19DF82520CD
:10D64000AC2A05D020607846296038609220E5E752
:10D650006D4601A818F043FF000659D4684618F03B
:10D660006FFF000654D4E91D002002F039FA0006CD
:10D670004ED47068CDF813003089ADF81700D6F895
:10D680000A00CDF81900F089ADF81D00042008A9A2
:10D6900002F026FA00063BD44FF00040F8F762F99A
:10D6A000000635D405F047F9000622D49DF8240081
:10D6B000000704D4684601F099FA000619D400F076
:10D6C00001FF000615D43C4D01213B4805F04FF900
:10D6D00000060AD5F2F7BAFD00F080F9000608D47A
:10D6E000F2F7C9FD2078000603D400F027FF0006FA
:10D6F00006D504F0F7FC00E00AE0F8F72EFA8DE713
:10D7000095F800010028DFD1F8F792F9000601D55D
:10D71000206883E7012005F0A1F87FE72DE9FF41AC
:10D7200080462E208DF800000F46072000F022FCD6
:10D730001A4C00061DD4FF2002F04FFA000618D440
:10D7400002A8F8F76AFB000613D49DF80800144EEF
:10D75000144D48B1912020609C20306078462860AC
:10D76000912004B0BDE8F08101A800F0D7F80006D0
:10D7700001D52068F5E79DF804004FF0020110F094
:10D780008C0F4FF0920003D19DF80520B42A15D0DC
:10D7900020607846316028609220E2E7080000109F
:10D7A0000C00001010000010A0C907209CC7072023
:10D7B00032B9030002C1030048C6072054208DF887
:10D7C0000C0001216B46424603A818F0A0FA9228EB
:10D7D0009DF80000387003D0794620682960C0E7C2
:10D7E000002020603060784628600020B9E770B5DE
:10D7F00006460D46072000F0BDFB364C000604D45B
:10D80000FF2002F0EAF9000601D5206870BD294624
:10D81000304601F0C1F930490020206008607846A8
:10D820002E490860002070BD0EB501218DF804104E
:10D830004A218DF800108DF80100022101AB02AAE7
:10D84000684618F064FA0106224801D500680EBD4A
:10D8500000210160204801607846204908600020CE
:10D860000EBDFEB5074604208DF80800072000F025
:10D8700081FB184C000624D4684600F04FF80006DF
:10D880001FD49DF80000144D10F08C0F134E4FF074
:10D8900092004FF0020103D19DF80120B42A05D077
:10D8A00020607846296030609220FEBD4B208DF8C4
:10D8B0000400012102AB3A4601A818F028FA00063C
:10D8C00001D52068FEBD00202060286078463060C9
:10D8D0000020FEBD080000100C0000101000001019
:10D8E00070B5FF48002404704470C470012018F023
:10D8F0007AFA0106FB4801D5006870BDFA4A9168C2
:10D9000042F2107395686D1A9D42FBD30460F7488C
:10D9100004607846F6490860002070BD2DE9F043A8
:10D920008DB0074639208DF82800F2A00024006849
:10D93000EC4EDFF8B8830325A1460B908DF82450F8
:10D9400009AB6A4602210BA818F0E1F9D8B1D8F862
:10D950000000052800D214B120280CD018E08DF862
:10D96000245009AB6A4601210AA818F0D0F9000634
:10D970000ED40124E2E708A9002000F060FA8DF837
:10D980002190002CDAD19DF82400022804D00BE06D
:10D9900030680DB0BDE8F0839DF800008DF82000E0
:10D9A0009DF801008DF821009DF8200038709DF849
:10D9B00021007870D0489DF8201000F82A1F9DF8AB
:10D9C00021104170C64901208870C6F80090784641
:10D9D000C749C8F8009008600020DAE71CB50620A7
:10D9E0008DF80000C5480178012059B1BC490022DA
:10D9F00001AB0A704A708DF804000121684618F0E6
:10DA000086F91CBDB74A88211160B849086078467C
:10DA1000B749086088201CBD2DE9FC41054600205F
:10DA200005218DF80410B5498DF80000AF4E097836
:10DA3000AF4FAC4C81B1AA496B46B14A0870012185
:10DA400001A818F064F900060FD5F2F7FFFBFFF705
:10DA5000C5FFF2F710FC13E0882020600120306041
:10DA6000784638608820BDE8FC8125B19DF800002B
:10DA70006D1EA84206D1A2499DF8000081F8000160
:10DA80002068F0E7922020602020306078463860DF
:10DA90009220E8E72DE9FF5F24208DF8080003A914
:10DAA000002000F0CCF98F4D00067DD49DF80C00CD
:10DAB0008E4E8F4F00074FF0920804D42620C5F8F1
:10DAC0000080306042E04FF0000B8DF804B001ABF5
:10DAD0008B4A012102A818F01AF9000672D4192005
:10DAE000FFF79AFF00066DD485494FF027090878A3
:10DAF000072802D0FFF772FF24E0DFF8FCA10C46F4
:10DB0000AAF1040A504651F8012F40F8302F4A6814
:10DB100042608A688260CA68C0F812200A7C8275F6
:10DB2000D1F81120C260B1F8151001820F20FFF763
:10DB300073FF000646D4FFF751FF000642D4207859
:10DB4000082809D0C5F80080C6F8009078463860EB
:10DB5000922004B0BDE8F09F5046D4F8061040F87B
:10DB60004E1F61898180607B217BDFF88C8100EB17
:10DB70000120A8F84800607800F00F01000900EBD0
:10DB8000800001EB40008DF80000A07800F00F014C
:10DB9000000900EB800001EB40008DF80100E07807
:10DBA00000F00F01000900E00CE000EB800001EB49
:10DBB00040008DF8020008F144016846F2F70FFFBB
:10DBC000000601D52868C4E7607900F00F0100095C
:10DBD00000EB800001EB4001207900F00F0200090A
:10DBE00000EB800002EB4000C0EB001001EB800175
:10DBF000A8F846103A490120C870C5F800B0784628
:10DC0000C6F800B038600020A3E72DE9F0438BB0E0
:10DC1000054639208DF820003AA04FF00008006832
:10DC2000304C324E1B27C146CDF824008DF81C70B5
:10DC300007AB6A46022109A818F069F890B130686C
:10DC400005283AD2B8F1000F37D18DF81C9007ABF8
:10DC50006A46012108A818F05AF800062DD44FF0A2
:10DC60000108E3E79DF801009DF80010052300EB93
:10DC7000012028800622A91C0DF10200F2F7DEFD2A
:10DC800000061AD405230622E91D02A8F2F7D6FDE4
:10DC9000000612D40523062205F10C010DF10E0039
:10DCA000F2F7CCFD000608D40523062205F1110188
:10DCB00005A8F2F7C3FD000602D520680BB069E69F
:10DCC0000D481622294614302CF056FB0449012039
:10DCD0004870C4F8009078460549C6F8009013E0F3
:10DCE000AA00001008000010008000400C00001086
:10DCF00010000010070300004CC707208AC1030072
:10DD000048C607200702000008600020D6E72DE97A
:10DD1000F04389B0044639208DF81C00F8A04FF07C
:10DD200000080068F74DF84E1527C146CDF82000D1
:10DD30008DF8187006AB6A46022108A817F0E7FFB5
:10DD400090B1306805285DD2B8F1000F5AD18DF836
:10DD5000189006AB6A46012107A817F0D8FF000605
:10DD600050D44FF00108E3E79DF8050000F00F01E3
:10DD7000000900EB800001EB40008DF814009DF8D5
:10DD8000060000F00F01000900EB800001EB4000ED
:10DD90008DF815009DF8070000F00F01000900EB59
:10DDA000800001EB40008DF81600211D05A8F2F758
:10DDB00016FE9DF80900042300F00F01000900EB96
:10DDC000800001EB40019DF8080000F00F020009FF
:10DDD00000EB800002EB4000C0EB001001EB800084
:10DDE000E080052221466846F2F728FD000609D4A6
:10DDF00004231A4604F108010DF10A00F2F71EFD92
:10DE0000000602D5286809B0C4E5DDF80E00E06020
:10DE10009DF8120020749DF81300607414222146AE
:10DE2000BA482CF034FBBA4901200870C5F80090BC
:10DE30007846B849C6F8009008600020E3E72DE96D
:10DE4000F0470546B248B14EDFF8BC82DFF8C49215
:10DE5000AC4F0C46052D05DC0078B8B93046FFF70D
:10DE600056FF07E00A2D08DC407878B9A74814303F
:10DE7000FFF7CBFE000621D408E0112D04DCC078AA
:10DE800020B9FFF707FEF5E7122D0FD09F48001FBE
:10DE9000132D66D2DFE805F01517191B1E21252763
:10DEA0002D30353840454A4E51545A00807890BB49
:10DEB00096482A30FFF732FD000647D53868BDE89E
:10DEC000F087707C44E0406805E0008900E040890C
:10DED00020803EE0C06820603BE001692160007D59
:10DEE00005E0B08A24E0D0F81A102160807F20710C
:10DEF0002FE050F81F1F16E0416A216090F82800BB
:10DF0000F5E750F8291F0EE0016B2160416B61605D
:10DF1000806BA0601DE019E0C16B2160B0F840008B
:10DF200012E050F8421F21600079E0E7B6F84400A3
:10DF300020800EE0B6F84600FAE7B6F84800F7E7AA
:10DF400050F84E1F21608088A08002E096F82B00D8
:10DF50002070002038607946C8F80000C9F8001029
:10DF6000ADE7922025213860C8F800107946C9F83D
:10DF70000010A4E7664AC3074FF0000100D01170FB
:10DF80008307002B01DA517000E000D09170400748
:10DF900000D5D1705B4801605B48016078465D49FF
:10DFA0000860002070471CB501208DF800005AA0C1
:10DFB0006B46006801900022022101A817F0A7FE1D
:10DFC0001CBD30B597B0044608208DF84C0053486E
:10DFD00001250078002855D02022492168462CF0E0
:10DFE000C5FA8DF8005034F8031B4D48484A13AB6E
:10DFF000085C8DF8010014F8011C4A48415C8DF85A
:10E0000002102178415C8DF803106178415C8DF835
:10E010000410A178405C8DF805006068CDF806001A
:10E02000A068CDF80A00E068CDF80E002069CDF8B0
:10E030001200A08AADF81600D4F816000690608B86
:10E04000ADF81C00B4F81D00000A8DF81E00607FBA
:10E050008DF81F0010208DF8200033A00168CDF846
:10E0600021104068CDF8250031218DF829100020BD
:10E07000107050709070D07014AA684617F047FE68
:10E0800017B030BD1F49882008601F4805607846DA
:10E09000204908608820F3E77FB504461F48012522
:10E0A000007858B309208DF80000208802A9F2F703
:10E0B0004AFC9DF808101B48415C8DF801109DF842
:10E0C0000910415C8DF802109DF80A10405C8DF833
:10E0D0000300608801A9F2F78BFD20798DF8060016
:10E0E0000B4900200246087048708DF80C5003ABB5
:10E0F0000721684617F00BFE04B070BD1AE000005F
:10E1000007010000080000100C0000104CC7072099
:10E11000AA00001010000010080100008AC10300CE
:10E1200032B9030002C10300465072696E742D318A
:10E1300031000000FA4988200860FA4805607846F6
:10E14000F94908608820D7E71CB5012039218DF8EE
:10E150000410F6498DF80000097831B16B460022B1
:10E16000012101A817F0D3FD1CBDED4A88211160E3
:10E17000EC4908607846EC49086088201CBD1CB555
:10E1800001200A218DF80410E8498DF80000097873
:10E1900051B1E74900200246087048706B460121E2
:10E1A00001A817F0B4FD1CBDDD4A88211160DD49CE
:10E1B00008607846DC49086088201CBDFEB50E4624
:10E1C000002521218DF800108DF8085004232946E0
:10E1D0000DF10102F2F7F0FAD14C000625D402ABA2
:10E1E000D44A0521684617F092FD00061DD4D14F90
:10E1F00035600020FFF710FC000616D4206848B1F7
:10E20000C848C949326892B12560056078460860FF
:10E210000020FEBD39780B29EBD1042303223146BF
:10E22000781DF2F70BFB0006E3D52068FEBD9222B5
:10E23000226027220260784608609220FEBD2DE908
:10E24000FC41BA49B74EB84F0978B54DB9B1A021D4
:10E250008DF80010010A8DF801108DF80200B44805
:10E26000002401AB047011208DF80400B14A032191
:10E27000684617F04CFD000609D5286809E4882097
:10E28000286001203060784638608820F6E7A94889
:10E29000102180F8001104742C60784634603860D6
:10E2A0000020EBE7FEB5A1499E4E9F4F09789C4D9B
:10E2B000D1B1A1218DF800100024042321460DF1D5
:10E2C0000102F2F779FA00060CD4994802AB994A98
:10E2D000047011208DF808000521684617F017FD1D
:10E2E000000609D52868FEBD88202860012030601E
:10E2F000784638608820FEBD8E48102180F80011D5
:10E3000004742C607846346038600020FEBD2DE92E
:10E31000FF4188468549834E834F0978804D29B156
:10E32000A2218DF804105AB104210AE08820286047
:10E330000120306078463860882004B0BDE8F08164
:10E3400005218DF805106946F2F7FDFA9DF80000E9
:10E35000794C6946205C8DF806009DF80100205C30
:10E360008DF807009DF80200205C8DF808004046FB
:10E37000F2F7E9FA9DF8000003AB6E4A205C8DF8D5
:10E3800009009DF801000821205C8DF80A009DF825
:10E390000200205C8DF80B006548002404701120F9
:10E3A0008DF80C0001A817F0B2FC000601D5286812
:10E3B000C3E76048102180F8001104742C6078468F
:10E3C000346038600020B8E7FEB5584B554D564EC6
:10E3D0001B78534C6BB142F20F73984201D89942AB
:10E3E0000FD9862020601320286078463060862070
:10E3F000FEBD88202060012028607846306088209B
:10E40000FEBDA2238DF800300AB1062200E00722EB
:10E410008DF80120020A8DF802208DF80300080A09
:10E420008DF8040042488DF8051000270770112070
:10E430008DF8080002AB3F4A0621684617F067FCDA
:10E44000000601D52068FEBD3A48102180F8001171
:10E450000774276078462F6030600020FEBD2DE9EC
:10E46000FC4132492F4E304F09782D4DB9B1A321CF
:10E470008DF80010010A8DF801108DF802002C486B
:10E48000002401AB047011208DF80400294A0321F7
:10E49000684617F03CFC000609D52868EEE688209F
:10E4A000286001203060784638608820E6E6214800
:10E4B000102180F8001104742C60784634603860B4
:10E4C0000020DBE62DE9FC41A4208DF8040017486C
:10E4D000144E154F0078124D78B1154800246B4644
:10E4E000047011208DF80000124A012101A817F0D4
:10E4F0000EFC000609D52868C0E6882028600120A7
:10E500003060784638608820B8E60A48102180F8E4
:10E51000001104742C607846346038600020ADE649
:10E52000080000100C000010100000108AC1030049
:10E53000AA00001048C6072002C103002DE9FC41D3
:10E5400005208DF80400FD48FD4EFE4F0078FE4C7E
:10E5500098B1FE4800256B4605708DF80050FC4AC6
:10E56000012101A817F0D3FB00060ED5F1F76EFECE
:10E57000FFF734FAF1F77FFE18E0882020600120D1
:10E58000306078463860882078E69DF8000048B111
:10E59000102807D092202060202030607846386014
:10E5A00092206BE6EA4981F800010D54206865E687
:10E5B0002DE9FF410446E148E34DE1490278E14895
:10E5C000012782B12278012A14D0022A14D0032A0A
:10E5D0002ED0042A2ED086222A6006220A6079468E
:10E5E00001608620A9E688222A600F6079460160D2
:10E5F0001046A2E6102000E011208DF80000207BDC
:10E600008DF801006E464FF0000804234146B21C0D
:10E610006068F2F7D1F8000608D4A0680523B21D9F
:10E6200044460021F2F7C8F8000605D5286884E6BC
:10E630001220E2E71320E0E7C4486A4603AB047007
:10E6400044708DF80C700B21104617F060FB74E6D7
:10E650002DE9FF410446B948BB4DB9490278B94894
:10E6600001279AB118228DF800202278012A14D0AF
:10E67000022A14D0032A2ED0042A2ED086222A6001
:10E6800006220A6079460160862056E688222A60C2
:10E690000F607946016010464FE6102000E011201F
:10E6A0008DF80100207B8DF802006E464FF00008C7
:10E6B00004234146F21C6068F2F77EF8000608D495
:10E6C000A0680523F21D44460021F2F775F8000604
:10E6D00005D5286831E61220E2E71320E0E79B48E1
:10E6E00003AB0022047044708DF80C700C21684656
:10E6F00017F00DFB21E6FEB59049934E01250978F0
:10E7000071B116218DF80010002400680523214600
:10E710000DF10102F2F750F800060AD53068FEBD8F
:10E7200088203060864805607846864908608820E1
:10E73000FEBD864802AB0022047044708DF808507C
:10E740000621684617F0E3FAFEBDFEB57B497E4E12
:10E750000125097889B118218DF8001016218DF84E
:10E76000011000240068052321460DF10202F2F792
:10E7700023F800060AD53068FEBD88203060704856
:10E78000056078466F4908608820FEBD6F4802AB7F
:10E790000022047044708DF808500721684617F075
:10E7A000B6FAFEBDFEB56549674E0125097871B11F
:10E7B00017218DF8001000240068052321460DF173
:10E7C0000102F1F7F9FF00060AD53068FEBD882086
:10E7D00030605B48056078465A4908608820FEBD75
:10E7E0005A4802AB0022047044708DF8085006218C
:10E7F000684617F08CFAFEBDFEB55049524E012511
:10E80000097889B118218DF8001017218DF80110B1
:10E8100000240068052321460DF10202F1F7CCFF28
:10E8200000060AD53068FEBD882030604448056087
:10E830007846444908608820FEBD444802AB002267
:10E84000047044708DF808500721684617F05FFA8D
:10E85000FEBD2DE9F04104463848394E394F007865
:10E86000394D86B08846E8B3208802A9F2F76BF8E4
:10E8700019208DF800009DF808103648415C8DF88D
:10E8800001109DF80910415C8DF802109DF80A10E6
:10E89000405C8DF80300608801A9F2F7A9F920799E
:10E8A0008DF806002948002405AB04704470082048
:10E8B0008DF8140003AA0721684617F028FA00060D
:10E8C00012D404231A46414603A8F1F7B7FF000605
:10E8D0000AD40423032208F1040104A8F1F7AEFFCF
:10E8E000000600E003E00AD5286806B026E5882087
:10E8F000286001203060784638608820F5E72C6079
:10E900007846346038600020EFE72DE9FC5F0D4663
:10E910000A490D4C0A4E09780A4F00296BD0232171
:10E920008DF80010010A8DF801104FF000098DF8E4
:10E9300002008DF8049001AB054A0DE08AC1030086
:10E940000C0000101000001008000010AA000010B9
:10E9500048C6072002C103000321684617F0D7F913
:10E96000000643D4DFF868830020FFF755F800065F
:10E970003CD498F8001129B198F80000092801D07A
:10E980001028F1D1FFF72AF800062FD498F80011CB
:10E99000404671B3027805F10A0A092A05F10F0B06
:10E9A0004FF005034FF00602294638D0C01CF1F79E
:10E9B00045FF00061AD4C64805230622691D093002
:10E9C000F1F73CFF000611D4C14805230622514649
:10E9D0000F30F1F733FF000608D4BD4805230622A7
:10E9E00059461530F1F72AFF000636D52068BDE8F4
:10E9F000FC9F08E0FFE78820206001203060784617
:10EA000038608820F3E7142128462BF0B7FD9220C8
:10EA1000206027203060784638609220E7E708F1D0
:10EA20000100F1F70BFF0006E0D405230622691D63
:10EA300008F10700F1F702FF0006D7D4A448052328
:10EA4000062251460D30F1F7F9FE0006CED4A0485B
:10EA50000523062259461330C4E7C4F800907846CF
:10EA6000C6F8009038600020C1E72DE9FE430F464C
:10EA70009849994DDFF864820978DFF8649229B3E8
:10EA800023218DF80010010A8DF801108DF8020085
:10EA900000268DF8086002AB8D4A0321684617F006
:10EAA00036F900060FD48A4C0020FEF7B5FF0006A9
:10EAB00009D494F8000110B120780E28F4D1FEF7A3
:10EAC0008DFF00060BD52868BDE8FE838820012154
:10EAD0002860C8F800107946C9F80010F4E794F8E7
:10EAE0000001E8B3E07800F00F01000900EB8000BE
:10EAF00001EB40008DF80400207900F00F010009BF
:10EB000000EB800001EB40008DF80500607900F01B
:10EB10000F01000900EB800001EB40008DF80600BA
:10EB2000394601A8F1F75BFFE07900F00F01000919
:10EB300000EB800001EB4001A07900F00F0200091A
:10EB400000EB800002EB4000C0EB001001EB800006
:10EB50007880207A38712E607946C8F8006000E02D
:10EB600003E00020C9F80010AEE73E609220BE80AE
:10EB700027212860C8F800107946C9F80010A3E7DB
:10EB8000102101605449002008605449086078460B
:10EB900053490860002070477CB50C4602218DF86F
:10EBA000001055218DF80410024601216B4601A882
:10EBB00017F0ADF848494A4A484B50B192280BD05B
:10EBC0009DF8000020709220086078461060922026
:10EBD0007CBD444D012028709DF80000207000206D
:10EBE000086018607846106000207CBDF0B597B0D2
:10EBF000044608208DF84C003648374D374E0078D3
:10EC0000374F00285CD02022492168462BF0AEFC0B
:10EC100051208DF8000034F8031B3348085C8DF850
:10EC2000010014F8011C3148415C8DF80210217874
:10EC3000415C8DF803106178415C8DF80410A17877
:10EC4000405C8DF805006068CDF80600A068CDF83E
:10EC50000A00E068CDF80E002069CDF81200A08A05
:10EC6000ADF81600D4F816000690608BADF81C00C5
:10EC7000B4F81D00000A8DF81E00607F8DF81F009B
:10EC800010208DF82000AFF660300168CDF821101B
:10EC90004068CDF82500164831218DF82910002450
:10ECA000047044708470C47013AB14AA684617F0E3
:10ECB0002EF82C60784634603860002017B0F0BD24
:10ECC0008820286001203060784638608820F5E789
:10ECD00048C607208AC10300080000100C0000107D
:10ECE0001000001002C0072032B9030002C1030067
:10ECF000AA000010F0B54178FD4AFE4BFE4C962567
:10ED000009B1192903D902201560186015E00526FC
:10ED10000E2916D006DC052913D0062911D00D299D
:10ED200004D10EE00F290CD019290AD0F34F007836
:10ED3000795C884209D015601E6078462060962074
:10ED4000F0BD0078801E3128F5D2002010601860D8
:10ED5000784620600020F0BD2DE9F04F0120E44A04
:10ED6000E44BE54C0225E54F4FF032094FF00E0A17
:10ED70004FF00D0B4FF006084FF00A0E4FF0070C46
:10ED800003261A286AD2DFE800F0691112171A2543
:10ED9000292D3135393D4115154552560D5A5E62C2
:10EDA000211D664587F812B01320EAE77E70BD701A
:10EDB0000320E6E731212EE0FD700420E1E73D71FC
:10EDC0000520DEE787F817801820DAE787F8168035
:10EDD0001720D6E787F805900620D2E787F8069037
:10EDE0000720CEE787F807A00820CAE787F808A021
:10EDF0000920C6E787F809C00A20C2E787F80AC0D9
:10EE00000B20BEE787F80BB00C20BAE787F80CE0C0
:10EE10000D20B6E700213954401C1928B1D9002033
:10EE200010601860784620600020BDE8F08F87F8F9
:10EE300010801120A5E787F811E01220A1E787F8DC
:10EE400013C014209DE787F814C0152099E7052109
:10EE50007975162095E73E76192092E78F2010608D
:10EE600078461E6020608F20DFE72DE9F04F95B0D7
:10EE70004FF040584046012212A9CDF834801CF0D2
:10EE80000DFE9B4C00066AD408F10100012211A975
:10EE90000D901CF003FE000661D499494FF0010962
:10EEA000962781F800909DF84800924D924EFF28D9
:10EEB00005D057280AD04846276028600FE09DF803
:10EEC0004400FF28F7D107202760F6E79DF84400AB
:10EED0004FF0030A802807D02760C5F800A07846C5
:10EEE0003060962015B0A0E70DA8F7F713FE0006D6
:10EEF00035D40FA8F7F71FFE000630D440461CF0AB
:10EF0000E4FDA0F1010850460D994FF0060AB0EB60
:10EF1000117FE1D121F070414145DDD20F9AB0EB74
:10EF2000127FD9D122F070404045D5D20229D3D3E7
:10EF30000228D1D3DFF8CCB10F990D9888422AD09E
:10EF4000022269461CF0AAFD000608D49DF80000C4
:10EF5000FF2806D06846FFF7CDFE000603D52068DF
:10EF6000C0E78DF800900F990D98884207D29DF860
:10EF7000002002448A4202D9052027609DE79DF8BF
:10EF80000010084420F070410D904145A4D8D3D121
:10EF9000CDF834B0D0E74FF000002060286078460C
:10EFA00030604FF000009DE7FEB54FF040573C4603
:10EFB00038461CF08AFD5449461820461CF08BFD4B
:10EFC00005466846F7F7B7FD494C000621D400987E
:10EFD000B84219D020F0704101F56C312A4601A8E1
:10EFE00000912BF0BFF80199491C6943B14201D34C
:10EFF000B81C03E0A1F56C3141F040500090684628
:10F00000F7F78FFD000604D46846F7F779FD000690
:10F0100001D52068FEBD3749002020600860784691
:10F02000354908600020FEBD1CB53548304C0078DD
:10F0300088B11AF0F2F808B1344800E03448009082
:10F0400048F25700ADF80400022201A900981CF014
:10F0500030FD00060BD42B4800906846F7F750FDB2
:10F06000000604D46846F7F75CFD000601D5206869
:10F070001CBD204900202060086078461E490860B9
:10F0800000201CBD1E48007870472DE9FC41064653
:10F090000D464FF040501CF018FD441E1848144F08
:10F0A0004FF00008007860B16846F7F733FD0006BE
:10F0B00004D401A8F7F73FFD000607D53868BDE87E
:10F0C000FC81C6F80080C5F8008009E0A41E2C6011
:10F0D000DDE90010401A306002D52968084430602C
:10F0E0000449C7F800807846C1F80080024911E061
:10F0F000080000100C00001010000010A4C9072028
:10F10000B000001002000030FFAF030000B003B0F9
:10F11000009005B008600020D1E71CB500200090E9
:10F12000019001A96846FFF7B0FF000603D40098DC
:10F1300008B100201CBD01201CBD2DE9FC4180460A
:10F140000024FB48009401940078FA4EFA4FFB4DDE
:10F1500038B101A96846FFF798FF000608D528686E
:10F16000ADE7052028607846346038600520A6E7C2
:10F17000DDE90010411A08EBC80202EB0810B1EB00
:10F18000400F07D29620286004203060784638600F
:10F19000962094E72C6078463460386000208EE733
:10F1A00010B54078E54C0B281AD008DC01280ED0A9
:10F1B000022815D009280CD00A2806D109E00C280D
:10F1C0000ED0102805D0112803D0182002E0782096
:10F1D00000E00F20FFF7B1FF000603D5206810BD47
:10F1E0000C20F7E7D3490020206008607846D24918
:10F1F0000860002010BD2DE9F04F044693B04FF099
:10F2000040501CF062FCA0F1010AC948C94FDFF868
:10F2100028830078C94E002500287DD010A94920F8
:10F220000CF038F9000678D49DF84000032873D01C
:10F23000022811D160781A286ED2DFE800F08E0D16
:10F240000D0D0D0D0D0D0D8E8E0D8E0D0D8E0D8E69
:10F250000D0D0D8E0D0D8E0D2046FFF7A1FF000642
:10F260006FD4607808B1192809D99620306003203E
:10F27000794638609620C8F8001013B0D5E5DFF85D
:10F28000C0920E280ED006DC052817D0062815D00F
:10F290000D2804D106E00F2855D0192853D019F8AD
:10F2A000000018E004F110002AF0F0FF202802D935
:10F2B00084F83050202099F80D100AE004F1110074
:10F2C0002AF0E4FF202802D984F83150202099F850
:10F2D00005102038084420706846F7F72CFC00061B
:10F2E0002FD4009820F07041AAEB010921788346C1
:10F2F00049450DD9FF22322102A82BF037F94A46A1
:10F3000002A958461CF0D5FB00061AD48D4800907F
:10F3100022782146009801E01FE012E01CF0C9FBB2
:10F3200000060ED420780099084420F07041009027
:10F33000514501D1834800906846F7F7F2FB00067B
:10F340000BD5306899E7A01C2AF0A0FF202802D92D
:10F3500084F822502020C01CBDE7356079463D600E
:10F360000020C8F8001088E72DE9F84F07464FF055
:10F3700040501CF0AAFBDFF8B8B1461E6F4C9BF85A
:10F380000000DFF8B081DFF8B09100254FF0050AEA
:10F39000F0B16846F7F7CFFB000631D4DBF8043054
:10F3A00000998B4214D03222394618461CE0DBF813
:10F3B00004105846491CCBF8041021F07041B142AA
:10F3C00001D160494160DBF804000099884209D10D
:10F3D000C4F800A07946C8F800500520C9F800100C
:10F3E000BDE8F88F322239461CF058FB000607D4DE
:10F3F0003878FF28DBD03846FFF77CFC000601D5C3
:10F400002068EDE73978DBF804201144CBF80410CC
:10F4100021F07041B14202D14A49CBF80410256075
:10F420007946C8F800500020C9F80010D8E72DE947
:10F43000F14FDFF8FC800027404C98F800003D4D6C
:10F440003D4E8EB0B9464FF0050A00286FD00DA88A
:10F45000F7F771FB000637D44FF040501CF035FB36
:10F46000A0F1010B70E0022269461CF017FB0006B8
:10F470002AD49DF80000FF2814D09DF8011005291A
:10F480001DD006291BD00B2919D0D8F804204146DD
:10F49000104420F07042C8F804005A4517D0D8F83C
:10F4A000040016E0D8F80400401C20F07042C8F8B0
:10F4B00004005A4548D12348C8F8040044E068468F
:10F4C000FFF752FF000610D520680FB0ADE41D48CD
:10F4D000486020F07041594507D9962020600620E9
:10F4E0002860784630609620EFE79DF801000128FB
:10F4F00003D0052801D0062804D19DF80020D8F8B3
:10F5000004108F1A052803D0062801D00B281BD120
:10F51000BDF80A100E98814216D1C8F80470C4F8DC
:10F5200000907846C5F8009030600020CDE710E0EC
:10F53000B00000100C0000101000001008000010B7
:10F54000A4C9072002000030D8F804000D998842B1
:10F5500089D1C4F800A07846C5F800903060052035
:10F56000B3E7F0B5BD48BE4EBE4F0078BE4C87B085
:10F570000025A8B3B948001DF7F7CCFA00062CD433
:10F5800001A81FF0CCFA000627D4694621200CF010
:10F590004CF8000621D49DF80000ADF8040069463F
:10F5A0001F200CF042F8000617D49DF80000ADF8BB
:10F5B0000A00694626200CF038F800060DD49DF8A4
:10F5C0000000ADF80C001FF03BFB000605D4002145
:10F5D00001A81FF021F800060AD5206807B0F0BD89
:10F5E000FFE7052020607846356038600520F5E7A4
:10F5F00025607846356038600020EFE72DE9F84354
:10F60000964E974FDFF85C823078974C002560B1BA
:10F610006846F7F74FF9000663D47078B8B11FF069
:10F62000E0FA000609D575705BE005202060794698
:10F630003D60C8F80010BDE8F8832068052854D064
:10F640008648001DF7F75CFA00064AD47570DFF8AB
:10F650001C928648FFF788FE000642D42068D8B97D
:10F660009DF8000017281AD0152818D0192816D090
:10F6700099F801001A28ECD2DFE800F00D0E0E0E0A
:10F680000E0E0E0E0E0D0D0E0D0E0E0D0E0D0E0E9F
:10F690000D0D0E0E0D0EDCE720680528CBD05B208B
:10F6A0000BF08DFD00061CD499F80100062809D046
:10F6B00004DC022806D0052817D103E00B2801D06E
:10F6C000122812D15C200BF07AFD000609D49DF8B7
:10F6D0000000172801D0182807D11FF065FA00068E
:10F6E00001D52068A7E701207070256079463D604C
:10F6F0000020C8F800109EE770B505465748002165
:10F70000574A03785748584C8EB0002B3ED0AB0B6D
:10F710003CD057A01FF0EEF8000634D4002159A0C9
:10F720001FF0E8F800062ED4280411D5FFF719FFC2
:10F73000000628D4FFF762FF20680028FAD01FF0E7
:10F740007FFA00061FD401201EF0E1FF00061AD444
:10F7500053200BF034FD000615D4012003F07EF891
:10F76000000610D4FFF760FC00060CD40F256E468F
:10F770008DF801503EA1B01C2AF064FD6846FFF7E9
:10F780003AFD000608D520680EB070BD21601160FA
:10F79000794601600020F7E78DF8015039A1B01CCF
:10F7A0002AF050FD6846FFF726FDEDE72DE9F05FF2
:10F7B0002A4C16468B464FF0010A012803D0606898
:10F7C00010F0405F05D1254884F802A0001DF7F72E
:10F7D000A1F9DFF88C80DFF88C90234DA078012808
:10F7E0000DD1224F2148FFF7BFFD000613D4286832
:10F7F000052813D078781528F4D01828F2D0254899
:10F800003146C0893060A278584609F001FA0700F5
:10F810000DD0052F0BD02868BDE8F09F9120AD21B9
:10F820002860C8F800107946C9F80010F4E7584677
:10F830003168F1F730FA67B184F802A03068002827
:10F84000CCD0002028607946C8F80000C9F8001024
:10F85000E2E7A078401CA070F0E70000B0000010C4
:10F860000C00001010000010080000109CCA0720B7
:10F870008E9888818A80208693908D808B80208AC4
:10F880008B0A000086E3E0ADA0AB20AEE7A8E9A5B7
:10F89000AD0A00008C0400102DE9FF470220039000
:10F8A00016F0BEFA0024FD48FD4EDFF8F8934470D0
:10F8B0008460254603274FF03208C4608DF8047039
:10F8C0008DF8055003AB02AA022101A8CDF80080F3
:10F8D00016F06BFB000603D5306804B0BDE8F08776
:10F8E0009DF808009DF8091000EB012009EB450187
:10F8F0006D1C8886032DE1D3EB48346004607846A4
:10F90000EA4908600020E8E7E64A02EB4000808E02
:10F910000880E34900200860E34908607846E3492D
:10F9200008600020704708B569460220FFF7ECFF29
:10F930000106DB4801D5006808BDBDF80030DA4992
:10F94000DA4AB3F57A7F07D2932303600B2008606D
:10F9500078461060184608BD0023036078460B60A7
:10F960001060184608BD2DE9FF418846CB4D0221A5
:10F9700003910124E968CB4A8440C94F0C4202EB51
:10F9800040061CD104218DF804108DF805003220AA
:10F99000009003AB02AA022101A816F006FB0006A4
:10F9A00003D5386804B0BDE8F0819DF808009DF8E3
:10F9B000091000EB01207087E8680443EC60718F48
:10F9C000A8F80010B8490020386008607846B749A8
:10F9D00008600020E6E73EB5044641208DF80400AB
:10F9E0000C2002903220009002AB2246012101A897
:10F9F00016F0DBFA0106AA4801D500683EBDA7490A
:10FA00008A6842F080028A60A64922681439CA6373
:10FA100062680A64A2684A6400210160A248016029
:10FA20007846A249086000203EBD0EB570B101289D
:10FA30000ED002281DD09A49882008609A490D20CE
:10FA4000086078469949086088200EBD102200E0C1
:10FA50000522121D019209228DF808208DF8090057
:10FA600032200A46009001AB022102A816F09DFA4E
:10FA70000EBD0A22EDE70EB50022029210228DF88B
:10FA800004208DF805008DF80610080A8DF807008F
:10FA9000322001AA009002AB0421104616F085FA2C
:10FAA0000EBD38B504466946FFF75DFF7C4A000687
:10FAB00001D5106838BDBDF8001039B1491E89B2B2
:10FAC000ADF800102046FFF7D6FF38BD0520764977
:10FAD000106000200860784674490860052038BD31
:10FAE0002DE9FE4F0D466D496E4E81466E4FDFF893
:10FAF000BC81143E6A4C88684FF0930A4FF0070BA4
:10FB0000B9F1050F59D2DFE809F0301818034F009A
:10FB10008946800742D40120FFF7C3FF98BB6149A3
:10FB200001201431FFF781FF000643D4D9F80810F3
:10FB300041F00201C9F8081030E0C0070DD1FFF70D
:10FB4000B0FF00BB57490020FFF76FFF000631D41C
:10FB50005248816841F001018160B9F1050F2CD252
:10FB6000DFE809F00A12161C2200000604D46846D9
:10FB7000FFF731FF00061DD4F06B2860306C686021
:10FB8000706CA86022E015E0B0692860B08B03E0DB
:10FB9000D6F81E002860708CA88017E0F06A2860F4
:10FBA00096F83000287111E029460220FFF7DBFEAD
:10FBB00000060BD52068BDE8FE8FC4F800A079468A
:10FBC000C7F800B09320C8F80010F4E700202060C8
:10FBD00079463860C8F80010EDE730498A688243FA
:10FBE0008A60CA688243CA602D49002008602E4995
:10FBF000086078462D490860002070472DE9F04FD5
:10FC0000264D042289B08046284F0026DFF89890C0
:10FC1000234C28466A704FF0860A4FF0010B0229E8
:10FC200009D0032907D0042922D0052920D0082192
:10FC3000C4F800A043E0067003291FD01CE0174859
:10FC4000A9701730F5F7C3FB14481030F5F7BFFB68
:10FC50001248124D00781E3590B1A5F800B0B8F8E2
:10FC60000010A980A5F802B0B8F80200E8801FE0F3
:10FC700080F800B0052901D00021E0E70121DEE78E
:10FC8000B8F800002880AE80B8F802106980EE80D5
:10FC900088420DD91321C4F800A010E0B80000106C
:10FCA00008000010D2C907200C000010100000103E
:10FCB000A888E98888420AD91421C4F800A07846A7
:10FCC000C9F800103860862009B0BDE8F08F694699
:10FCD0000220FFF748FE000669D4DFF814844FF0D5
:10FCE000810A98F8000020B92888BDF800108842E1
:10FCF0006CD82888401E81B20220FFF7BCFE0006A7
:10FD000079D402A90220FFF790FE206838B10528B7
:10FD10000AD09328D8D1D9F800100829D4D198F85E
:10FD2000001079B120B10DE098F80000F0BB11E0AF
:10FD3000BDF80830AA88934204D3BDF80A00288091
:10FD4000AB8010E00143DCD1BDF80800A88098F832
:10FD5000000040B96888BDF80010884200D9084604
:10FD6000ADF800006880BDF80000401E81B202209E
:10FD7000FFF781FE00063ED402A90220FFF755FEE0
:10FD8000206828B193289FD1D9F8001008299BD169
:10FD900098F8001061B158B9BDF80820EB889A4274
:10FDA00006D8BDF80A00688090B219E00EE022E0A3
:10FDB000014313D0BDF80000401E80B2ADF8000032
:10FDC00029888142CFD998F8000050B1C4F800A02A
:10FDD0007846C9F800603860812075E7BDF80800F2
:10FDE000E8802888401E81B2A8F804100220FFF79E
:10FDF00042FE000601D5206866E726607846C9F80D
:10FE00000060386000205FE72DE9F047B84DDFF86B
:10FE1000E492DFF8E4826878B84C002720B1032828
:10FE200019D004280FD107E0052020607946C8F8D2
:10FE30000070C9F8001051E54F200BF0C0F9000622
:10FE40004AD40320687027607946C8F80070002003
:10FE5000C9F8001042E50026A9490220FFF7E5FD98
:10FE6000932804D1D8F80000082835D10126A888A5
:10FE7000401C80B2A880A97836EA010110D0522037
:10FE80000BF09DF9000627D41EF0DAFE000623D4FD
:10FE9000812020607946C8F80070C9F800101DE57F
:10FEA0002168052904D092491E314988814202D235
:10FEB0006F70502017E08EB991498D48091D1030A0
:10FEC000F5F727FB000607D48D498948093117301B
:10FED000F5F71FFB000601D52068FFE4A87800288D
:10FEE000B9D026B15220BDE8F0470BF068B95120D7
:10FEF000F9E700B587B0002106918DF804003220A3
:10FF000001AA009006AB0121104616F04EF807B08A
:10FF100000BD70B588B003004FF00000774D0E466D
:10FF200007900ED0012B0ED0022B0ED088207249E4
:10FF300028600D20086078466E490860882008B067
:10FF400070BD102402E0052400E00A24012098403E
:10FF5000241DFFF742FE000601D52868EFE70820C0
:10FF60008DF804008DF80530224631460DF106006B
:10FF70002AF002FA322001AA009007ABA11C104619
:10FF800016F013F8DBE77CB50C4605466946FFF72B
:10FF9000EAFC5A4B000605D401A92846FFF7B4FC39
:10FFA000000601D518687CBDBDF80400BDF800103E
:10FFB000401A2080504900201860086078464D495A
:10FFC000086000207CBD7FB5054615208DF808002F
:10FFD0000420039032200C46009003AB01AA0121BB
:10FFE00002A815F0E2FF0106444802D5006804B0FB
:10FFF00070BDBDF804102980BDF8061021800021D5
:020000040001F9
:1000000001603D48016078463A4908600020EEE70B
:100010000EB50222029216228DF804208DF80500FA
:1000200041F288300A46009002AB022101A815F087
:10003000BCFF0EBD00B587B00021059140218DF8B1
:1000400004100168CDF805104168CDF809108068EA
:10005000CDF80D00264801AA05AB816821F080018A
:100060008160322000900D21104615F09EFF4EE772
:1000700070B58CB0064680208DF824001E200A90B2
:1000800032200D4600900AAB01AA012109A815F003
:100090008CFF1A4C000608D4BDF8040028801C22EE
:1000A0000DF1060130462AF067F920680CB070BDEA
:1000B0003EB504460220029081208DF804003220D3
:1000C00001AA009002AB0121104615F06EFF010657
:1000D0000A4801D500683EBDBDF80410218000210A
:1000E00001600548016078460249086000203EBD75
:1000F000B8000010100000100C00001008000010E4
:10010000BEC90720F0B54478FD49FE4AFE4BA22542
:100110000CB1192C03D902200D60106015E00526E2
:100120000E2C16D006DC052C13D0062C11D00D2C6D
:1001300004D10EE00F2C0CD0192C0AD0F34F00780C
:100140003C5DA04209D00D60166078461860A22080
:10015000F0BD0078801E3128F5D2002008601060C4
:10016000784618600020F0BD2DE9F04F0120E44AE8
:10017000E44BE54C0225E54F4FF032094FF00E0AF3
:100180004FF00D0B4FF006084FF00A0E4FF0070C22
:1001900003261A286AD2DFE800F0691112171A251F
:1001A000292D3135393D4115154552560D5A5E629E
:1001B000211D664587F812B01320EAE77E70BD70F6
:1001C0000320E6E731212EE0FD700420E1E73D71D8
:1001D0000520DEE787F817801820DAE787F8168011
:1001E0001720D6E787F805900620D2E787F8069013
:1001F0000720CEE787F807A00820CAE787F808A0FD
:100200000920C6E787F809C00A20C2E787F80AC0B4
:100210000B20BEE787F80BB00C20BAE787F80CE09C
:100220000D20B6E700213954401C1928B1D900200F
:1002300010601860784620600020BDE8F08F87F8D5
:1002400010801120A5E787F811E01220A1E787F8B8
:1002500013C014209DE787F814C0152099E70521E5
:100260007975162095E73E76192092E78F20106069
:1002700078461E6020608F20DFE738B54FF04040A1
:1002800000906846F6F75EFC9D4C000604D4684674
:10029000F6F769FC000601D5206838BD99490020B1
:1002A00020600860784698490860002038BD2DE934
:1002B000FC4119F08DF8934E934F914D002438B3C3
:1002C0009349012008706846F6F746FC000604D4FE
:1002D00001A8F6F752FC000602D52868BDE8FC81AB
:1002E0004FF040401BF0F1FB009A0C21401EB1EB97
:1002F000127F0BD122F07042824207D2019AB1EBF9
:10030000127F03D122F07041814201D3FFF7B5FF84
:100310002C607846346038600020DFE7FEB54FF08F
:10032000404528461BF0D1FB7A49471828461BF068
:10033000D2FB06466846F6F720FC714C000621D435
:100340000098A84219D020F0704101F508313246DA
:1003500001A8009129F006FF0198401C7043B842A3
:1003600001D3009504E0A0F5083040F04040009033
:100370006846F6F7F8FB000604D46846F6F7E2FB99
:10038000000601D52068FEBD5E490020206008609F
:1003900078465D4908600020FEBD5D4800787047E2
:1003A0002DE9FC4105460C464FF040401BF08DFB0B
:1003B000461E5748524F4FF00008007858B1684623
:1003C000F6F7CAFB000604D401A8F6F7D6FB000630
:1003D00006D5386882E7C5F80080C4F8008008E0D8
:1003E0002660DDE90010401A286002D52168084423
:1003F00028604449C7F800807846C1F80080424927
:10040000086000206AE72DE9FC418046002440484E
:100410000094019400783B4E3B4F394D38B101A90F
:100420006846FFF7BDFF000608D5286856E7052097
:10043000286078463460386005204FE7DDE9001019
:10044000411A08EBC80202EB0810B1EB400F07D2CB
:10045000A22028600420306078463860A2203DE762
:100460002C60784634603860002037E710B540785B
:10047000234C0B281AD008DC01280ED0022815D0F6
:1004800009280CD00A2806D109E00C280ED0102823
:1004900005D0112803D0182002E0782000E00F20BA
:1004A000FFF7B1FF000603D5206810BD0C20F7E769
:1004B0001449002020600860784613490860002035
:1004C00010BD2DE9F04F044693B04FF040401BF0B3
:1004D000FCFA471E0E48DFF82C90DFF82CA00078BD
:1004E000074E002500287DD010A962200AF0D2FF17
:1004F000000678D49DF84000C00773D020460BE07A
:10050000080000100C0000101000001012CA072094
:1005100054C10720FF1F0200FFF7A8FF000671D497
:10052000607808B1192809D9A22003213060C9F8E0
:1005300000107946CAF8001013B07EE6DFF8D482C6
:100540000E280ED006DC052817D0062815D00D2859
:1005500004D106E00F2857D0192855D018F800000C
:1005600018E004F1100029F091FE202802D984F847
:100570003050202098F80D100AE004F1110029F005
:1005800085FE202802D984F83150202098F80510E3
:100590002038084420706846F6F7EFFA000631D498
:1005A00000982178834620F07040A7EB0008414571
:1005B0000ED9FF22322102A829F0D8FF424602A913
:1005C00058461BF076FA00061CD44FF040400090CD
:1005D0002278214600981BF06CFA000612D420788D
:1005E000009901E01AE00DE00844009020F070400E
:1005F000B84202D14FF0404000906846F6F7B3FA97
:1006000000060BD5306897E7A01C29F03FFE202894
:1006100002D984F822502020C01CBBE735607946FF
:10062000C9F800500020CAF8001085E72DE9F84FFE
:1006300007464FF040401BF048FADFF8DCB1461E99
:10064000764C9BF80000DFF8D881DFF8D8910025C0
:100650004FF0050AF8B16846F6F78FFA000632D473
:10066000DBF8043000998B4215D032223946184607
:100670001DE0DBF804105846491CCBF8041021F0AB
:100680007041B14202D14FF040414160DBF80400BB
:100690000099884209D1C4F800A07946C8F80050F2
:1006A0000520C9F80010BDE8F88F322239461BF04A
:1006B000F5F9000607D43878FF28DAD03846FFF776
:1006C00021FD000601D52068EDE73978DBF804202C
:1006D0001144CBF80410B14203D14FF04041CBF8A4
:1006E000041025607946C8F800500020C9F80010B1
:1006F000D9E74948007818B14748001DF6F72CBAE9
:10070000464905200860464900200860784645496A
:100710000860052070472DE9F04FDFF8FC803F4C62
:100720003F4E98F800003F4F8FB000254FF005096D
:1007300078B30DA8F6F721FA00060DD44FF0404A21
:1007400050461BF0C2F9A0F1010B1DE002226946E0
:100750001BF0A4F9000602D520680FB06DE59DF8E6
:100760000000FF2805D025607846356038600020FD
:10077000F3E7D8F80400401C20F07042C8F80400E9
:100780005A4501D1C8F804A0D8F804000D99884250
:10079000DCD1C4F800907846356038600520DCE78D
:1007A0002DE9F8431C4E1E4FDFF8788030781B4C43
:1007B000002560B16846F6F77DF8000620D4707811
:1007C00088B11EF00EFA000609D5757018E00520F4
:1007D000206079463D60C8F80010BDE8F8832068C5
:1007E00005280FD075701048FFF720FF000607D4CA
:1007F00020680528F1D06A200AF0E1FC000601D546
:100800002068EAE7256079463D600020C8F80010BE
:10081000E3E7000012CA072054C1072008000010B7
:100820000C000010100000109CCA07202DE9F84FA2
:10083000054600794C4C4D4FDFF83481862608B1CF
:100840001E2802D9052026604AE0288848F6AD61B6
:100850004FF0140A884203D92660C7F800A040E090
:1008600068884FF0170BB0F5B46F03D32660C7F854
:1008700000B036E06846F5F7BFFF000667D4288869
:10088000BDF80010401A4FF4B46148435FEA000914
:10089000E2D46846F5F7C0FF000658D46888BDF872
:1008A0000010411A11EB090FE0D432490120F5F78D
:1008B000BFFD00064BD430490220F5F7B9FD000614
:1008C00045D468790F380D2808D2DFE800F0101001
:1008D00010101007101010100710100008202660CC
:1008E000386079468620C8F80010BDE8F88F2846A1
:1008F000F5F725FB00062AD4A81CF5F731FB000606
:1009000025D4281DF5F73DFB000620D4681DF5F71A
:10091000C7FF00061BD4002568460095F6F70EF8C1
:10092000000614D468460095F6F717F800060ED4B2
:100930000120ADF800006846F5F7D9FF000606D49F
:10094000ADF800506846F5F7E3FF000601D52068D2
:10095000CBE7032009498DF80000022008706846A3
:10096000F5F7A9FAC1E70000080000100C0000101C
:100970001000001064C1072069C1072000000010AA
:100980002DE9F04F91B005A8F5F794FFF94C00065A
:100990007ED46846F5F7B5FF0006F9D4DFF8D8A392
:1009A0004FF010014FF002099AF800004FF00008D4
:1009B00002074FF0010734D59DF81400A0F10E0294
:1009C0000E2A6DD2DFE802F007070F0F0F1C076C2D
:1009D0006C6C6C6C6C0F8AF802008DF8141009E0D6
:1009E000ADF800905CE0BDF80010032958D1401C20
:1009F0008DF8140005A8F5F753FF0006C8D4EFE7FB
:100A0000BDF8000003284BD19AF802008DF81400BD
:100A1000554605A8F5F744FF0006B9D4ADF8009097
:100A20003CE0554640063BD59DF814000E2804D006
:100A30000F2802D0102833D115E0BDF80020042A79
:100A40002ED18AF802008DF8141005A8F5F728FFBA
:100A500000069DD41420ADF800006846F5F747FF66
:100A6000000695D41CE0BDF80000032818D1ADF8AD
:100A700000706846F5F74CFFA8788DF8140005A8BB
:100A8000F5F70EFF000688D40420ADF8000000E062
:100A90005BE26846F5F72BFF0006AFD485F80080CF
:100AA0009DF81420B54DB64E88214FF0640B4FF0E1
:100AB00010401B2A71D2DFE812F070009604400645
:100AC0004006400640061D061D061D061D061D06A5
:100AD0001D061D061D061B001B00BF02F1037C0343
:100AE0005D04E7047B067B067B067B0670007D04C5
:100AF000BDF800200A2A7AD007DCDBD2DFE802F05A
:100B00004D1A51F29BBDD3E2F3F9DFF878B25A2ABD
:100B100067D008DC0B2A7DD00C2A7CD0392A7BD008
:100B2000402A3AD116E25B2A77D0642A76D0B42ADA
:100B3000F7D124E0904912200AF0ACFC000688D4DA
:100B40009AF80010012001F048018AF8001001F025
:100B500085FE000685D49DF814000E280DD1694647
:100B600062200AF097FC00068DD49DF80000C007B3
:100B700003D0F0F79DF9000685D4B4202DE07E491E
:100B80006920491C0AF086FC000686D49AF8010008
:100B9000000603D501F012FF6FE2CFE2ADF800903E
:100BA000F6E001F00EFF0006C9D40EA92E200AF0CF
:100BB00071FC0006C3D49DF814000E2805D00F2840
:100BC00010D19DF8380080070CD5FCF765FA0006B7
:100BD000B5D42068052805D00A20ADF80000D7E07C
:100BE00005E0FFE0042050E2ADF80070F1E30020E2
:100BF000FCF7BFFA0006A2D4206800286FD00EA927
:100C00002E200AF047FC000699D49DF814000E2807
:100C10000BD004E083E05CE0D5E033E1BEE00F28D8
:100C2000E0D19DF838008007DCD56B200AF0C7FAC8
:100C3000000684D4D6E70FA969200AF0F6FC000666
:100C400088D49DF83C00C00603D401F03CFF0006A8
:100C50008AD46846F5F766FE000685D4BDF8000024
:100C6000042801D2401CF5E3ADF800706846F5F7A2
:100C70004FFE000689D40520AFE701F021FF0006F2
:100C800092D46846F5F74EFE00068DD4BDF80000FC
:100C90000228E7D3ADF800706846F5F739FE000684
:100CA00088D4062099E701F011FF000690D4684629
:100CB000F5F738FE00068BD4BDF800000428D1D328
:100CC00007208AE71B200AF07AFA000693D40C204A
:100CD00083E701F0F2FE00068DD408207DE75AE09C
:100CE00007E000E01FE001F0E5FE00068CD40920DB
:100CF00073E701F0DCFE000686D40EA92E200AF070
:100D0000C9FB000695D49DF814000E2805D00F28C5
:100D10007ED19DF8380080077AD50B205DE7022050
:100D2000FCF727FA24E201F055FE000688D40EA94C
:100D30002E200AF0AFFB00068AD49DF814000E287E
:100D400005D00F287DD19DF83800800779D50E4D4C
:100D500001206F811DF060FB00068BD456200AF045
:100D60002EFA000686D4A5F80A9002201DF054FB46
:100D7000FEE30000080000105CC107200C0000101A
:100D800010000010008000408C040010ADF800B08E
:100D90006846F5F7ACFD11B0BDE8F08F1DF021FFFE
:100DA000000688D42068052804D09DF814000E2879
:100DB00007D0E8E1C4F800807846C5F800803060CC
:100DC0000CE35A2009E7F4F7CDFD000684D4FAF7C6
:100DD000B1FA00067ED4F4F72BFE52E32760C5F883
:100DE000008025E16846F5F7B7FF000684D49DF83A
:100DF000000038B3F8484FF05B09007800283FF452
:100E0000CDAE6846F5F72BF800068FD4F34800E026
:100E100043E20078D8B19DF800001B2817D068463F
:100E2000F5F715FD000687D46F46B81CF5F720FDD1
:100E3000000692D4381DF5F72CFD00068DD46846C7
:100E400001E054E37BE0FDF727F9000685D469460D
:100E50000420FEF745FE000684D4BDF80000401CC7
:100E600080B2FDF7FCFA50B192286ED1EFF7EEF99F
:100E700013208DF800006846F4F7E7FFFEE3ADF8B5
:100E80000090DAE2D448007828B30121D44801F078
:100E90006EFD000685D4FDF751FB000696D4D048C0
:100EA00090F80001002885D16846F4F7D8FF0006C5
:100EB0008CD49DF800000E283DD06846F5F7C7FC9D
:100EC000000693D4DAF8081001919AF80C108DF806
:100ED000081001E062E139E0DAF80D10CDF80910F0
:100EE0009AF811008DF80D0004200DF10201FEF7B3
:100EF000F7FD000689D4BDF80200401CADF80200E1
:100F00001120FEF7F6FF00068DD469460220FFF798
:100F100000F8000687D41220FEF7EBFF000688D405
:100F20000220FEF7BEFD000688D469460220FEF7C7
:100F30007CFD00068AD4FBF79BFC000686D4DBF818
:100F400008104020CAF8041047E665E2A44981F879
:100F50000081A9E7DBF80810DAF80400081AA149B3
:100F6000884203D2A048007801289CD1C1468DF860
:100F700000806846F4F747FF00068BD4B846384631
:100F80000DF11C0BC0B207466946F5F751FA000691
:100F900084D4C7EBC70101EB0B0AAAF1070138465D
:100FA000F4F71AFF00068CD4AAF107006946F4F79B
:100FB000B0FA000685D47F1CF8B20428E2D907A84D
:100FC000F4F700FF000695D406A8F5F7C5FE000665
:100FD00090D49DF8180018B9F5F7DAFE000689D408
:100FE000694612200AF056FA00068DD49DF80000DA
:100FF00040070AD56846F4F7EAF9000684D4694642
:101000000120F4F744FF000684D4694662200AF008
:1010100041FA000688D49DF80000C00704D00020E3
:10102000EFF75CFF000685D4C4F80080C5F8009097
:10103000784630600120AEE6BDF80020172A7BD04C
:101040000EDC142A29D006DC012A76D0022A17D019
:10105000032A73D18FE0152A58D0162AF9D139E026
:101060001B2A4DD06BDC182A6BD0192A2CD01A2AD7
:10107000EFD17BE0642AECD1EFE3000688D48DE564
:1010800001F09FFC00068ED41420ADF800006846E5
:10109000F5F72DFC000686D4A6E501F0FCFC000661
:1010A00088D46846F5F73EFC00068CD4BDF80000F5
:1010B0001028FFF4D7ADADF800706846F5F728FCAE
:1010C000000685D4192088E501F0D9FC000686D4F5
:1010D000162082E501F0E5FC000686D46846F5F7A7
:1010E00021FC00068AD4BDF800001028E1D3ADF839
:1010F00000706846F5F70CFC000685D41B206CE5F3
:1011000001F0C3FC000685D4152066E501F0C6FC9D
:10111000000688D46846F5F705FC0006AED4BDF895
:1011200000001028C5D3ADF800706846F5F7F0FB55
:101130000006A3D4182050E509E0BDE0BDE0BDE005
:10114000FFE701F09FFC000698D4172045E501F069
:10115000ABFC000692D46846F5F7E4FB00068DD49C
:10116000BDF800001028A4D31A2036E501F090FC49
:10117000000688D46CE301F02DFC00068BD41DF032
:1011800013FD000687D4392027E500BFF4F7EAFBFA
:10119000000685D4FAF7CEF8000670D5F4F7DDFC2A
:1011A000F9E500068DD4F1E5206805287FF416AE38
:1011B00000E6BDF800201F2A4BD008DC012A7BD0B6
:1011C000022A13D0032AD6D01E2A76D114E0202A70
:1011D00029D0212A72D153E08AC10300DE00001019
:1011E00048C6072040420F009EC2072001F0E9FBDD
:1011F000000688D41E2048E701F035FC000688D49C
:101200006846F5F78FFB000688D4BDF80000182863
:101210007FF628ADADF800706846F5F779FB00065B
:1012200087D42020D9E401F024FC00068CD4684641
:10123000F5F778FB000687D4BDF800001828E7D939
:10124000ADF800706846F5F763FB000687D41F20F1
:10125000C3E401F00BFC00068BD46846F5F762FB93
:10126000000686D4BDF800001828D1D9ADF800706A
:101270006846F5F74DFB000684D42120ADE4AFE0CD
:1012800001F0FAFB000684D46846F5F74BFB000634
:1012900088D4BDF800001828BAD9D9E2BDF80020DA
:1012A000292A43D00BDC012A06D0022A0CD0032ABB
:1012B00089D0282A89D10DE0CDE017E179E02A2AEA
:1012C0001ED02B2A75D147E001F07BFB000690D49D
:1012D0002820DAE601F0BBFB00068AD46846F5F761
:1012E00021FB000685D4BDF800001E2890D9ADF87A
:1012F00000706846F5F70CFB000685D42A206CE4E4
:1013000001F0ABFB00068BD46846F5F70BFB00063B
:1013100086D4BDF800001E2891D9ADF8007068464B
:10132000F5F7F6FA000686D4292056E401F092FB80
:10133000000671D46846F5F7F5FA00066CD4BDF8DE
:1013400000001E2891D9ADF800706846F5F7E0FA64
:10135000000661D42B2040E401F082FB00065BD440
:101360006846F5F7DFFA000656D4BDF800001E28DF
:1013700092D96DE2BDF80020372A0BD02ADC012A71
:1013800069D0022A7FF464AE01F01BFB000643D44F
:1013900037207AE601F058FB00063DD46846F5F7A1
:1013A000C1FA000638D4BDF800002028FFF45AAC7A
:1013B0004EE20FE0BDF80020382A0FD00ADC012AE7
:1013C00049D0022ADED101F0FCFA000624D43820EC
:1013D00003E46FE1392A3FF4D9AE4BE60020DAE4AA
:1013E000F4F726FBDDE6BDF800003E2815D006DC4C
:1013F000012830D0022809D0032877D13FE03F28C8
:1014000075D0402828D0642870D10CE001F0D9FABA
:10141000000601D43E202FE479E001F05AFB0006DB
:1014200075D43F2028E41DF0DCFB00066FD4206853
:1014300005283FF4BDAE40207FE06846F5F757FA37
:10144000000664D4042020607846C5F8008030602F
:101450000420A0E42CE157E1FAF7F4F9000656D491
:101460000327ADF800706846F5F741FA00064ED440
:1014700027607846C5F80080306003208BE401F0D7
:10148000A9FA000643D4A9E4BDF8000009284FD00A
:101490000DDC2BD2DFE800F02A1D2CF33C090706F7
:1014A000050020E40EE4FFF7FEBBFFF7E6BB522881
:1014B0007ED007DC0C283FF40CAC502840D05128DB
:1014C00014D197E0532874D0542873D064280DD1D8
:1014D000C3E1E549122009F0DDFF000617D49AF8B0
:1014E000001001F008018AF800100DE175E15CE1DF
:1014F0008AF8008001F065FA000608D4ADF80070A3
:101500006846F5F705FA000601D4042006E481E0F8
:1015100001F0D9FA00067DD46846F5F703FA000613
:1015200078D4BDF800000428FFF49CAB0520ACE59E
:1015300001F0BDFA00066DD45020ADF800007CE744
:101540006846F4F78CFC000664D49DF800000E2871
:1015500035D06846F5F77BF900065BD4DAF8081059
:1015600001919AF80C108DF80810DAF80D1000E0CF
:1015700019E1CDF809109AF811008DF80D0004203A
:101580000DF10201FEF7ACFA000643D4BDF80200EB
:10159000401CADF802001120FEF7ABFC000639D468
:1015A00069460220FEF7B5FC000633D4122002E0A3
:1015B0003AE051E06BE0FEF79CFC00062AD4694655
:1015C000122009F067FF000624D49DF800004007B0
:1015D0000AD56846F3F7FBFE00061BD469460120D6
:1015E000F4F755FC000615D4FAF7D2F9000611D429
:1015F00051204AE56846F5F795F900060AD4BDF88A
:101600000000C0B20546FAF76BFA000602D4102DAE
:101610004CD300E077E0ADF800706846F5F778F954
:10162000000670D452208FE46846F5F77BF9000677
:1016300069D4BDF80000C5B22846FAF785FA00065D
:1016400061D40A2D32D3ADF800706846F5F760F921
:10165000000658D4532077E46846F5F763F900068E
:1016600051D4BDF80000C5B22846FAF713FA0006B7
:1016700049D41E2D1AD3ADF8007001E0D2E02BE062
:101680006846F5F745F900063DD454205CE4684609
:10169000F5F748F9000636D4BDF80000C0B205469B
:1016A000FAF7D2F900062ED4182D07D26D1CE8B235
:1016B000ADF800006846F5F72BF9BCE48DF8008022
:1016C0006846F4F7A0FB00061DD4FBF7D1F800062E
:1016D00019D4FBF7E1FC4BE50120FBF74AFD0006BE
:1016E00011D420680028E8D001F074F900060AD46B
:1016F000FFF72DBBBDF80000012805D0022807D058
:1017000063286AD10AE076E0012001F0A7F8B4E48A
:1017100001F057F900066ED4632015E4534890F8A1
:10172000000100283FF4AFAE0221504801F01FF93C
:10173000000660D4FCF702FF7DE4BDF800005C28E1
:1017400029D006DC012812D002281ED0032844D15B
:101750003CE05D2812D05E287FF4B8AE44480078A3
:1017600000283FF48CAC3C2009F029FD85E40120E1
:1017700001F074F8000675D45D20A4E43B2009F064
:101780001EFD00066ED45E209DE401F01AF90006ED
:1017900068D45C2097E4FEF737FB000662D420682B
:1017A000052855D004E500065CD41DF0FDF9F8E4E9
:1017B000BDF8000079281FD00BDC012814D00328C5
:1017C000CAD101201CF0A3FF00064BD401F002F99E
:1017D000E9E77A281BD07B282DD021607846C5F810
:1017E00000903060882026E4012001F037F80006E0
:1017F00038D4792067E417E05D2009F0E0FC0006AA
:1018000030D4FDF7AEFE00062CD47A205BE4FDF761
:10181000F5FE0028C6D0052807D0EEF717FD0120F9
:101820001CF075FFEEF727FD1CE01DF0BDF900066A
:1018300018D47B2047E41DF0D4F9000612D42068A8
:101840000528AFD09DF81400172803D0182801D020
:10185000032038E4FDF7A8FB8AE41DF0C2F9000676
:101860007FF5A2AC20689BE45CC1072048C6072036
:101870008AC103003EB54FF00040F4F773F82B4CDB
:10188000000609D401A8F5F715F8000647D4684604
:10189000F5F75DF8000601D520683EBD009800060A
:1018A0002ED49DF804000E2808D10120ADF80800C0
:1018B00002A91A20F5F705F8000630D46846F4F7B7
:1018C00015FB00062BD46846F3F7F4FE000626D479
:1018D0006846F4F701FB000621D469469DF8040030
:1018E000F4F7FCFF00061AD46846F3F7BCFE0006C6
:1018F00015D469469DF80400F4F7E3FF00060ED402
:1019000000248DF800406846F4F7CAFF000606D4AC
:101910008DF800406846F4F7CEFA000602D5F4F7D9
:101920001CF93EBDF4F784F83EBD0000080000102D
:101930002DE9F04F05460079D84CD94FD94E93B0D8
:101940004FF0860808B11E2804D90520C4F800808D
:10195000306017E0288848F6AD614FF0140B8842DC
:1019600005D900BFC4F80080C6F800B00AE0688856
:101970004FF0170AB0F5B46F0AD300BFC4F8008067
:10198000C6F800A078463860862013B0BDE8F08F16
:1019900008A8F4F731FF00067CD42888BDF8201091
:1019A000401A4FF4B46148435FEA0009DAD408A84A
:1019B000F4F732FF0006EFD46888BDF82010411A12
:1019C00011EB090FDAD4B8494FF0000A012081F871
:1019D00000A0B649F4F72CFD0006DDD4B44902207E
:1019E000F4F726FD0006D7D40520FEF7F6F800062A
:1019F000D2D408A8F5F7B0F90006CDD49DF82000A0
:101A00004FF0010B00287DD0AA4800780028FAD0BA
:101A1000FCF79AFB0BA90520FCF711FA0006BBD4D2
:101A20000FA90320FEF75CF80006B5D405220FA924
:101A30000BA828F0DBFB78B1422009F0C0FB0006C0
:101A4000AAD4012000F00AFF9220206031203060EB
:101A500078463860922098E7FCF7A5FA00069BD4F8
:101A600090480068232809D13F2009F0A8FB000610
:101A700092D49148018821F0020101800BA9002035
:101A8000FCF7DDF9000687D49DF82C00400602D54E
:101A9000012001E0A3E00020804608A90420FEF711
:101AA0001FF8000687D40BA90620FCF7C8F900062A
:101AB00093D4BDF82000BDF82C60401C864201D1B3
:101AC000012000E000208146B8F1000F13D1B9F1E8
:101AD000000F10D1761EB6B209A93046FCF7C5FF3B
:101AE00000067CD4BDF824002880BDF8260068805C
:101AF0009DF82800287108A90420FDF7F1FF0006D1
:101B00006DD400E06EE0BDF82000401CB04212D061
:101B10004E2009F054FB000661D4012000F09EFE27
:101B200000065CD48F2020605E4807210160784663
:101B300038608F2029E701A93046FCF7E6FE000651
:101B40004DD48DF820A0012711A93846F4F770FC78
:101B5000000644D407EB870101A80144052211A81F
:101B6000491F28F043FB10B18DF820B005E07F1C21
:101B7000042FE9D99DF8200060B350480680452025
:101B800009F01DFB00067CD4642009F018FB000658
:101B900077D4494801260DF10407018821F002019C
:101BA00001804248019901609DF808100171404888
:101BB000DDF8091001609DF80D10017106EB86003B
:101BC000C1193046491FF4F726FC000659D4761C8B
:101BD000042EF3D958EA090004D0334900E050E05C
:101BE00081F800B02846F4F7AAF9000649D4A81CE9
:101BF000F4F7B6F9000644D4281DF4F7C2F900063C
